:020000040800F2
:1000000000000220CD6A0008C16A0008C16A000829
:10001000C16A0008C16A0008C16A00080000000047
:10002000000000000000000000000000C16A00089D
:10003000C16A000800000000C16A0008C96A00081F
:10004000C16A0008C16A0008C16A0008C16A0008E4
:10005000C16A0008C16A0008C16A0008C16A0008D4
:10006000C16A0008C16A0008C16A0008991900083D
:10007000C16A0008C16A0008C16A0008C16A0008B4
:10008000C16A0008C16A0008C5080008C16A000802
:10009000C16A0008C16A0008C16A0008C16A000894
:1000A000C16A0008C16A0008C16A0008C16A000884
:1000B000E90A0008090B0008C16A0008310F0008AE
:1000C00041170008C16A0008C16A0008C16A000837
:1000D000710A0008FD0D0008C16A0008C16A000825
:1000E000C16A0008C16A0008C16A0008C16A000844
:1000F000C16A0008C16A0008C16A0008A91900089D
:10010000C16A0008C16A0008C16A0008C16A000823
:10011000C16A0008C16A0008C16A0008C16A000813
:10012000C16A0008C16A0008C16A0008C16A000803
:10013000C16A00080000000000000000C16A000859
:10014000C16A0008C16A0008C16A0008C16A0008E3
:10015000C16A0008C16A0008C16A0008C16A0008D3
:10016000C16A0008C16A0008C16A0008C16A0008C3
:10017000C16A0008C16A0008C16A000800000000E6
:1001800000000000C16A000800000000000000003C
:10019000C16A00080000000000000000C16A0008F9
:1001A000000000000000000000000000C16A00081C
:1001B000C16A0008C16A0008C16A0008C16A000873
:0401C000C16A000808
:10020000BFF34F8F0549064BCA6802F4E060034311
:10021000CB60BFF34F8F00BFFDE700BF00ED00E0F4
:100220000400FA05704700BF08B5FFF7E9FF00BFFB
:1002300000207047044B197802460B1E18BF01239B
:1002400001201370704700BF40000120124A9188BE
:10025000034648BA1880D18849BA5980118949BAE9
:100260009980518949BAD980918949BA1981D1892E
:1002700049BA5981118A49BA9981518A49BAD981B1
:10028000918A49BA1982D18A49BA5982128B51BAD4
:1002900016209982704700BF40000120024AD369AE
:1002A0000133D361704700BF40000120704700BF99
:1002B00000B5184BDB68C3F30223C3F1070C03F14D
:1002C000040EBCF1040F28BF4FF0040CBEF1060F62
:1002D0004FF0FF3E8CBF033B00230EFA0CFC21EADB
:1002E0000C010EFA03FE994022EA0E02431C41EA79
:1002F000020109D000F160400B0100F5614CD9B258
:100300008CF800135DF804FB024A0801C3B282F8BE
:100310002330F7E700ED00E02DE9F04182B0804A9C
:10032000866D156800230193C36D3468082202FAB4
:1003300003F12142804604D001680F68780700F17C
:10034000BB8078489840204205D0D8F800104A6910
:10035000170600F1A780744A9A40224205D0D8F8C7
:1003600000000168880700F1938010229A40224221
:1003700004D0D8F800000168090774D44FF0200CAD
:100380000CFA03F0204218D0D8F800402268D406B6
:1003900013D5B06098F8351005293CD0D8F8006026
:1003A0003768780340F1A1803668310340F1AC80B2
:1003B000D8F83C700FB14046B847D8F85430002BFD
:1003C0004ED0D8F85400C2071DD5D8F80040574980
:1003D000052288F835202668A1FB051526F00107BF
:1003E000A80A276004E0D8F800402268D30704D5A3
:1003F000019B013383420193F5D90026012188F83E
:10040000346088F83510D8F84C304BB3404602B011
:10041000BDE8F0411847D8F800703D6825F0160097
:100420003860D8F80040626922F080016161D8F834
:100430004030002B6ED0D8F80050286820F0080417
:100440002C60D8F85C203F219140B160D8F8503042
:100450000026012788F8346088F83570002BD5D144
:1004600002B0BDE8F081B260D8F800301F687A03AE
:1004700033D41A68D70503D4186820F0080119602E
:10048000D8F840700FB14046B847D8F85C3075E7EF
:10049000B260D8F8543043F00407C8F85470D8F864
:1004A0005C3062E7B060D8F8543043F00207C8F817
:1004B0005470D8F85C304EE7086820F004030B60F5
:1004C000D8F85C108A40B260D8F85420D8F85C3074
:1004D00042F00107C8F8547033E71B681B03CFD5FF
:1004E000D8F84870002FCED1CFE7336813F480706E
:1004F0007FF45EAF3468012124F01002326088F886
:10050000340088F8351053E7D8F84470002F7FF492
:1005100052AF52E7D8F84870002F8CD191E700BF56
:10052000000000200100800004008000B5814E1B07
:100530002DE9F04F0023784D784E794C83B003E0DD
:100540000133102B00F0C680D1F800C001229A4080
:1005500032EA0C0702EA0C0EF2D1D1F804C02CF0FA
:100560001007022F17D1DF0800EB870C03F00707F5
:10057000DCF820A04FEA87084FF00F0B0F690BFA49
:1005800008F907FA08F72AEA090847EA080ACCF83E
:1005900020A0D1F804C0D0F800B00CF003074FF051
:1005A00003094FEA430C09FA0CF807FA0CF72BEA97
:1005B000080A47EA0A0BC0F800B04F6827F0100994
:1005C00009F1FF37012F6FEA080814D8D0F808A006
:1005D000CF6808EA0A0B07FA0CF747EA0B09C0F8DC
:1005E00008904F68D0F804A0C7F300179F402AEA8C
:1005F000020217434760C26808EA02078A6802FAE3
:100600000CFC4CEA0707C7604A68D20098D500275F
:1006100001976A6C42F480476F646A6C23F00308A8
:1006200002F4804708F1804B01970BF59C3A019A40
:10063000DAF8089003F0030292000F279740B042C7
:1006400029EA070C19D0374FB84246D0364FB84286
:1006500049D0364FB8424CD0354FB8424FD0354FC5
:10066000B84252D0344FB8420CBF4FF006094FF099
:10067000080909FA02F24CEA020CCAF808C04F68ED
:1006800022686FEA0E08FF0354BF08EA02024EEA2E
:10069000020222604F686268BF0354BF08EA020288
:1006A0004EEA020262604F68A268FF0254BF08EA85
:1006B00002024EEA0202A2604F68E268BF0203F142
:1006C000010354BF08EA02024EEA0202102BE26064
:1006D0007FF43AAF03B0BDE8F08F012707FA02F2CA
:1006E0004CEA020CC9E7022707FA02F24CEA020CB4
:1006F000C3E7032707FA02F24CEA020CBDE704271E
:1007000007FA02F24CEA020CB7E7052707FA02F2F1
:100710004CEA020CB1E700BF003802400000024082
:10072000003C01400004024000080240000C02406E
:10073000001002400014024000180240836B93F83E
:100740003D1093F83E202129C8B2D2B228D02228E9
:1007500024D01968086820F480620A601968086863
:1007600040F400720A601968486820F480524A60B8
:10077000196848684FF0000C20F400624A60A3F842
:100780002AC0186C48B94FF0200C83F83DC093F88C
:100790003E1083F83E0040290FD07047202AD8D160
:1007A00019684A6822F400624A6019680020588576
:1007B0004B6843F44070486070477047836B18681B
:1007C000026800214FF0200C22F4806202605985FB
:1007D00083F83DC083F83E10196C41F01000186496
:1007E000704700BF836B1868016821F48061016065
:1007F000586B00225A850265996B4FF0200C0A65F0
:1008000093F83D0083F83DC083F83E20704700BF59
:100810002B4A0368904210B43DD0B0F1804F31D0E4
:10082000A2F57C44A0422DD004F5806C604529D00F
:100830000CF58062904225D002F57844A0422AD07F
:1008400004F5705C604521D00CF5806290421DD0AB
:1008500002F58064A04219D0A4F5983C604515D0FB
:100860000CF58062904211D002F58064A0420DD058
:1008700003608A68C2620968816201235DF8044BE3
:10088000436170474A6823F070031343CC6823F434
:1008900040732343ECE74C68CA6823F0700323439A
:1008A00023F44073134303608A68C2620C68846255
:1008B0000969016301235DF8044B4361704700BF80
:1008C00000000140694A136A19685868890701D510
:1008D00080064DD419685868490701D5000618D418
:1008E00019685868C90701D5410606D419685868BF
:1008F000890601D541017FD470471968C807F5D52D
:10090000116E6FF0010041F4803111661860136AB6
:10091000ECE7116EC90603D4106E40F40051116665
:10092000986810F4401F1ED1996B11F4401F02D03B
:100930009868400517D45968490514D49968906B94
:1009400001F0405101430ED1586820F080015960F8
:10095000106E20F480511166106EC00503D4116E24
:1009600041F0010010666FF00C011960136AB7E7DF
:10097000116EC90603D4106E40F4007111669968B7
:10098000906B01F04051014340D0D96C44F27C702F
:1009900089B200FB01F1C1F30F3C42F61F308445E0
:1009A000A2F868C059D942F62D418C4558D942F673
:1009B000E550844557D943F2C7218C4594BF4FF089
:1009C000030C4FF0040C92F85C0082F86AC0012816
:1009D0000DD0012182F85C10986820F00101996027
:1009E0009868C00726D54FF0000C82F85CC06FF005
:1009F00012011960136A6DE7516E6FF0200041F02B
:100A0000020151661860126A10607047D86A10F4CB
:100A1000700F1ED1586820F020015960106E20F42C
:100A200080711166106EC104AFD4116E41F00100E7
:100A30001066AAE7596821F0806020F02001596013
:100A4000106E20F4885C2CF0010141F0010010666A
:100A5000C9E79968480598D4DCE74FF0000CB2E785
:100A60004FF0010CAFE74FF0020CACE74000012063
:100A700010B40A4B0A4AD86ED3F8A410C4680C808C
:100A8000D96E4B684FF400744FF4806023F040033C
:100A90004B60946190615DF8044B70474000012009
:100AA000000402400F4B03F1C401DA6EC3F89C004E
:100AB00082B0C3F8A41093689B07FCD50088D0606F
:100AC00000210191D368019390680190019B5168C6
:100AD00041F040035360106840F04001116002B0E3
:100AE000704700BF4000012010B54FF080442369DB
:100AF000DB0706D5034841688847226922F00103D5
:100B0000236110BD000000204A4B1869C10700D4C2
:100B10007047494B93F8C6204AB193F8C72062B991
:100B200046494FF480508861013283F8C720414A1A
:100B3000136923F001011161704793F86A10481C92
:100B4000B2EB400F6DDB04296BD0122AECD910B444
:100B500093F85C4083B00022012C019255D0196AB1
:100B6000012083F85C008C68E20714D4344A354CC9
:100B700012688868A4FB0242940C04EB440240F023
:100B8000010088600192019C2CB10198421E0192E3
:100B9000019C002CF9D18868C40736D51A6E22F45E
:100BA000E06424F0010040F480721A664C6860052D
:100BB00005D5186E20F4405C4CF480521A661C6E09
:100BC00014F4805018BF586E4FF0000418BF20F086
:100BD00006006FF02202586683F85C400A60196ACA
:100BE00019484C6844F0806C4CF020024A60406820
:100BF000C20602D0154CA14207D18A6812F0405FAC
:100C000003D1886840F080448C600A4A002183F850
:100C1000C710136923F00100106103B05DF8044BA5
:100C200070470648416981F4805C4CF080518161D5
:100C30008BE700BF0004004040000120000002409C
:100C40000000002083DE1B43002301400020014000
:100C5000674B93F80121202A01D00020704710B57E
:100C6000644A212483F8014105294FF0400494612E
:100C700040F29380002800F09080013950FA81FC06
:100C800000F1FF3EAEEB0C04E1434FF4047211F0AF
:100C90000301A3F808214FF0020235D08646007800
:100CA000102804D183F80A019EF8000003229C1842
:100CB000012984F8080102F1010225D0022911D08E
:100CC0001EF8011F102906D19818013280F808116A
:100CD0009EF8001092B2541C1A4482F80811A2B275
:100CE000FC2A5AD81EF8011F102906D19818013283
:100CF00080F808119EF8001092B2541C1A4482F831
:100D00000811A2B2FC2A48D89EF8011010290EF151
:100D1000010006D19C18013284F808119EF80110D8
:100D200092B203EB020E541C84458EF80811A1B256
:100D300042D0FC2931D890F801E0BEF1100F06D165
:100D40005C18013184F808E190F801E089B24A1C8E
:100D500092B21944FC2A81F808E11ED890F802E00A
:100D6000BEF1100F06D19C18013284F808E190F80A
:100D700002E092B2511C1A4482F808E18AB2FC2ABD
:100D80000BD8C178102900F1030EB6D19C1801329E
:100D900084F80811C17892B2AFE7164A164CC3F82E
:100DA000E84000204FF0200C4FF4800183F801C18F
:100DB000A3F8EE00916110BD901C13FA80FC194459
:100DC0000D48C3F8E8000332A3F8EE20D3F8C8407A
:100DD000084A1020032381F808018CF80831E368E1
:100DE0004FF4800143F08003E3609161012010BD66
:100DF00040000120000802404801012070B54A4C23
:100E0000D4F8C8301A68D968950601D5880629D45F
:100E1000160601D50D0604D4500601D54A0619D48C
:100E200070BDD4F8E820511CC4F8E8101078586060
:100E3000B4F8EEC00CF1FF35AEB2A4F8EE60002EAF
:100E4000EED1DC6824F08002DA60D96841F040001D
:100E5000D86070BDD868202520F04006DE6084F898
:100E6000015170BD314DD4F80C22A8685B68111A8D
:100E7000DBB2882984F808320DD90025102BC4F87C
:100E80000C0284F8105284F81152C9D14FF0010CB1
:100E900084F811C270BD94F81162002E39D0022B73
:100EA0000FD0032B24D0102B16D194F81002002859
:100EB000B6D00026511C84F81162C4F80C121370CD
:100EC00070BD94F810525DB9012284F8115284F873
:100ED0001022C4F80C0270BD94F81052002D9FD05F
:100EE0000021C4F80C0284F8101284F8111270BDAD
:100EF00094F81022002A93D00529F1D990F805C062
:100F00008B1F9C45ECD1D4F8146206B1B047A860A1
:100F1000E6E7102BBAD094F81002002880D0561CB7
:100F2000C4F80C62137070BD400001200000002066
:100F3000F0B49C4BD3F8182295695169546893F822
:100F4000560210288AB04CD0C6B2402E49D0964FD7
:100F50000F40002F00F0F180A70500F17E8193483B
:100F60002840002800F02E8191480840002800F019
:100F70009481650540F191818E4F0F40002F40F024
:100F8000918193F85562B3F842C21FFA8CF1F0B226
:100F900021B3D3F83C526C1CC3F83C422F78176144
:100FA000B3F8426206F1FF3C1FFA8CF1A3F842123B
:100FB000B3F84252ACB28CB929280FD1506820F452
:100FC00080672826576093F855C293F856220CF094
:100FD00003010A43C3F8482283F855620AB0F0BC03
:100FE000704711F0011F44D0A00500F11D81724E21
:100FF0000E40002E78D06D4A2A40002A47D06C4F10
:101000000F40002F00F08A80650540F18780694A13
:101010000A40002A00F09F81A405DFD5D3F84402DE
:1010200093F85562212ED9D1B3F842128CB2002C1C
:1010300040F0B281042800F07582082800F0728226
:1010400010F5803F00F06E82D3F818727D6825F4A9
:10105000E0627A6093F855C293F856620CF0030090
:1010600006432021C3F8486283F8564283F855129C
:10107000B4E7514E0E40002E36D0A705BBD5D3F8AD
:101080005C02C7B21761494A2A40002AB7D14B4DCA
:101090000D40002D4AD0600548D5464E0E40002E2A
:1010A00000F01881A20599D5D3F84442B3F8421252
:1010B0008FB2032F00F0DA81B3F842C21FFA8CF22C
:1010C000022A00F0ED81D3F83C52D3F81822681CB4
:1010D0001669C3F83C022E70B3F842C20CF1FF311E
:1010E0008CB2A3F8424279E72F480840002882D00A
:1010F000A60580D593F85672F8B2D3F84472D3F8A7
:1011000048C293F85562222E00F0648100200190BD
:101110005769019792690192019A6CE7254D0D403C
:10112000002D7FF479AF0AB0F0BC70472148084029
:101130000028B7D10AB0F0BC704721480840002809
:101140003FF40DAFA6057FF50AAF93F855C254687A
:1011500024F4E0665660099750690990146844F0D9
:1011600001061660D3F81802099A0268ACF128014A
:1011700022F4806402295FFA8CF5046040F24D810C
:10118000D3F84872222F02D0222D7FF427AF0025FA
:101190004FF0200CC3F8485283F855C283F85652DA
:1011A0001CE700BF40000120020001000400100005
:1011B000800001000400010008000100400001005F
:1011C00010000100B34F0F40002F49D0600547D5F4
:1011D000B14E0E40002E48D193F85542B3F842125A
:1011E00088B2E7B200283FF4F9AED3F83C52126956
:1011F0006E1CC3F83C622A70B3F842C20CF1FF3493
:10120000A1B2A3F84212B3F8420285B2002D7FF4D6
:10121000E5AE2A2F7FF4E2AED3F818727A6822F492
:10122000806428267C60CEE693F85672402F00F04A
:10123000FF80D3F82802B0F5804F00F0BE80D3F8CD
:101240006862002E40F0FD80D3F85C62F71107F071
:10125000060C4CF0F0001061CDE693699369BDE691
:101260008D4D0D40002D3FF4B9AEA1057FF5B6AE12
:10127000B3F84242A1B200293FF4B0AED3F83C72B9
:101280001269781CC3F83C023A70B3F842C20CF100
:10129000FF35AEB2A3F84262A0E67F4D0D40002DAF
:1012A0003FF49CAEA4057FF599AEB3F842C21FFA95
:1012B0008CF100293FF492AED3F83C62741CC3F861
:1012C0003C4230781061B3F84222551EAFB2A3F809
:1012D000427283E693F85522222A7FF47FAEB3F858
:1012E0004262B0B203283FF6EEAE841E012CD3F862
:1012F0004472D3F8181240F24D810D68022F14BFCA
:1013000025F4806545F480650D60D3F81822566891
:1013100026F4E0605060D3F83C421769611CC3F8C2
:101320003C122770B3F842C20CF1FF35AAB2A3F801
:10133000422293F8556293F8564206F003073C4365
:101340002020C3F8484283F85502002093F8562223
:1013500083F8560242E693F85542B3F8407293F888
:101360005652D3F84462E2B2E8B2002F40F08D80CA
:10137000212A00F0238140287FF430AE222A7FF416
:101380002DAEB3F842128CB2002C00F0108193F80D
:101390005672402F00F08A81D3F83C42D3F818727D
:1013A000651CC3F83C5222783A61B3F842C20CF192
:1013B000FF36B0B2A3F8420210E693F85562D3F8B4
:1013C0005C72212E16BF47F0010707F0FE07FFB23F
:1013D000176110E6D3F8686216B9402800F00A8158
:1013E000D3F868622EB9D3F82802B0F5404F00F068
:1013F0000881B3F84262B0B2002840F0A88006909D
:1014000056690696976906970698106840F4007624
:1014100016600022C3F86822EDE52049C3F84412A3
:101420002026C3F8487283F8556283F85672D5E5D2
:10143000D3F8680298B9D3F85C6206F0FE0717612A
:10144000D9E5D3F86872012F7FF4D5ADD3F85C02EB
:10145000C61106F0060747F0F1001061CBE5D3F89E
:101460005C6246F00107F8B21061C4E5042C05D0B7
:10147000082C03D014F5803F7FF425AED3F8187202
:10148000396821F480653D601DE6212A3FF479AF7B
:1014900071E700BF40000100040001000000FFFFF1
:1014A000042C6DD0082C6BD014F5803F68D0D3F895
:1014B00018120F68022C14BF27F4806747F4806766
:1014C0000F6093F8555293F8562205F0030002433B
:1014D000C3F84822D3F83C62D3F81842771C21693C
:1014E000C3F83C723170B3F842C2D3F83C52D3F81F
:1014F00018020CF1FF3296B2A3F8426204696F1C25
:10150000C3F83C722C70B3F842C2D3F818120CF135
:10151000FF35AAB2A3F842224E6826F44074202078
:101520004C6010E7D3F81872796821F4E0667E60A9
:1015300038680025202240F400743C60C3F848520B
:1015400083F8552293F8562283F8565246E5B3F8AD
:101550004262B0B2012864D0B3F84272BEB2022E29
:1015600000F08C80106840F480671760D3F8186230
:101570000022029270690290B7690297029A48E7C6
:10158000D3F818521220C3F848022E6846F40074AB
:101590002C609FE7022F0D6800F0AF8025F4806675
:1015A0000E60D3F818120C6844F400670F60D3F88B
:1015B0001802436823F4806444600FE5042EB1D020
:1015C000082EAFD016F5803FACD0D3F8185269681A
:1015D00021F4E0626A6093F8556293F8560206F0CF
:1015E000030420432025C3F8480283F8567283F889
:1015F0005552F3E408965069089096690896089A3F
:10160000F9E4079657690797906907900798166855
:1016100046F480771760D3F868220132C3F8682255
:10162000E9E4042F18D0082F16D0BCF1120F13D004
:10163000D3F844721068022F14BF20F4806040F485
:1016400080601060D3F818620022059277690597D0
:10165000B0690590059ADCE6166826F48060106093
:10166000D3F81872002204927E690496B869049037
:1016700004983A6842F400763E60CAE6D3F84462C1
:101680001068022E3DD020F480661660D3F8180250
:10169000026842F400670760D3F818220026039618
:1016A0005069039097690397039AB2E6D3F868529A
:1016B00085B9D3F86402D3F81812D3F86042012830
:1016C00023D0C4F307270F61D3F868520135C3F85C
:1016D000685283E4D3F86822012A1ED0D3F86862E6
:1016E000022E7FF47BAC93F85502222821D093F888
:1016F000551221297FF472AC4EE645F480620A60EF
:1017000055E740F480671760C6E7E2B20A61D3F894
:1017100068620236C3F8686260E4D3F86072D3F896
:101720001852FAB22A61D3F868620136C3F86862C7
:1017300054E4D3F818120B6843F480740C604DE441
:1017400038B5914C9148D4F8182253695168034236
:1017500024D0C80522D5D4F8585213F4813F45F05F
:1017600001006FF48075C4F85802556100F0A18043
:10177000D4F8580213F4823F40F002056FF4007071
:10178000C4F8585250611BD113F4843F01D0C905ED
:1017900037D4D4F85812002940D138BD13F4813F12
:1017A00009D0CD05E4D413F4823FEDD0D4F858121B
:1017B0000029F2D032E013F4823FE5D0C805E8D525
:1017C00094F856C2B4F8421294F85552BCF1200F66
:1017D000E8B289B2D4F848526FD0D4F8585245F0E4
:1017E0000401C4F85812156845F400711160D4F86A
:1017F00018226FF48060506113F4843FC9D0D4F88C
:101800001822D4F858326FF4006543F00800C4F889
:1018100058025561D4F858120029BED094F855C228
:10182000ACF12902012A3DD994F85532602B4FF0D2
:1018300000051CBF202384F85532C4F8485284F8B0
:101840005652D4F81822136823F400651560D4F8B2
:10185000180201680A0549D5436823F4006545600C
:10186000D4F84C02002849D090F83510484A026557
:10187000022948D080214165FEF7B4FF94F8552233
:10188000282A8AD1D4F858526B0786D50020414BBC
:10189000C4F844322021C4F8480284F8551284F870
:1018A000560238BD00202821C4F8480284F8551299
:1018B000C7E713F4823F83D166E700298DD100F09A
:1018C000F701212903D0282887D1212D85D194F82B
:1018D0005552D4F844020428E9B21ED008281CD07E
:1018E000212933D06FF48065556185E794F855223E
:1018F000602A04BF202284F85522BFE7D4F85002A2
:101900000028B1D1BAE705684FF0050C80F835C062
:10191000286820F001032B60B0E72829E0D11D489A
:10192000C4F8440255686FF4806025F4E0615160AA
:101930005061156825F48061116000202022C4F8F0
:10194000480284F8552284F8560255E71148C4F835
:10195000440294F8555294F8561205F003000143DE
:1019600020254FF0000CC4F8481284F8555284F832
:1019700056C251686FF4806021F4E0655560506193
:1019800011680140116037E74000012000010100AB
:10199000E50700080000FFFF024BD3F85002FEF7F6
:1019A000BBBC00BF40000120024BD3F84C02FEF745
:1019B000B3BC00BF4000012010B45649564B4A69E1
:1019C00082F0800040F400048C61D9690131D96152
:1019D000B3F8C42090B2C4001FFA84FCACF5804177
:1019E0000AB288B293F86C12DC69002AB8BFCCF551
:1019F000804203EB410C01F1010101F03F0183F84A
:101A00006C12BCF97012B8BF12B2ACF87022521A44
:101A1000D3F8F0120A44D3F8F412C3F8F0228A4241
:101A200083B04DDAB3F8FA2202F1FF3C21211FFA0C
:101A30008CF2A3F8F812A3F8FA22002A62D0D3F8A5
:101A40000843D3F80C23A11AB1F5807F2AD131487D
:101A5000446984F4806C4CF0806282612F4A304883
:101A600030494FF000749461DA6EC3F89C00C3F8FB
:101A7000A41093689B07FCD54AF6AA200021D060E9
:101A80000191D468019493680193019B506840F0E0
:101A900040015160146844F04003136003B05DF8E6
:101AA000044B7047D3F80813CCB2043403EB440C56
:101AB000ACF80803D3F808030130C3F80803CDE7F6
:101AC000D3F804138A4215DDB3F8F82202F1FF3C83
:101AD00040F201211FFA8CF2A3F8FA12A3F8F822BF
:101AE000002AACD110494FF0210CC3E9BF41A3F843
:101AF000F8C2A4E7212440F2012CA3F8F842A3F88D
:101B0000FAC29CE7094940F2012CC3E9BF41A3F89E
:101B1000FAC294E70008024040000120000402409D
:101B2000D898000804010120B91B0008311B0008E7
:101B30001D4A92F81035112B00D970472DE9F0415C
:101B40001A491B4E48691B4D0133DCB282F810451F
:101B500080F4807206EB440742F080738B6197F843
:101B60000480697B41454FEA440711D83E446A7DB1
:101B70007679B24202D82C77BDE8F081AB690120BA
:101B800013F8361002F012FE0028F4D02E75F2E79A
:101B9000286910F83810002002F008FE0028E5D06F
:101BA00085F80C80E2E700BF4000012000080240F9
:101BB000D8980008000000201C4A92F8103503B99C
:101BC00070472DE9F0411A4841695C1EE4B281F486
:101BD000007545F00076122C82F8104586610FD80A
:101BE000144D154E05EB4407727B3F79BA424FEA1C
:101BF000440811D84544707D6D79A84202D83477E5
:101C0000BDE8F081B169012011F8351002F0CEFD78
:101C10000028F4D03575F2E73369002013F8371047
:101C200002F0C4FD0028E5D03773E3E7400001204F
:101C300000080240D898000800000020234B10B58F
:101C40004FF08062224C9A61D4F81405D4F818152C
:101C5000884226D0D4F81425D4F8180582421DD025
:101C6000D4F81835DAB2043204EB420CBCF814058F
:101C7000D4F81835013381B2C4F818351548A4F8E2
:101C80001C17FEF70FFF14494A6982F0200040F448
:101C900000138B61E1690131E16110BD4FF6FF7105
:101CA000ECE794F81E376BB90C48FEF7FBFE0A4AC6
:101CB000506980F0400141F480039361E169013192
:101CC000E16110BD0648FEF7EDFEF0E700040240BA
:101CD000400001205C070120000802400499000830
:101CE0000299000838B5224C94F81F27E36905468D
:101CF00052B1D4F8000338B1D4F8FC125A1A142A9D
:101D00002FD90023C4F80033D4F82007D4F80813DF
:101D1000D4F80C2301309142C4F8200723D0D4F822
:101D20000C33D9B2043104EB4102B2F80803D4F801
:101D30000C3301331FFA80FCC4F80C3300B2D4F822
:101D400024270C49288001320B4D086AC4F8242747
:101D5000C2F30E0405EB4403A0F800C00B6201209F
:101D600038BD8047CDE74FF0FF304FF6FF7CE6E708
:101D7000400001200000002040000020704700BF0C
:101D8000024B93F82B17017001207047400001208F
:101D9000002945D04B1E10FA83F1421E48F205037C
:101DA000002012F801CF80EA0C2010F4004F0CBF85
:101DB000400083EA400080B210F4004F0CBF4000A6
:101DC00083EA400080B210F4004F0CBF400083EA69
:101DD000400080B210F4004F0CBF400083EA400086
:101DE00080B210F4004F0CBF400083EA400080B284
:101DF00010F4004F0CBF400083EA400080B210F4A2
:101E0000004F0CBF400083EA400080B210F4004F46
:101E100014BF83EA400040008A4280B2C1D17047BB
:101E20000846704770B5124D4FEA104ED5F818624B
:101E300004E0D5F82C47E41AA2420ED3BEF1010FFC
:101E40000CBF7469B46920EA0404A4B2B4FA84F43F
:101E500064098C42EDD0002070BD00232022C5F81B
:101E6000483285F8543285F85522032070BD00BFF2
:101E70004000012010B41849D1F81842636913F0EA
:101E8000800327D1626912F4806212D1D1F82C3715
:101E90001B1A012BF2D9D1F8580281F854222024C0
:101EA0002043C1F85802C1F84822032081F8554266
:101EB0000DE06FF48062626104202024C1F85802B2
:101EC00081F85432C1F84832012081F855425DF85A
:101ED000044B70470020FAE740000120034BB3F8A1
:101EE000681002464BBA0220138070474000012060
:101EF000704700BF08B5024B024A1A60FEF780F92E
:101F000000C00120AD700DB0002070470020704768
:101F1000024B93F8301701700120704740000120F8
:101F20004379012B00D0704780790228FBD8094AF9
:101F3000012882F83007F6D192F8311721B106490D
:101F40004FF400628A617047034B4FF00060986164
:101F5000E9E700BF4000012000080240084B596A31
:101F6000642202FB01F111F5001304D503F57F1C77
:101F70000CF57F533F339A1502700120704700BF64
:101F8000000000204379012B00D070478079421E69
:101F9000632AFAD80449830532330448A1FB0312AB
:101FA00051094162704700BF1F85EB5100000020BE
:101FB000024B93F8281001700120704700000020A8
:101FC0004379012B00D070478079421E072A9CBFBD
:101FD000014A82F82800704700000020074B4FF0AC
:101FE000000C93F82C1093F82D3080F800C00122DB
:101FF00041708270C3700420704700BF0000002051
:10200000074B93F82F2093F82E100170531C4FEAC2
:10201000910C9B10427080F802C0C370042070477E
:10202000000000204379022B00D0704710B4837960
:102030009A08911E06290ED8104C03F0FC0C94F857
:102040002F3084F82EC00133B2EB930FBCBF0CF1DC
:10205000FF3C84F82FC0C07901308408A21E062AF4
:1020600009D8064890F82E10B4EB910F03D8A300BE
:102070005C1E80F82F405DF8044B70470000002084
:10208000024B93F81F170170012070474000012098
:1020900000B50A4B197B93F80DC01A7D41705B7D2A
:1020A00080F802C04FF0000E012180F800E0C170FE
:1020B0000271437106205DF804FB00BF00000020A0
:1020C000034B0B2193F832270270417002207047B6
:1020D000400001204379012B00D0704780790A2805
:1020E0009CBF024A82F83207704700BF40000120BF
:1020F00010B5114B1A8E5101B1EB020C044660EB86
:10210000000041024FEA4C23981841EADC5E4EF190
:1021100000018B0143EA906C8301181A6CEB010EED
:1021200080184FF00003054A4EF1000104F0AAF9AF
:1021300042BA2280022010BD00000020400D0300A2
:102140004379022B00D07047C088074942BA93B246
:10215000064801FB03F38342F5DC0549054AA1FB70
:102160000313980C10867047400D03003F62B007C0
:1021700083DE1B43000000204379012B00D0704711
:10218000807904289CBF024A82F83307704700BF59
:1021900040000120054B06495B6B064A591A8B101B
:1021A00002FB03F303700120704700BF0000002012
:1021B00008990008ABAAAAAA704700BF034B1321D5
:1021C0001A7F027041700220704700BF000000209B
:1021D0001B4B93F83427032A31D810B519491A4CF0
:1021E000096AB0F8092090F806E083F834E7091B83
:1021F000002483F83547C3F83847B0F8074060BA81
:10220000040452BA1FFA80FCA3F83C2748BF4FF4DD
:10221000004C92B254BFA3F83E07A3F83EC79445C2
:102220004FEA610138BFA3F83CC7BEF1010FC3F804
:10223000241704BF83F835E7C3F8381710BD70477B
:1022400040000120000000204000002000207047D6
:102250004379012B00D07047827912B102490B708B
:10226000704701480270704740000120094B0A4A3C
:10227000D3F840374FF47A7101FB03F39909A2FBBD
:10228000012399090A0202F47F0343EA0161016014
:102290000420704740000120632D3E054379042B44
:1022A00000D07047D0F80600054A064903BA02FB81
:1022B00003F30548A1FB03129109C0F840177047CA
:1022C000400D0300D34D62104000012000207047F4
:1022D000002070470020704700207047704700BF03
:1022E000704700BF704700BF00207047704700BFB5
:1022F000414B93F82F1000297BD030B53F4A32F87C
:10230000025B6BBA038001234C1E8B4204F007046E
:102310006CD265B2C4B3012D2CD0022D24D0032D74
:102320001CD0042D14D0052D0CD0062D04D032F86D
:10233000024B65BA0223458032F8024B65BA20F899
:102340001350013332F8024B65BA20F813500133B1
:1023500032F8024B65BA20F81350013332F8024BC1
:1023600065BA20F81350013332F8024B65BA20F8F1
:102370001350013332F8024B65BA20F81350013381
:102380005FFA83FC8C4531D2144603F1010E34F818
:10239000025B6DBA20F81350B2F802C09CFA9CFCA4
:1023A00020F81EC064889D1C64BA20F81540D488AB
:1023B000DD1C64BA20F8154014891D1D64BA20F88C
:1023C000154054895D1D64BA20F8154094899D1DFF
:1023D00064BA20F81540D489DD1D64BA083320F8AA
:1023E0001540DDB28D4202F11002CDD34800C0B2DB
:1023F00030BD4800C0B270470000002084070120B3
:1024000000207047704700BF1F4B93F82F2093F8B0
:102410002E1001328B1A48BF03339A10013212F08A
:10242000FF032ED0194AB2F88417012B49BA018054
:1024300027D0B2F88617022B49BA418021D0B2F8D2
:102440008817032B49BA81801BD0B2F88A17042B56
:1024500049BAC18015D0B2F88C17052B49BA018151
:102460000FD0B2F88E17062B49BA418109D0B2F8C5
:102470009017072B49BA818103D0B2F8922751BA3D
:10248000C1815800C0B27047000000204000012008
:102490002DE9F84381FB0151AC0B5B0044EA814616
:1024A000B6FBF2F7C11B4FEAE07060F10008A1FB38
:1024B000030503FB0851002303F094FF002970DBA0
:1024C000B0F1004F0A4671F1000106464FF00104D9
:1024D0000CDBB30843EA8276B6F1004F4FEAA20262
:1024E0004FEA440472F10001E4B2F2DA97030025E6
:1024F00047EA964EB10300234FF08042980840EA25
:10250000827399424FEAA2027EEB0200F6DB53EAA5
:1025100002004FF0000042D08446C61842EB0C0780
:10252000B1427EEB07094FEA930808DB891B6EEB8B
:10253000070EDB1842EB020918184CEB090C460891
:1025400048EA8273921046EACC7053EA02064FEAD8
:102550006C0CE2D1C71700FB05F5A0FB041004FBCF
:10256000075426184D1846EB06036A1846EB030776
:102570007801550140EAD264521947EB040351181F
:1025800046EB0306002E0CDB11F5005746F1000464
:10259000B80B40EA8445FF2D28BFFF25E8B2BDE80F
:1025A000F8830020BDE8F8832DE9F0410026154CA2
:1025B00082B080464FF400753746D4F80823D4F82B
:1025C0000C339A420DF10600F7D0FFF78BFB002881
:1025D000F3D0BDF90600013D00FB00F1ADB207EB01
:1025E000A1370644002DE8D101234FF40072314693
:1025F0003846FFF74DFF88F80000012002B0BDE823
:10260000F08100BF400001200E4900B5844601F171
:102610000E0E0D2300200CEA030202F00F0312F04D
:102620000F0205D000225A405B08FCD102F00102E3
:1026300042EA40008E4580B202D031F8023BEAE720
:102640005DF804FB229900080E4900B5844601F1AB
:102650001E0E40F2D56300200CEA0303C3F30A0206
:1026600013462AB100225A405B08FCD102F0010255
:1026700042EA40008E4580B202D031F8023BEBE7DF
:102680005DF804FB3299000870B5214D002405F176
:10269000080E3EF8023D03406400DEB2A4B2B44628
:1026A00046B100268CEA06065FEA5C0CFAD106F019
:1026B00001031C43AE45ECD1F4B1072C04D84FF60E
:1026C000FF701080002070BD0125A4F10806158060
:1026D00016F0FF0214D1C0F34015C0F3C006C0F3DA
:1026E000800246EA450C42EA4C04C0F3400040EA4E
:1026F00044030B80012070BDC0F340151480ECE74B
:10270000C2F1080305FA03F4604080B2E3E700BFBA
:10271000509900082DE9F041364B05468E46174684
:1027200093E8070084B00DF1040CE046ACE8030028
:102730000DF10E060024ACF8002036F8020D6400FE
:1027400015EA0002A4B206D0002151405208FCD183
:1027500001F001031C434645EFD1002C3FD00F2C64
:1027600006D84FF6FF7500203D8004B0BDE8F0812B
:102770000126A4F110003E8010F0FF0733D1C5F30D
:10278000403CC5F3C02242EA4C08C5F3802343EA2B
:102790004804C5F3402646EA4400C5F3C01747EA9B
:1027A0004001C5F3801C4CEA4102C5F3401848EAD9
:1027B0004204C5F30013C5F3C00043EA440640EAEF
:1027C0004607C5F3800141EA470CC5F3400545EAD9
:1027D0004C020120AEF8002004B0BDE8F081C5F342
:1027E000403C3C80CDE7C7F110018E406E40B5B251
:1027F000C5E700BF589900081B491C4B4A6993F86C
:1028000099C782F0400242F480028A6193F89817D7
:102810008C4502D093F8C42702B9704793F89AC741
:10282000D3F8941741F82C0093F89A1793F8980767
:1028300001315FFA81FC604583F89AC702F1FF32EB
:1028400098BF4FF0000C93F8991798BF83F89AC778
:102850005FFA82FC03EB8C000131D0F89C0783F80F
:10286000991783F8C4C77047000002404000012058
:1028700010B41A4CD4F8181208E04A6912F0100C7F
:102880000CD1D4F82C371A1A012A18D84B6913F036
:102890004003F2D000205DF8044B70476FF0100049
:1028A00048614FF0200CC4F858320120C4F8483277
:1028B00084F8543284F855C25DF8044B7047D4F85C
:1028C000580284F854C220210843C4F8580284F8FE
:1028D000551203205DF8044B704700BF40000120F3
:1028E00070B41B4ED6F8185208E06C6914F480637B
:1028F00017D1D6F82C47A41AA14208D36B6920EA55
:102900000304A3B2002BF0D1184670BC70472022FC
:10291000C6F8483286F8543286F85522032070BC37
:102920007047286840F400712960D6F818526FF497
:1029300080636B61002404222021C6F8582286F8A7
:102940005442C6F84842012086F8551270BC7047C0
:1029500040000120F8B5264CD4F84432042B074639
:102960000D46164608D0012B06D013F5803F03D044
:10297000D4F84802122805D1D4F81822116841F47D
:1029800080731360D4F8182204E0D4F82C07811B5C
:102990008D4215D35069C307F7D5D4F82812B1F585
:1029A000804F18D11761134832462946FFF798FF28
:1029B00028B1D4F85842042C0CBF01200320F8BDE4
:1029C00000234FF0200CC4F8483284F8543284F8C5
:1029D00055C20320F8BDF02313610748324629464B
:1029E000FFF77EFF0028E4D1D4F818221761DAE758
:1029F00040000120020001000800010010B51F4C3A
:102A0000D4F8C807C36823F00101C160036A41F22A
:102A1000111213420AD1026A40F244410A4205D11E
:102A2000036823F001020260D4F8C8071449112397
:102A3000C4F8D437FDF7ECFED4F8C827D4F8D00793
:102A40001368D4F8D81723F07003034323F44070BD
:102A500008431060D4F8C837D4F8D407D4F8CC476A
:102A6000D86201229C625A61D96841F00100D860A5
:102A70001C6844F001021A6010BD00BF4000012034
:102A80000C08012030B448490268D1F82C470025D1
:102A9000022380F8353080F83450156825F00103A2
:102AA0001360026804E0D1F82C371D1B052D50D8A7
:102AB0001568ED07F7D4D0E90134C1682343D0E9A4
:102AC00004540B432B432343D0E906412343046AB8
:102AD00015680B4323433549446A2940042C43EAD3
:102AE000010303D1D0E90B5425432B431360016844
:102AF000426A4B69042A23F0070545EA020508D11A
:102B0000826A846915435CBB012A47D0022A2ED011
:102B10006AB34D61036826495FFA83FCACF1100289
:102B20001824B2FBF4F5294423F47F7323F0030542
:102B300091F88C10C1655F2A88BF04353F228A4016
:102B400000244FF0010C8565AA60446580F835C00B
:102B500004E020210322416580F8352030BC704715
:102B6000B4F5005F0CD0022A04D9032AD1D1C26A7D
:102B7000D201CED540210125416580F83550EDE7E1
:102B8000032AC6D801A454F822F000BF752B000810
:102B90006F2B0008752B00089D2B0008C36AB3F14A
:102BA000C07FB6D1E6E700BF400001203F8010F0B3
:102BB000D89800080D4B0E4A1868A2FB00218B091B
:102BC000013BB3F1807F0BD24FF0E0220948536103
:102BD0004FF0F00C0021072380F823C091611361AE
:102BE00000220F214FF0FF30FDF762BB00000020F4
:102BF000D34D621000ED00E030B4174BD3F814252C
:102C0000D3F81815501AB0F5807F10D1134D144920
:102C10008024AC610A6922F00400086130BFD3F857
:102C20001425D3F81805121AB2F5807FF1D0D3F825
:102C30001455E9B2043103EB410C4FF40044ACF8F5
:102C40001445D3F81425054D4FF400000132C3F8A4
:102C50001425A86130BC70474000012000080240E4
:102C600000ED00E0B0F5804F70B438DA10F5804F19
:102C700032DB00F5804290B241001FFA81FC194A14
:102C8000D2F81435D2F818451D1BB5F5807F10D148
:102C9000154E16488021B161036923F004040461D4
:102CA00030BFD2F81455D2F81835EC1AB4F5807F3D
:102CB000F1D0D2F814650C48F1B2043102EB4105B1
:102CC0004FF40004A5F814C5D2F814350133C2F846
:102CD0001435846170BC70474FF0000CCFE74FF69D
:102CE000FF7CCCE7400001200008024000ED00E03E
:102CF00004490023C1E90133C1E903334B610B836C
:102D0000704700BF4000012002484022002103F02C
:102D1000D5BD00BF8407012005490023C1F88437D1
:102D2000C1F88837C1F88C37A1F89037704700BFD9
:102D3000400001202DE9F04FA64BA749A74AA84F14
:102D4000AFB001F50064824603F50060CDE90A40AA
:102D500003F58055069102F500660C920021802251
:102D60000EA80895079309960D9703F0A7FD9D4CB3
:102D70004FF40075D4F80813D4F80C339942F9D005
:102D80000DF11600FEF7AEFF0028F3D0DDE9068056
:102D90004646BDF91690B8F802E036F8043BB0F8A4
:102DA00002B00696DDE908120F9E1EFB09F848F3F3
:102DB0008F3E13FB09F31BFB09F7764443F38F3C6B
:102DC00047F38F3B30F8043B0F964E8831F8047B75
:102DD0000790089113FB09F017FB09F141F38F37B6
:102DE00040F38F3E16FB09F0568832F8041B139B04
:102DF000099240F38F380E9811FB09F24344604466
:102E000042F38F38DDE911C2139316FB09F33A44FC
:102E10001499159F0E9043F38F36109B12929E4487
:102E2000DC4441443E44CDE910ECCDE91416DDE923
:102E30000A86C3461E9F3BF804EBB8F80210CDF893
:102E400028B01EFB09FC4CF38F3211FB09F13A4408
:102E50001F9F1E92DDE90C0341F38F3847447188B0
:102E60001F9736F8047B0B965E88B0F802B011FB12
:102E700009F141F38F3C17FB09F116FB09F730F814
:102E8000046B0C9041F38F3E33F8041B0D9316FB3B
:102E900009F0259E1BFB09F247F38F3B11FB09F953
:102EA00042F38F3849F38F3340F38F32DDE9221933
:102EB0005E44DDE920B0249F2596013D3B44F34468
:102EC00060441144C144ADB2CDE920B0CDE922192E
:102ED0002493002D7FF44EAF5446CAF8005044F8B6
:102EE000045F0EAA029201940395019DDDF80890FB
:102EF000A5F1040AD046CE460AF1020BDEE9007CB9
:102F00008CFB0C6387FB0721B00B950B40EA8344D5
:102F100045EA8147E6195BD4B514B20300234FF0AC
:102F200080419B0843EA81739A424FEAA10175EB05
:102F30000100F6DB53EA01004AD000200446CDF838
:102F400000E0C71841EB040CBA4275EB0C0E4FEAD7
:102F5000930608DBD21B65EB0C05DB1841EB010780
:102F6000181844EB070446EA81738910470853EAAE
:102F7000010647EAC4704FEA6404E2D1642606FB06
:102F800000F2002ADDF800E004DA02F57F1C0CF5FF
:102F90007F523F32C2F3875508F8015BD8450EF1E6
:102FA000080EABD1019FB84509F1100901D0C24606
:102FB000A0E7039B029802330AF106014030042B7C
:102FC00003930191029090D108202FB0BDE8F08FBB
:102FD0000025E1E76CA900086C9900086CC10008A5
:102FE0006CD10008400001202DE9F047364A374DEA
:102FF0005369374F044683F0020040F40031916179
:1030000005F604004FF42A72002103F057FC002655
:10301000A000304C85F8AC6AA5F8B06A05F6B42C6F
:1030200005F6C42EA7F6AC58324657F804ABDCF8C8
:1030300000909AF8003008EB8301D1F8B41D0144E8
:10304000CCF800109AF802A008EB8A03DCF804A080
:10305000D3F8B43D03449A4508BF8945CCF8043001
:1030600018D10CF1080C08340EF1100E0EB901261F
:10307000DBE7154E1848194F0423B3617269C5F890
:10308000040382F0020444F40031C5F8F472B16123
:10309000BDE8F087CEE90022CEE90222A4F5005176
:1030A000C1E90022C1E90422C1E90822C1E90C22D8
:1030B000C1E91022C1E91422C1E91822C1E91C2288
:1030C0008031A142ECD1CCE7000802404000012051
:1030D0006CD9000858440120DB1B0400B9A2010090
:1030E0002DE9F04F484C94F8E53A0022A1B084F85D
:1030F000E42A002B00F00C83444894F8EC1A057F76
:1031000094F8ED7AD4F8E86AA94228BF294640220B
:10311000AF4206EB050338BF2F4684F8EC1A0DEBDF
:1031200002000021C4F8E83A84F8ED7A03F0C6FB07
:1031300094F8EE0A94F8EF8A0130C3B2984584F807
:10314000EE3A00F0C982324D324AEE1896F88C9D64
:1031500096F880AD09EB490BAB44D3449BF898CD6E
:103160009BF8A4ED02EB8C0102EB8E07D1F8B45D65
:10317000D7F8B40D264E09953344264F93F88F8D1A
:1031800093F8839D93F8925D089008EB480AB24447
:10319000CA4493F8868D9AF8A4CD9AF898BD05EBA9
:1031A0004509B14407EB8C02C14493F8955DD2F810
:1031B000B40D99F898AD0A9007EB8B0E93F8890D32
:1031C000DEF8B41D99F8A4BD0B9105EB450307EBA0
:1031D0008A0C33440344DCF8B41D93F8986D0D91C8
:1031E00093F8A41D07EB8B0E07EB860807EB81070E
:1031F000DEF8B42DD7F8B45D0C92D8F8B42DCDE933
:103200000E524FF400750DE0400001200000002038
:10321000B8DC0008C0CB0008CE4F396921F00402A9
:103220003A6130BFD4F80803D4F80C339842F3D095
:103230000DF11E00FEF756FD0028EDD0BDF91E3041
:10324000D4F8F01AD4F8F42A089E03FB03F901EB32
:10325000A9301A44C4F8F00AC4F8F42ADDE90902D6
:10326000B2F802C0778841881CFB03F830F804CB21
:103270000990B34617FB03F60B9F1CFB03F046F3C4
:103280008F3911FB03F646F38F3E48F38F313E46EC
:1032900040F38F3832F8040B0A9205F1FF3A10FB25
:1032A00003F21FFA8AF536F8040B3BF804ABCDF8AD
:1032B00020B010FB03FC1AFB03FB10984BF38F3A72
:1032C0005044019010901198484402901190129827
:1032D00040440090129013987044039013901498F7
:1032E00042F38F3B58440490149015987F880B96B6
:1032F000014405911591169917FB03F64CF38F3293
:10330000DDE90E7C0A441692DDE90C20B7F802A034
:1033100051881AFB03F832F804AB0C9246F38F3B4A
:103320001AFB03F211FB03F6418842F38F3A30F89F
:10333000042B0D9046F38F3911FB03F612FB03F0BB
:1033400046F38F3E37F8042B0E97664612FB03F7C1
:1033500036F8042B48F38F3140F38F3847F38F3022
:1033600012FB03F747F38F32179F5F441797189F9D
:1033700057441897199F4F4419971A9F47441A9713
:103380001B9F77441B971C9F0F9638441C901D98D9
:10339000BCF8026001441D911E990A441E9216FB5E
:1033A00003F31F9A43F38F3717441F97002D7FF4C1
:1033B00039AF94F8F8BA684808258561BBF1000F69
:1033C00000F09081029E019886FB06379A0B80FBE5
:1033D000001642EA8745039F8B0B87FB072043EAD1
:1033E000864C009B910B41EA804683FB037294F864
:1033F000E41AB80B04EB411A40EA824965444E4492
:10340000BBF1010FCAF8FC5ACAF8006B5FD0059EE9
:1034100086FB0637049E9A0BDDE9168586FB063C83
:1034200042EA87409F0B47EA8C49484485FB0525C3
:1034300088FB0878CAF8040BBE0B900B40EA854362
:1034400046EA884C6344BBF1020FCAF8083B3ED001
:10345000DDE9180989FB092780FB0008DDE91A531B
:10346000960B46EA8742870B47EA884C624483FB07
:10347000033685FB0579CAF80C2BBD0B9A0B42EA83
:10348000864045EA89484044BBF1030FCAF8100B57
:103490001DD0DDE91CC686FB0627DDE91E308CFB4E
:1034A0000C69950B45EA8742B70B47EA894883FBCD
:1034B0000335424480FB0007CAF8142B9A0B830B98
:1034C00042EA854643EA874C6644CAF8186B94F88A
:1034D000E5AA214E4D1CEAB24FF400219245B1619C
:1034E00084F8E42A3FF608AE1B4810278761BBF139
:1034F000000F00F0EA80DFF86880DFF868E098F8F5
:103500002850B4F8083C0295691EAEF1E409CAB22D
:103510000133002509EB4216D4F800CCDEF8049004
:10352000D8F838700493019502988246002800F07C
:10353000A9800A4B03EBC503F11AA1F1200250093F
:103540000130002110F003004FEAC50A0A4676D088
:103550000AE000BF00ED00E0000802403C0B012043
:1035600000000020400C0120012829D0022816D09C
:1035700069485AF800A05868824500F3B680A0EB6D
:103580000A0000900120039000984FF0000A824545
:10359000B8BF0246039803F12003B8BF0146D3E940
:1035A00000A08245D5BFA0EB0A00AAEB00004FF0B7
:1035B000010A4FF0000A8242BCBF02465146203346
:1035C000D3E900A08245D5BFA0EB0A00AAEB00001A
:1035D0004FF0010A4FF0000A20338242BCBF02467E
:1035E00051469E422BD147E0A0EB0A004FF0000A63
:1035F0008242BCBF02465146D3E9080A5045D5BFB6
:10360000AAEB0000A0EB0A004FF0010A4FF0000AFD
:103610008242BCBF02465146D3E9100A5045D5BF8D
:10362000AAEB0000A0EB0A004FF0010A4FF0000ADD
:1036300060338242BCBF024651469E421CD0D3E951
:1036400000A08245CBBFAAEB0000A0EB0A004FF020
:10365000000A4FF0010A8242B8BF024603F120037C
:103660001868B8BF5146D3F804A05045BCDCAAEB9B
:1036700000004FF0010ABBE712EB0C0C49EBE279BA
:103680004FFA81FA049A3B7850194AEA43014207FB
:1036900039701FFA80FA07D1204B0137F91AB1F5BA
:1036A000897F27D2012201920135E8B2584506F1FF
:1036B0000806FFF439AF019DCEF80490C4F800CCA1
:1036C0000DB1C8F83870A4F808AC154C4FF480164A
:1036D000A66121B0BDE8F08F00231248124D84F896
:1036E000EE3A47E594F8E41AF1E6AAEB0000009000
:1036F000039149E7238BCEF804900133C4F800CC42
:10370000C8F83870A4F808AC238321B0BDE8F08F66
:1037100094F8F8BAE8E600BF3C0B01204C0C0120FD
:103720000008024038DA000838E2000810B4094CFA
:1037300084460FCCCCF8000020788CF81000CCF830
:103740000410CCF80820CCF80C3011205DF8044BA4
:10375000704700BF20EE02084379012B00D070476C
:103760002DE9F04182798D4CD1094FEA02201ABF30
:1037700048F2050080EA4220400081B20D0446BFB5
:1037800048F2050585EA410149008EB2330446BF7F
:1037900048F2050383EA4603730084F82B279AB2A4
:1037A000170446BF48F2050383EA420353009FB261
:1037B0003E0446BF48F2050383EA47037B0098B204
:1037C000050446BF48F2050383EA400343009DB267
:1037D000280446BF48F2050383EA45036B009EB206
:1037E000310446BF48F2050585EA46067600B4F87E
:1037F00029171FFA86F8414582B025D094F8552242
:10380000A4F829874FF0FF0C84F828C7202AD4F8A1
:10381000283719D1D4F82C8794F8557284F8213DB3
:103820000020C3F30725C3F30746C3F3076105224E
:10383000202F84F8200D84F8225D84F8236D84F80D
:10384000241D84F8202E02D002B0BDE8F081D4F807
:10385000187205E0D4F82C37A3EB0806192E27D8E8
:10386000BB69D84310F00205F4D094F85462012EDD
:10387000EAD0012184F854123A6822F400633B60D4
:103880004FF0210E464F84F855E24FF0100C002502
:103890004246A02084F856C2C4F85852C4F8447274
:1038A000FFF758F860B1D4F8583284F85452CBE797
:1038B0002027C4F8485284F8545284F85572C3E75C
:1038C000D4F81832019059690191986901900199D1
:1038D000344F05265A6912F080052DD1596911F42B
:1038E00080601AD1D4F82C57A5EB0802012AF1D92F
:1038F000D4F8586284F8540220273E43C4F8586232
:10390000C4F8480284F85572D4F85842042C9BD16C
:103910001D6845F400721A6096E76FF48060042118
:103920004FF0200C5861C4F8581284F85452C4F86F
:10393000485284F855C2E7E7BE46751E1EF8010BD3
:1039400018615A695207A9B224D519B37D781D614F
:10395000023EB6B20237596911F004050AD159691D
:1039600011F48060D9D1D4F82C57A5EB0802012AB4
:10397000F1D9BDE7002EADD11F68202047F40072B9
:103980001A6084F8550284F8546284F8566202B0D2
:10399000BDE8F0810E467746DDE700BF400001201C
:1039A0000000FFFF600D01202DE9F04F784D95F8E4
:1039B000286E95F8293EB34285B004463AD095F872
:1039C000C407B8B3E17801F00303012B00F09A803B
:1039D000022B00F0B380A2787F2A34D095F82A8E8B
:1039E000D5F8242E42F8284095F82A4E95F8280E4E
:1039F00001345FFA84FC604585F82ACE1ED995F81B
:103A0000293E95F83087013385F8293EB8F1010F3A
:103A100005D1604F85F831874FF40066BE6195F897
:103A2000C4473CB1611ECAB205EB820985F8C427C0
:103A3000D9F89C47204605B0BDE8F08F4FF0000A4A
:103A400085F82AAEDBE76379002BC7D0617895F85B
:103A50002B07884201D0FF29C0D1D4F890B0D5F807
:103A6000C8AE4D4AD4F80690ABEB0A03A3FB0201A3
:103A70004A4A002302F006FD99FA89F7C11B95F81E
:103A8000308701EBD1704710A7F12202B8F1020F85
:103A900022EAE27308D13F49486980F4006747F0A1
:103AA00000628A61D4F890B0EF693C4AA7EB0A0C37
:103AB000DFF8E4A01BBA0093ACFB0A01002302F07C
:103AC000E1FC024613BAA7EB0B01344A0193A1FBB8
:103AD0000A01002302F0D6FC00BACDF80C90029047
:103AE000E946B9E80F001027677195F8297EC4F8F8
:103AF0000600B742C4F80A10C4F80E20C4F8123009
:103B000084D06BE795F82BA794F801B0D3457FF4E8
:103B100062AF0021982205F5636085F82C3E02F023
:103B2000CDFE85F830BE2678217985F8316E4FF0CC
:103B30007F0B85F832BE85F8341E4FE795F82B775A
:103B40006278BA4202D0FF2A7FF445AF2978002973
:103B50007FF441AF12480126982285F82C6E02F0BE
:103B6000ADFED4F8943085F8307E94F80080217949
:103B700085F8318E4FF07F0918BA042785F8329EF8
:103B800085F8341E85F8357EC5F8360E26E700BF69
:103B9000400001200008024040420F00400D030099
:103BA000700E01202DE9F04FB34EB44BF26BADF225
:103BB000AC4D20200192986192F80580B8F1000F79
:103BC00007D14FF4001601209E610DF2AC4DBDE807
:103BD000F08F019BAA4DDC78C4F3800707EB470206
:103BE00005EB8209303599F830A099F8317005EB72
:103BF00082010AEBC800A8AC716303910F30002169
:103C0000B0FBFAF52046ABB26A00029302F056FE12
:103C1000039B002F00F09D80029A511E88B20DF286
:103C2000A22B98490BEB400E4FF000098022002D8B
:103C300000F08880AEEB040CACF1020040080130CB
:103C400010F00300A44634D0012820D002280ED062
:103C5000208891F800A0400012EA0A0F18BF40F037
:103C600001002CF8020B520804BF01318022BCF87D
:103C7000000091F800B0400012EA0B0F18BF40F0AE
:103C800001002CF8020B520804BF01318022BCF85D
:103C9000000091F800A0400012EA0A0F18BF40F09F
:103CA000010052082CF8020B01D101318022F445A9
:103CB00048D0BCF800A091F800B0604612EA0B0FA3
:103CC0004FEA4A0C18BF4CF0010C20F802CB520806
:103CD000824608BF01313AF802CB91F800B008BF24
:103CE000802212EA0B0F4FEA4C0C18BF4CF0010C6B
:103CF00052082AF802CC01D180220131B0F802A08A
:103D000091F800B012EA0B0F4FEA4A0B18BF4BF0C4
:103D1000010B520808BF013100F1060CA0F802B0F7
:103D200091F800A0808808BF802212EA0A0F4FEAAB
:103D3000400018BF40F0010052082CF8020CB4D02B
:103D4000F445B6D109F101095FFA89FC67453FF6F0
:103D50006EAF002D00F0E0800298DFF82C9100F1AA
:103D6000FF3B1FFA8BF20DF2A22A0AEB420B0DF178
:103D7000980851001BF0020FDFF800A1019147469F
:103D80005ED120889B680DF11202414698470DF2E2
:103D9000A224002860D0BDF812509DB1F76BB9F88D
:103DA000140097F888C050FA85FE6544A9F814E01D
:103DB00087F88850DAF8142082F0400141F480033B
:103DC000CAF81830736B08F1020739E0BDF81230F9
:103DD0008F1C9BB1F06BB9F814E090F888205EFA64
:103DE00083FC134480F88830A9F814C0DAF8143042
:103DF00083F0400040F48002CAF818205D4545D0A9
:103E0000756B34F8020BAB680DF11202984718B3CA
:103E1000BDF8120098B1F16BB9F814E091F8882060
:103E20005EFA80FC104481F88800A9F814C0DAF822
:103E3000145085F0400343F48000CAF81800736BF7
:103E40009B682546394635F8020B0DF1120298475A
:103E50002C46B91C0028B9D1084E0B4F7469F98A59
:103E600084F0800242F400050131B561F9820DF25F
:103E7000AC4DBDE8F08F00BF0000002000080240FC
:103E8000D89800085A0C0120400001200DF1140BB5
:103E900000218222584602F011FD716B019B91F8BE
:103EA0000090012409F1FF3504FA05F7BCB208F1CE
:103EB00002073B449E46002319465D46ECB1B8F824
:103EC0000080204618EA000F4FEA430318BF43F072
:103ED000010301F007020FFA83F9072A01F1010A31
:103EE000C0F34F0008BF05F8019B1FFA8AF114BF09
:103EF0001FFA89F300230028E4D17745B84601D0A2
:103F00000237DBE7F66B019696F805805C46B8F160
:103F1000000F07D12F4B54E605AC822229462046DC
:103F200002F0CCFC08F595670DEB0703A446A3F25D
:103F30009241002748F205021CF801BB87EA0B25D5
:103F40002E0454BF6D0082EA4505A8B2050454BF93
:103F5000400082EA400086B2370454BF760082EA0D
:103F60004606B7B23E0454BF7F0082EA4707BBB2A1
:103F70001D0454BF5B0082EA43039DB22F0454BF6B
:103F80006D0082EA4505A8B2060454BF400082EAEB
:103F9000400086B235044CBF82EA46067600614591
:103FA000B7B2C9D147B10C494A8A002001324A82CE
:103FB0000DF2AC4DBDE8F08F019821464246063027
:103FC00002F0E2FB08F102040137BFB2BC42FBDCA5
:103FD000A0E700BF00080240400001202DE9F04F9B
:103FE000C178A94A4479A94BADF2AC4DC1F3800B1D
:103FF00002F130060BEB4B070DF1140A0190811D05
:1040000006EB8706224650465E63A5B202F0BCFB73
:10401000002C00F0FC816A1E0DF1150C4FEA4B08D4
:104020001CFA82FE5046002348F2050110F8017B7D
:1040300083EA07231F0454BF5B0081EA43039AB25B
:10404000170454BF520081EA420293B21F0454BFC6
:104050005B0081EA43039AB2170454BF520081EA1D
:10406000420293B21F0454BF5B0081EA43039AB239
:10407000170454BF520081EA420293B21F0454BF96
:104080005B0081EA43039AB217044CBF81EA420203
:104090005200704593B2C9D10AEB0409180A26AF41
:1040A0000AF80400002189F801304FF40272384602
:1040B00002F004FC7449D84401EB880B0235ADB220
:1040C0009BF83090E90049444A1E92FBF9F3002B1B
:1040D0009AF8000040F3CB800021CDE9024680220F
:1040E0008E46AC469B464E464FF0000327F81E30E6
:1040F00007EB4E08002E00F0B180104206F1FF34AD
:1041000014BF01230023520804F0030508D1013134
:10411000C8B2014684458CBF1AF8010010468022BF
:104120000124A64240F298804FFA85F9002D40D034
:10413000A14528D0B9F1020F12D0104203FA04F3BE
:1041400018BF43F00103E2409BB208D12144C8B23A
:10415000014684458CBF1AF80100104680220134C4
:1041600010424FEA430318BF43F0010352089BB2C9
:1041700008D10131C8B2014684458CBF1AF801004C
:104180001046802201345D00104218BF45F0010541
:104190005208ABB208D10131C8B2014684458CBF88
:1041A0001AF801001046802201345FFA84F94E4566
:1041B00052D910424FEA430318BF43F0010352089B
:1041C0009DB208D10131C8B2844501468CBF1AF8AE
:1041D00000001046802210424FEA450318BF43F00A
:1041E00001035FEA520904F101049DB209D10131D2
:1041F000C8B2014684458CBF1AF8010048464FF00A
:10420000800910EA090F4FEA450218BF42F0010287
:104210005FEA590593B208D10131C8B2014684451D
:104220008CBF1AF801002846802528424FEA430235
:1042300018BF42F0010293B26A0808D10131C8B236
:10424000014684458CBF1AF80100104680220334D1
:104250005FFA84F94E45ACD8A8F800300EF101049D
:104260001FFA84FEDE45FFF63FAFDDE90246A8AD4A
:104270004FF402720021284602F020FB4FF00009A3
:10428000DDF804800EE000BFD89800080000002090
:10429000726837F81A00904725F81A00654898F8B0
:1042A0000540466BA31C1FFA89FA04B1DC00307884
:1042B00001194A1E92FBF0F4A24509F10109E7DB5E
:1042C000777801267B1E9E40B1B2A0B2002900F093
:1042D0009A80421E94B20DF2A228574A08EB440677
:1042E0000023002800F08C80771BBC1E640801347A
:1042F00014F003042F4640D0012C2AD0022C14D0F5
:1043000037F802CB92F800B011EA0C0F03F1010369
:1043100014BF4FF0010C4FF0000CDBB2082B4CEA3D
:104320004B04147004BF0023013237F802EB1478F9
:1043300011EA0E0F03F1010314BF4FF0010E4FF00D
:10434000000EDBB2082B4EEA4404147004BF0023B5
:10435000013237F8024B92F800A0214203F1010329
:1043600014BF01240024DBB2082B44EA4A04147071
:1043700004BF00230132BE4242D03C4692F8009076
:1043800034F8028B013311EA080FDBB214BF4FF08F
:1043900001084FF0000848EA4907082BB4F800B0BC
:1043A000177004BF01320023177811EA0B0F03F1D5
:1043B000010314BF4FF0010B4FF0000BDBB24BEACF
:1043C0004707082B177001D100230132B4F802E02F
:1043D00092F800C011EA0E0F03F10103DBB214BF23
:1043E0004FF0010E4FF0000E4EEA4C07082B1770ED
:1043F00008BF002304F1060708BF0132A488AAE71A
:1044000049087FF46EAF0DF2AC4DBDE8F08F4FEA76
:10441000870826AF29468AF800508AF801504FF4E1
:104420000272384602F04AFA04488044294698F855
:10443000309048E6000000201A0F0120D8980008AC
:10444000234A244903461068234A30B40C68186094
:1044500003CA224DC3F80340C3F80A10C3F806008C
:1044600003CD1F4D59611F491F4CB2F800C01861A0
:104470000A682868C3F81E20986107CC1B4CC3F853
:104480002100C3F8251003CCAD88C3F82920184AB1
:104490009D832C25A3F80EC083F82D5094F800C0FE
:1044A000C3F82E00134CC3F8321003CA2288D96314
:1044B000A3F83F2093F83F109863A94283F836C0D1
:1044C00083F837500CBF3F20402030BC704700BFFE
:1044D00034EE020838EE02083CEE020848EE02080C
:1044E00054EE02085CEE020860EE020870EE02086C
:1044F0007CEE020884EE020808B5094B094993F8DE
:10450000332700F8012B01EB820C7E22DCF8B01D72
:1045100002F0A4FA02F034FA0130C0B208BD00BFC4
:1045200040000120B8DC00082DE9F04383B0614C65
:1045300000230093D4F82C2794F85512202922D177
:104540005D4D5E4E2F68FB08A6FB0315290A01EBA3
:10455000810808EB8806D4F81872009603E0B96960
:1045600011F0020313D0009B5D1E0095002BF6D1C5
:104570002020C4F8483284F8543284F855020320CD
:1045800003B0BDE8F083022003B0BDE8F08394F8E7
:104590005462012EF7D04FF0010C84F854C23D68EC
:1045A00025F400613960D4F84C12D4F81882D1F89F
:1045B00058900B652127102684F8557284F85662AE
:1045C000C4F858323E4F91F834E03E4E0B64022559
:1045D000A4F84252C4F844723B4FCF63E6453B4FC8
:1045E000A4F84052C1E91133C4F83C62CF6407D04B
:1045F00091F835E081F834C0E64525D081F83430B3
:104600002321FEF7A7F960B1D4F85862042E4FF0C9
:1046100000080CBF0120032084F8548203B0BDE8D9
:10462000F083D4F81862019072690192B369019322
:10463000019A716841F480757560776847F400628B
:10464000726084F854029BE7D1F800C081F83550BD
:104650004B65DCF8007027F48027CCF800700F68F9
:104660007D608D680F68402D08F110031ED0BE607C
:104670000E68F360CD6D3F27AF40C9F808700E6833
:10468000336843F0160535600F687E6946F0800395
:104690007B610D6C25B10F683E6846F008033B60F6
:1046A00009680D6845F001070F60A9E7BB600B685A
:1046B000DE60DFE7400001200000002089B5F8142B
:1046C0000000FFFF600D01203D070008BD07000846
:1046D00038B52F4B2F4C08229A61E56972B600203D
:1046E000C4F81405C4F8180562B6E16E0B6843F00F
:1046F00002020A60E06E016841F001030360FEF708
:104700007DF972B62448254A426062B6244B4FF4C4
:104710008031022099619861E3695A1B0121B2F549
:10472000166F84F81E1713D205F51665B5EB030C4A
:104730000ED0E069E369191A8C4509D9194A15693F
:1047400025F00403136130BFE1690D1AAC45F6D8BA
:1047500094F83207144A02EB400EBEF8C41DB1F5BE
:10476000807F4DBA07D90E4C094904204FF400252B
:10477000A0618D6138BD94F85532202BF3D102220F
:10478000A4F8205D5C2084F8202EFFF7CDFEEAE738
:104790000008024040000120000000203D1C0008ED
:1047A0000000024000ED00E0B8DC0008012804D859
:1047B00008B570B9012902D908BD00207047144B13
:1047C00083F82C10134BE9B94FF480309861012025
:1047D00008BD114B0E4893F8552280F82D10202A61
:1047E00013D14FF0000C4FF0020E83F8211D83F817
:1047F00020CD582083F820EEFFF796FEB0FA80F126
:10480000480908BD0120986108BD002008BD00BF0F
:1048100000000020000802404000012038B5437924
:10482000022B00D038BD81790129FBD8084CC5790D
:1048300004EBC104627BAA42F4D92369084613F849
:104840003510FFF7B3FF0028ECD0257338BD00BF4B
:1048500000000020184B194901229A61C869CB69F0
:104860001A1AB2F5C87F0AD2154A136923F0040355
:10487000136130BFCB691B1AB3F5C87FF5D391F82C
:104880001F0758B910B50F4C217B94F80DC08C450B
:104890000CD8237D607D984201D810BD7047A46973
:1048A000012014F83310BDE810407FE7226912F8A8
:1048B0003110FFF77BFFECE70000024040000120D1
:1048C00000ED00E0000000204379022B00D070478B
:1048D000C17980796AE700BF4379012B00D0704726
:1048E0002DE9F0418479122C10D8144D144E05EBAB
:1048F0004402707B1779B8424FEA440813D8454404
:1049000096F815C06D79AC4502D83477BDE8F081D2
:10491000B369012013F83510FFF748FF0028F4D0E1
:1049200035753477F2E73169002011F83710FFF759
:104930003DFF0028E3D03773E1E700BFD8980008B7
:10494000000000202DE9F041244C94F81F377BB182
:1049500094F81055E5B9012584F81055A8460127AB
:104960001F4E727BBA422ED8707D40451DD83577D8
:104970001C4D1D4EC4F8F46240F201224023002079
:10498000C4E9C005A4F8FA22A4F8F832BDE8F08121
:10499000112D03D9112584F81055DFE7134800EBDA
:1049A00045010F7991F80580DAE7B7690FFA88F1C8
:1049B000012017F83110FFF7F9FE0028D7D086F84C
:1049C00014803577D4E73369002013F83710FFF7E8
:1049D000EDFE0028C8D03773C6E700BF40000120B5
:1049E00000000020DB1B0400B9A20100D8980008D9
:1049F0004A4B082270B59A6172B6494C0020C4F83F
:104A00000803C4F80C0362B694F81E17002961D09D
:104A1000E569E069E3691A1A632A09D841490E6910
:104A200026F004030B6130BFE269161A632EF6D933
:104A30003A483D4B4FF400214FF4802281619A6146
:104A4000FFF708FFE669E069831B632B09D8354946
:104A50000A6922F00400086130BFE3699A1B632AE7
:104A6000F6D92E48304E082181614FF400334FF4BF
:104A70008020B3614FF0000CB06184F81EC7FDF7D1
:104A8000BDFF72B6294E2A4A726062B629492A4889
:104A90004FF080638B61FCF705F8E069421BB2F5CB
:104AA000166F25D394F81F57FDB9E16E0A6842F0DE
:104AB00002030B60E46E206820F001052560FDF71D
:104AC0009DFF72B61D49716062B6144E4FF400220C
:104AD000B26170BD144D4FF48026AE61FFF7BAFE8F
:104AE00094F81F57114E002DDFD0FFF72BFFDCE7A6
:104AF00005F5166EBEEB0005D4D0E169E369581ADE
:104B00008542CFD9074A136923F00400106130BFF2
:104B1000E369581A8542F6D8C4E700BF000802408E
:104B20004000012000ED00E00000024000000020F5
:104B30009D0200080004024004990008B919000809
:104B40004379022B00D070472DE9F0418479302C55
:104B500000F28280C579002D70D0642D66D93F4F58
:104B60003F4E4FF4804507EB8404FFF7B1FDD4F8C6
:104B7000C82F941E02F2FE37B4F9020005FB00F0C4
:104B800040F38F30FEF76EF8B4F9041005FB01F125
:104B900041F38F30FEF766F8B4F9063005FB03F3F6
:104BA00043F38F30FEF75EF8B4F9082005FB02F2FC
:104BB00042F38F30FEF756F8B4F90A0005FB00F017
:104BC00040F38F30FEF74EF8B4F90C1005FB01F1FD
:104BD00041F38F30FEF746F8B4F90E3005FB03F3CE
:104BE00043F38F30FEF73EF834F9102F05FB02F245
:104BF00042F38F30FEF736F8A742BDD1FDF7FCFF38
:104C0000D6F81455D6F81845A54208D0154F1020EF
:104C1000B861D6F81415D6F818359942F8D1114E66
:104C20004FF48012B261BDE8F041E1E60E4A0B4F4D
:104C30000B4EA803A2FB00314D0994E7084E074F25
:104C400096F83387C8EBC80CCCEBCC0EA64407EB28
:104C50004E03B3F9DC5D86E7BDE8F081B8DC0008FF
:104C600040000120000802401F85EB512DE9F84F5C
:104C70004379022B01D0BDE8F88FDFF8D8A1714F3E
:104C800005460026FFF724FD6F4A3046AAF6C8788D
:104C9000934602F2FE3934E0FDF7E4FFCB4546D0FF
:104CA000A979BBF902000BF10204002940F0A480AD
:104CB000FDF7D8FFA979B4F90200002940F08C80F3
:104CC000FDF7D0FFA979B4F90400002974D1FDF7EC
:104CD000C9FFA979B4F9060000295DD1FDF7C2FF2B
:104CE000A979B4F90800002946D1FDF7BBFFA979DD
:104CF000B4F90A0081BBFDF7B5FFB4F90C0004F16B
:104D00000C0BAA79002AC7D097F83317C1EBC1045E
:104D1000C4EBC40CB44408EB4C0EBEF8DC3D13FBF2
:104D200000F040F38F30FDF79DFFCB45B8D1EA7915
:104D300000243AB1FDF760FF0134E979A4B2B4EB85
:104D4000412FF7DB414B534506F1010664D05AF879
:104D5000042FB2F900009BE797F833B7CBEBCB0CED
:104D6000CCEBCC0EB64408EB4E03B3F8DC2D12FBB3
:104D700000F040F38F30BEE797F833B7CBEBCB0CA6
:104D8000CCEBCC0EB64408EB4E03B3F8DC2D12FB93
:104D900000F040F38F30A8E797F833B7CBEBCB0C9C
:104DA000CCEBCC0EB64408EB4E03B3F8DC2D12FB73
:104DB00000F040F38F3091E797F833B7CBEBCB0C93
:104DC000CCEBCC0EB64408EB4E03B3F8DC2D12FB53
:104DD00000F040F38F307AE797F833B7CBEBCB0C8A
:104DE000CCEBCC0EB64408EB4E03B3F8DC2D12FB33
:104DF00000F040F38F3063E797F833B7CBEBCB0C81
:104E0000CCEBCC0EB64408EB4E03B3F8DC2D12FB12
:104E100000F040F38F304BE7D7F81455D7F81865FA
:104E2000AE4208D00A4A10249461D7F81405D7F886
:104E300018158842F8D1064F4FF48013BB61BDE8C6
:104E4000F84FD5E54000012044ED000840ED000892
:104E50000008024080EC00084379012B00D0704725
:104E60002DE9F041354A8079354902FB00F4A1FB78
:104E700004354FEA951808F580764FEA562840F237
:104E8000D137B84528BFB8462E4EFFF721FCB8F100
:104E9000040F38BF4FF0040800272B4D0020FDF70A
:104EA000E1FEAC1CB5F9020025E0B4F90200FDF703
:104EB000D9FEB5F90200FDF7D5FEB4F90600FDF7FD
:104EC000D1FEB4F90800FDF7CDFEB4F90A00FDF7F4
:104ED000C9FEB4F90C00FDF7C5FEB4F90E00FDF7EC
:104EE000C1FEB4F91000FDF7BDFEB4F91200FDF7E4
:104EF000B9FE34F9140FFDF7B5FEB44204F1020512
:104F0000D3D101374745C8D1FDF776FE0F4BD3F813
:104F10001405D3F81825824208D00D4E1027B7612A
:104F2000D3F81415D3F81845A142F8D1084D4FF421
:104F30008013AB61BDE8F0415AE500BF80841E00DC
:104F4000D34D621042F5000844F1000840000120F2
:104F5000000802402DE9F04FADF20C4DC3790090EE
:104F6000002B00F0DC809CB20098057A0DB9012678
:104F70000672009FBA79002A00F0C9806B4B6C4919
:104F800093F8335701934FF00008C5EBC506C6EB05
:104F9000C60740463A1801EB42092044B9F9DCAD96
:104FA00080B23028D044F5D9624F614D0DF1080C24
:104FB0004FEAE87B07F2FE3A0DF106060021CCF13C
:104FC0000209002009EB060E024603E0D3F8C83FB1
:104FD00033F90E10224492B2302A05EB82030844C2
:104FE000F4D9C1178A0342EA90415B4680034246E6
:104FF00001F0F8F9BA4526F8020F02D037F9021F7E
:10500000DFE7FFF765FB009C257A002D63D0DDF814
:1050100000B000270DF206460DF10600331A991E66
:105020004A08013212F007050DF106042AD0012DBD
:1050300022D0022D1CD0032D16D0042D10D0052D0A
:105040000AD0062D04D0BDF9080002ACFDF70AFE17
:1050500034F9020FFDF706FE34F9020FFDF702FEE8
:1050600034F9020FFDF7FEFD34F9020FFDF7FAFDEA
:1050700034F9020FFDF7F6FD34F9020FFDF7F2FDEA
:10508000A64221D0B4F90200FDF7ECFDB4F904000A
:10509000FDF7E8FDB4F90600FDF7E4FDB4F90800FA
:1050A000FDF7E0FDB4F90A00FDF7DCFDB4F90C00F2
:1050B000FDF7D8FDB4F90E00FDF7D4FD34F9100F5B
:1050C000FDF7D0FDA642DDD19BF8080001371FFA9D
:1050D00087F84045A0D8FDF78FFD019FD7F81465EC
:1050E000D7F81835B34209D0134D1021B946A9613C
:1050F000D9F81445D9F818259442F8D10E484FF440
:10510000801787610DF20C4DBDE8F04F70E4074940
:1051100001913120B0FBF3F84FEA883844E7009959
:1051200001221346CA7114461EE700BF4000012049
:10513000B8DC000844ED0008000802404379032B66
:1051400000D107E7704700BF2DE9F04FA14DA24AFB
:10515000AB8804464FF40061A1B00133916105F6BC
:10516000CC604FF489720021AB8001F0A7FBFFF700
:10517000AFFA2068A68810900023A5F8DE3FADF8AE
:10518000446010AF0DF1460A17F8015B6B4013F055
:10519000800F4FEA430318BF83F0D503DAB2510002
:1051A00012F0800F18BF81F0D501C8B2460010F090
:1051B000800F18BF86F0D506F5B26B0015F0800F92
:1051C00018BF83F0D503DAB2510012F0800F18BF78
:1051D00081F0D501C8B210F0800F4FEA400618BF29
:1051E00086F0D506F5B26B0015F0800F18BF83F07E
:1051F000D503DAB212F0800F4FEA420118BF81F0F6
:10520000D501BA45CBB2BFD18DF846300DF1620B56
:105210000023CDE91933CDE91B33CDE91D339DF8CA
:1052200040E01F930DF17E07DC4680202AE0013329
:10523000DBB2062B05D803F180010DEB010818F84D
:10524000401CC1F3C01646EA4500C1F3801545EA8B
:105250004002202631424FEA420218BF42F00102CA
:105260005FEA560E3CD10133DBB2062B4FF08000D3
:1052700004D819180DEB010E1EF840EC2CF8022F83
:10528000BC4554D000EA0E065FFA86F8B8F1000576
:10529000C0F3470118BF01250029C8D00EEA01025A
:1052A000D1B26E00002918BF46F0010610F47F7FCE
:1052B000B2B2C0F3870116D10133DBB2062B05D899
:1052C00003F180020DEB020515F8401CC1F3C01874
:1052D00048EA4606C1F3801040EA46024FF0200E2D
:1052E00070468E46CAE70EEA0105EEB24FEA420862
:1052F000002E18BF48F00108C0F3C7061FFA88F255
:10530000002E40F00C860133DBB2062B05D803F1EA
:10531000800E0DEB0E0010F8406CF10941EA4802D6
:105320002CF8022FBC45B6464FF04000AAD100230E
:10533000CDE91233CDE91433CDE91633274D189357
:105340003BF8022F26480D260021164016F00F0EBE
:1053500006F00F0C08D04FF0000888EA0C085FEA4E
:105360005C0CFAD108F0010E4EEA4101A84289B264
:1053700002D030F8026BE8E7BB452AF8021FDFD104
:10538000BDF84A30BDF85C20BDF85E10BDF848702D
:1053900006930292BDF86030BDF8622003910821A7
:1053A0000797049301920591BDF84C80BDF84EE03B
:1053B000BDF850C0BDF85270BDF85460BDF85650ED
:1053C000BDF85800BDF85AB0064B08940022802161
:1053D000BDE000BF400001200000024030990008FD
:1053E000229900080C0F0120069C21421C784FEAEC
:1053F000440418BF44F001041C70941CE4B2082C4F
:1054000040F0718193F8019018EA010F14BF012256
:10541000002242EA490A11EA0E0F5FFA8AF214BF2B
:105420004FF001094FF0000949EA42045C70022282
:105430000133013211EA0C0FD4B21A7814BF4FF0C5
:1054400001094FF0000949EA4209082C83F800904D
:1054500040F06E8193F80190394214BF012400247A
:1054600044EA490431425FFA84FA14BF4FF001095B
:105470004FF0000949EA4A025A70022401332942D6
:105480001A7804F1010414BF4FF001094FF000092C
:10549000E4B249EA4209082C83F8009040F06C819C
:1054A00093F80190014214BF0124002444EA490406
:1054B00011EA0B0F5FFA84FA14BF4FF001094FF0A5
:1054C000000949EA4A025A7001330222029C013261
:1054D00021421C7814BF4FF001094FF00009D2B2ED
:1054E00049EA4409082A83F8009040F06B81039A46
:1054F00093F80190049C114214BF0122002242EA59
:10550000490A21425FFA8AF214BF4FF001094FF0B5
:10551000000949EA42045C7002220133019C013215
:105520000C421C7814BF4FF001094FF00009D2B2B1
:1055300049EA4409082A83F8009001D10133002286
:10554000059C013C4FEA5101059400F0B980079C8D
:105550000C421C7814BF4FF001094FF0000949EAD2
:1055600044041C70541CE4B2082C7FF43DAF069A2E
:105570005C78114214BF0122002242EA440918EA71
:10558000010F5FFA89FA14BF0124002444EA4A0299
:105590005A700133022211EA0E0F93F8009002F1C3
:1055A000010214BF01240024D2B244EA4909082AA6
:1055B00083F800907FF43DAF5C7811EA0C0F4FEA5E
:1055C000440218BF42F001023942D4B214BF4FF076
:1055D00001094FF0000949EA44025A7002240133DC
:1055E00031421A7804F1010414BF4FF001094FF061
:1055F0000009E4B249EA4209082C83F800907FF4DC
:105600003EAF5C7829424FEA440218BF42F00102E3
:105610000142D4B214BF4FF001094FF0000949EA2A
:1056200044025A7002240133013411EA0B0FE2B232
:105630001C7814BF4FF001094FF0000949EA4409F2
:10564000082A83F800907FF441AF5C78029A1142F7
:105650004FEA4402039C18BF42F0010221425FFA64
:1056600082FA14BF4FF001094FF0000949EA4A02DB
:105670005A7001330222049C013221421C7814BF6B
:105680004FF001094FF00009D2B249EA4409082A53
:1056900083F800907FF442AF5C78019A0A424FEAA7
:1056A0004402059C18BF42F00102013C5A704FEAC7
:1056B000510103F101034FF0010205947FF447AF5C
:1056C000089FB8787F2800F0A6807A79002A00F039
:1056D000A6803846FEF782FC7F79002F00F09F807D
:1056E0000237FC009CE01C78033218EA010FD2B2AA
:1056F0004FEA440418BF44F00104082A1C707FF4E8
:105700004AAF93F8019011EA0E0F14BF0122002254
:1057100042EA490A11EA0C0F5FFA8AF214BF4FF00D
:1057200001094FF0000949EA42045C700133022488
:1057300039421A7804F1010414BF4FF001094FF007
:105740000009E4B249EA4209082C83F800907FF48A
:1057500047AF5C7831424FEA440218BF42F0010281
:105760002942D4B214BF4FF001094FF0000949EAB1
:1057700044025A700224013301421A7804F10104F0
:1057800014BF4FF001094FF00009E4B249EA4209A1
:10579000082C83F800907FF447AF5C786200029C8D
:1057A00011EA0B0F18BF42F0010221425FFA82FAA0
:1057B00014BF4FF001094FF0000949EA4A025A703C
:1057C00001330222039C013221421C7814BF4FF0A6
:1057D00001094FF00009D2B249EA4409082A83F8C6
:1057E00000907FF448AF049A93F80190019C114215
:1057F00014BF0122002242EA490A0C425FFA8AF2EF
:1058000014BF4FF001094FF0000949EA42045C70EF
:105810000222013394E67B79002B40F05D83002463
:105820001548164F466B90F82E5096F800907178F8
:1058300004954C4404F1FF3A9AFBF9F811FB08F384
:1058400070339AB20992A7F8DE2F002D00F05C8326
:1058500097F833870A4DDFF82CA00395C8EBC801F1
:105860004FF00009C1EBC1034FEAC8020593CB46D4
:10587000CDF80490029213E00000002040000120C7
:10588000C0CB0008B8DC0008049A09F101095FFAEE
:1058900089F50024AA428BF0010B019440F2B080FC
:1058A000039F019C059E07EB840CDCF8AC0D00EB1C
:1058B0000B0E10F80B509EF8024071190AEB4103D1
:1058C00032190AEB420CB3F9DC7DBCF9DC6DF81738
:1058D000BA198103D31741EA9741B803CDE90632DB
:1058E00000F080FD0746F0178103DDE906320AEB80
:1058F000850541EA9641B00300F074FD0AEB84048B
:10590000D5F8C83FD4F8C82FCDF818A0064603F242
:10591000FE30C246941E9D1E8046B4F90210B5F9B1
:10592000023006FB01F107FB031242F38F30FDF753
:1059300099F9B4F90400B5F9041006FB00F007FB6F
:10594000010343F38F30FDF78DF9B4F90600B5F983
:10595000062006FB00F007FB020141F38F30FDF744
:1059600081F9B4F90830B5F9080006FB03F307FB29
:10597000003242F38F30FDF775F9B4F90A10B5F92A
:105980000A3006FB01F107FB031040F38F30FDF7EF
:1059900069F9B4F90C10B5F90C2006FB01F107FB0D
:1059A000021343F38F30FDF75DF9B4F90E00B5F93A
:1059B0000E1006FB00F007FB010242F38F30FDF7EB
:1059C00051F934F9103F35F9100F06FB03F307FBCB
:1059D000003141F38F30FDF745F945459DD1019FD9
:1059E000D046DDF818A0002F7FF44EAF049A09F1DD
:1059F00001095FFA89F50126AA4201963FF650AFE8
:105A0000029BDFF8AC94A3EB08010020C1EBC107B7
:105A100001900497834619F8016B039C049A04EBE8
:105A2000860EDEF8AC5D05EB0B0C15F80B509CF800
:105A3000024050190AEB400311190AEB4106B3F971
:105A4000DC7DB6F9DC6DFA179003BA1940EA97418C
:105A5000D317B803CDE9053200F0C4FCF1170AEB07
:105A6000850507468803DDE9053240EA96410AEBE1
:105A70008404B00300F0B6FCD5F8C83FD4F8C82FB2
:105A8000CDF814A003F2FE31C2460646941E9D1EB8
:105A90008846B4F90200B5F9023006FB00F007FBB6
:105AA000030242F38F30FDF7DDF8B4F90410B5F9C5
:105AB000040006FB01F107FB001343F38F30FDF7F1
:105AC000D1F8B4F90610B5F9062006FB01F107FB81
:105AD000021040F38F30FDF7C5F8B4F90830B5F97E
:105AE000081006FB03F307FB013242F38F30FDF78A
:105AF000B9F8B4F90A00B5F90A3006FB00F007FB63
:105B0000030141F38F30FDF7ADF8B4F90C00B5F99E
:105B10000C2006FB00F007FB020343F38F30FDF778
:105B2000A1F8B4F90E10B5F90E0006FB01F107FB60
:105B3000001242F38F30FDF795F834F9103F35F934
:105B4000101F06FB03F307FB013040F38F30FDF716
:105B500089F8A8459DD1019FD046DDF814A0002FFB
:105B600000F0838100258BF0010B0195C94A4A455D
:105B70007FF451AFC84B099F93F828100691002F6E
:105B800000F04981029EDFF82C93A6EB0805002364
:105B9000C5EBC5028021D3460E9202930191049376
:105BA000CA46019E9AF800703E4214BF01240024A8
:105BB000750840F05D819AF801702026F8090AF115
:105BC000010AC7F380179AF800100E4214BF012192
:105BD00000217508019503D180220AF1010A019282
:105BE000049B069D04339EB20496002D00F00E81A6
:105BF000AA4ACDF83CA002EB840E02EB800C02EB2B
:105C0000870402EB8100DEF89877DCF89817D4F867
:105C10009837D0F898670A9700250B910C930D964A
:105C20000395029A0C9B0A9C0B980D9D0BEB0208A6
:105C300098F8927D98F88CAD98F88FED98F8956D5E
:105C400007EB4701194498F8863D0AEB4A090EEB29
:105C50004E0C06EB4602A144844498F8804D98F817
:105C6000830D19F804701CF800602A44CD5C98F884
:105C7000891D545C0E99CA198B190BEB42080BEB6A
:105C800043094A190BEB420E0BEB870A21440BEB3D
:105C9000410CB8F9DC0DB9F9DC9DBEF9DC8DDAF800
:105CA000C87F059709EB0002BCF9DC7DC3174244AD
:105CB0003A44990341EA9041D3178003CDE9073272
:105CC00000F090FB82464FEAE970820342EA994174
:105CD0004FEA8930DDE9073200F084FB4FEAE873D0
:105CE00099038146DDE9073241EA98414FEA88305D
:105CF00000F078FBDDE907320790F817810341EAED
:105D00009741B80300F06EFB0BEB86060BEB8505A5
:105D10000BEB8404D6F8C87FD5F8C82FD4F8C83F59
:105D200080460598CDF814B0D346CA46DDF81C90DD
:105D3000BE1E951E9C1E871E00F2FE310791B7F90C
:105D40000210B6F90230B5F90200B4F902C00BFB3B
:105D500001F20AFB032E09FB00E208FB0C2141F3D0
:105D60008F30FCF77FFFB7F90430B6F90420B5F99E
:105D700004100BFB03F00AFB0203B4F9040009FB57
:105D8000013208FB002343F38F30FCF76BFFB7F9B8
:105D90000610B6F906000BFB01F2B5F906100AFB76
:105DA0000023B4F9060009FB013208FB002343F38A
:105DB0008F30FCF757FF37F9081F36F9080F0BFB38
:105DC00001F235F9081F0AFB002334F9080F09FB1B
:105DD000013208FB002343F38F30FCF743FF0799A0
:105DE000B942ABD1029E039F069ADDF814B001368A
:105DF000F5B20137032D5FFA87F808BF00259045FB
:105E000003970295FFF40DAFDDF83CA0099B0499C0
:105E10008B423FF6C6AE224CFCF7EEFED4F81405DA
:105E2000D4F81865B0420FD01E4D1F4F1022AA6142
:105E30003B6923F00401396130BF1948D0F814459B
:105E4000D0F81865B442F2D1164D1548174F4FF4EB
:105E50008012AA61C3694FF00061B961C0F8C83E01
:105E600021B0BDE8F04FFEF7C3BD012601967DE6E7
:105E7000019A3D4214BF0120002093081CD19AF8DA
:105E8000013020260AF1010ADF09C3F380110196CF
:105E9000A6E600BF48F5000800000020B0ED0008AD
:105EA000400001200008024000ED00E00000024038
:105EB00044F500080C0F012001993B4214BF012753
:105EC0000027CE087FF47FAE9AF80150402201925D
:105ED000E9090AF1010A83E6124E3846F569FEF730
:105EE0007DF8D7F80620F1690F4EC5EB410014BAD2
:105EF000031BA3FB06010D4A002300F0C3FA05BAF9
:105F0000C7F80650FFF7E1BB064C094894F8338701
:105F1000DFF820A003904FEAC806029670E57146AC
:105F2000FFF798B94000012040420F00400D0300E8
:105F3000C0CB0008B8DC0008F0B5574C94F82C3EF4
:105F4000A7B023B994F89927F2B927B0F0BDD4F8D7
:105F50004057002284F82C2E75B1E069E669311AA9
:105F60008D4209D94D4F3B6923F004023A6130BF9D
:105F7000E669311A8D42F6D849484A4CFFF7E4F8F1
:105F80008025A56127B0F0BD94F89B0794F8985739
:105F9000D4F89477411CCEB2B54284F89B6798BF81
:105FA00084F89B37531E84F8993757F8205095F999
:105FB0000220AE78002A32DB00219822684600F0E9
:105FC0007DFCFF2194F82B078DF802108DF800005E
:105FD0006F788DF801702B798DF80430002101E085
:105FE0009DF805100631C9B26846FAF731FE00285F
:105FF000F6D094F82B272B4E2A702846FFF7A4F8EA
:106000008020B06194F8C477092F9ED804EB870EE6
:10601000013784F8C477CEF89C5727B0F0BD86F0DE
:10602000800304EB830C9F00DCF8E01FE9B12846F5
:10603000884798220021684600F040FC1A49AE7853
:106040008DF8026039440DF10600D1F8E830984728
:106050008DF8050001E09DF805000630C1B26846E4
:10606000FAF7F6FD0028F6D0CCE79822684600F053
:1060700025FCFE2201208DF802208DF805008DF808
:10608000066001E09DF805000630C1B26846FAF7E7
:10609000DFFD0028F6D0B5E74000012000ED00E06C
:1060A000700E012000080240381101204379012BB5
:1060B00000D0704782793AB10749084A8020886148
:1060C00082F81F37FEF73EBC0448034B80F81F27B9
:1060D0004FF4000199617047000002404000012028
:1060E00010B483B09A4B9B4A00200090196C41F089
:1060F00080541C64196C01F0805400940099019044
:106100001168954841F440441460126802F4404418
:1061100001940121019AC164986800F00C02042ADC
:1061200000F0CC80996801F00C04082C00F0C280CB
:106130008748826802F00C010C2900F0E280844A52
:10614000864901239370D1F82C0704E0D1F82C374D
:106150001C1A642C46D81468A403F7D57C4A9168AD
:1061600001F00C03082B3DD07B4C7C4900202066BD
:10617000D1F82C0704E0D1F82C47231A022B31D890
:1061800013689B01F7D447F6C07494FAA4FC4FF44B
:106190004030BCFA8CF490FAA0F04FF0706393FAA0
:1061A000A3FC4FF0E043BCFA8CF093FAA3F34FF456
:1061B000B473A340072404FA00F0034343F4800CB3
:1061C00065484CF01003012453600466D1F82C0795
:1061D0005F4A04E0D1F82C47231A022B02D8136837
:1061E0009C01F7D55E49086800F00F02042A0AD81E
:1061F00005240C700B6803F00F01052903D003B0D0
:106200005DF8044B7047524B986820F0F0029A609A
:106210001C68A201F3D59868504920F0030C4CF09B
:1062200002029A60D1F82C4741F2883004E0D1F89C
:106230002C27121B8242E2D89A6802F00C02082A2C
:10624000F5D147490B6803F00F04052C06D905204A
:1062500008700A6802F00F010529D0D13C4CA368F0
:1062600023F4E05040F4A052A260A16821F4604CF5
:106270004CF40043A360A06800F00C02082A45D04B
:106280000C2A1ED0374C324A4FF0F00C93689CFA1F
:10629000ACF13548B1FA81F103F0F002CA40024492
:1062A000324B92F8A007C4401C6003B05DF8044B69
:1062B000FCF780BC5B685A027FF53AAF244803685C
:1062C0004CE761686068646801F03F0C47F6C07392
:1062D00093FAA3F0B0FA80F21C401D482149B1FBAB
:1062E000FCF3D44003FB04F442684FF0E04C9CFA0A
:1062F000ACF1B1FA81F302F0E040D840B4FBF0F425
:10630000C1E7446863027FF51AAFD7E76168606848
:10631000646801F03F0C47F6C07393FAA3F0B0FA3B
:1063200080F21C400A480F49B1FBFCF3D44003FB48
:1063300004F442684FF4403C9CFAACF102F4403063
:10634000B1FA81F3D84001304200B4FBF2F49AE78D
:106350000038024000700040000047424000012029
:10636000003C02400024F400B0ED000800000020D2
:10637000094B4FF4E052986892FAA2F30749B3FA36
:1063800083F200F4E053D3400B44054893F8A01780
:106390000068C840704700BF00380240B0ED0008F8
:1063A00000000020094B4FF46042986892FAA2F373
:1063B0000749B3FA83F200F46043D3400B44054825
:1063C00093F8A0170068C840704700BF003802402B
:1063D000B0ED000800000020014BC3F81402704724
:1063E000400001207BB972B90029BEBF00204FF0E8
:1063F000004106E008BF00281CBF6FF000414FF0CD
:10640000FF3000F0BFB9ADF1080C6DE904CE0029F2
:1064100009DB002B1ADB00F04DF8DDF804E0DDE9C4
:10642000022304B07047404261EB4101002B1BDBAB
:1064300000F040F8DDF804E0DDE9022304B040425A
:1064400061EB4101524263EB43037047524263EBFD
:10645000430300F02FF8DDF804E0DDE9022304B087
:10646000404261EB41017047524263EB430300F04D
:1064700021F8DDF804E0DDE9022304B0524263EBC9
:106480004303704753B94AB9002908BF00281CBF0D
:106490004FF0FF314FF0FF3000F074B9ADF1080C50
:1064A0006DE904CE00F006F8DDF804E0DDE9022332
:1064B00004B070472DE9F047089D04468E46002B36
:1064C0004DD18A42944669D9B2FA82F252B101FAA8
:1064D00002F3C2F1200120FA01F10CFA02FC41EAB8
:1064E000030E94404FEA1C48210CBEFBF8F61FFA3D
:1064F0008CF708FB16E341EA034306FB07F19942D8
:106500000AD91CEB030306F1FF3080F01F8199428A
:1065100040F21C81023E63445B1AA4B2B3FBF8F064
:1065200008FB103344EA034400FB07F7A7420AD9EB
:106530001CEB040400F1FF3380F00A81A74240F213
:1065400007816444023840EA0640E41B00261DB17E
:10655000D4400023C5E900433146BDE8F0878B42B3
:1065600009D9002D00F0EF800026C5E90001304672
:106570003146BDE8F087B3FA83F6002E4AD18B424C
:1065800002D3824200F2F980841A61EB03030120F6
:106590009E46002DE0D0C5E9004EDDE702B9FFDEE2
:1065A000B2FA82F2002A40F09280A1EB0C014FEA8D
:1065B0001C471FFA8CFE0126200CB1FBF7F307FBEA
:1065C000131140EA01410EFB03F0884208D91CEB8D
:1065D000010103F1FF3802D2884200F2CB8043462A
:1065E000091AA4B2B1FBF7F007FB101144EA014409
:1065F0000EFB00FEA64508D91CEB040400F1FF3198
:1066000002D2A64500F2BB800846A4EB0E0440EA85
:1066100003409CE7C6F12007B34022FA07FC4CEA8E
:10662000030C20FA07F401FA06F31C43F9404FEA81
:106630001C4900FA06F3B1FBF9F8200C1FFA8CFE96
:1066400009FB181140EA014108FB0EF0884202FAEA
:1066500006F20BD91CEB010108F1FF3A80F08880AB
:10666000884240F28580A8F102086144091AA4B268
:10667000B1FBF9F009FB101144EA014100FB0EFEE9
:106680008E4508D91CEB010100F1FF346CD28E4518
:106690006AD90238614440EA0840A0FB0294A1EBA9
:1066A0000E01A142C846A64656D353D05DB1B3EB06
:1066B000080261EB0E0101FA07F722FA06F3F14036
:1066C0001F43C5E9007100263146BDE8F087C2F1DD
:1066D0002003D8400CFA02FC21FA03F39140014355
:1066E0004FEA1C471FFA8CFEB3FBF7F007FB10368E
:1066F0000B0C43EA064300FB0EF69E4204FA02F43A
:1067000008D91CEB030300F1FF382FD29E422DD98C
:10671000023863449B1B89B2B3FBF7F607FB1633C1
:1067200041EA034106FB0EF38B4208D91CEB010141
:1067300006F1FF3816D28B4214D9023E6144C91AC1
:1067400046EA004638E72E46284605E70646E3E6D1
:106750001846F8E64B45A9D2B9EB020864EB0C0EDB
:106760000138A3E74646EAE7204694E74046D1E7EA
:10677000D0467BE7023B614432E7304609E7644498
:10678000023842E7704700BF844641EA000313F035
:1067900003036DD1403A41D351F8043B40F8043B28
:1067A00051F8043B40F8043B51F8043B40F8043BEB
:1067B00051F8043B40F8043B51F8043B40F8043BDB
:1067C00051F8043B40F8043B51F8043B40F8043BCB
:1067D00051F8043B40F8043B51F8043B40F8043BBB
:1067E00051F8043B40F8043B51F8043B40F8043BAB
:1067F00051F8043B40F8043B51F8043B40F8043B9B
:1068000051F8043B40F8043B51F8043B40F8043B8A
:1068100051F8043B40F8043B403ABDD2303211D32A
:1068200051F8043B40F8043B51F8043B40F8043B6A
:1068300051F8043B40F8043B51F8043B40F8043B5A
:10684000103AEDD20C3205D351F8043B40F8043B2A
:10685000043AF9D2043208D0D2071CBF11F8013B28
:1068600000F8013B01D30B8803806046704700BFEE
:10687000082A13D38B078DD010F003038AD0C3F1FD
:106880000403D21ADB071CBF11F8013B00F8013BDF
:1068900080D331F8023B20F8023B7BE7043AD9D39E
:1068A000013A11F8013B00F8013BF9D20B78037073
:1068B0004B7843708B78837060467047830730B5A0
:1068C00048D0541E002A3FD0CAB2034601E0013C22
:1068D0003AD303F8012B9D07F9D1032C2DD9CDB262
:1068E00045EA05250F2C45EA054536D9A4F11002E5
:1068F00022F00F0C03F1200EE6444FEA121C03F1C4
:10690000100242E9045542E9025510327245F8D1AD
:106910000CF1010214F00C0F03EB021204F00F0C47
:1069200013D0ACF1040323F003030433134442F8FF
:10693000045B9342FBD10CF003042CB1CAB21C449B
:1069400003F8012B9C42FBD130BD64461346002C5A
:10695000F4D1F9E703461446BFE71A46A446E0E738
:106960000000000000000000000000000000000027
:106970000000000000000000000000000000000017
:1069800090F800F06DE9024520F007016FF0000C6F
:1069900010F0070491F820F040F049804FF0000417
:1069A0006FF00700D1E9002391F840F000F10800F2
:1069B00082FA4CF2A4FA8CF283FA4CF3A2FA8CF32A
:1069C0004BBBD1E9022382FA4CF200F10800A4FA91
:1069D0008CF283FA4CF3A2FA8CF3E3B9D1E90423E5
:1069E00082FA4CF200F10800A4FA8CF283FA4CF31C
:1069F000A2FA8CF37BB9D1E9062301F1200182FAD6
:106A00004CF200F10800A4FA8CF283FA4CF3A2FADB
:106A10008CF3002BC6D0002A04BF04301A4612BAE9
:106A2000B2FA82F2FDE8024500EBD2007047D1E9EC
:106A3000002304F00305C4F100004FEAC50514F07B
:106A4000040F91F840F00CFA05F562EA05021CBF4C
:106A500063EA050362464FF00004A9E730B540EA57
:106A60000104A30701D1032A0FD8844601F1FF3E98
:106A700007E01EF8011F03F8011B541EC1B19C461C
:106A800022466346002AF4D130BD0B46844619469F
:106A900053F8045BA5F1013424EA050414F0803FA7
:106AA000E4D1043A032A4CF8045B1946EFD8DDE739
:106AB0006244002CE8D003F8011B9342FBD130BDA7
:106AC00008B5F9F79DFB00BF704700BF2DE980486E
:106AD000084B094AD3B01968914200AF12D1074E52
:106AE000074A1E6082F30888A3F53039D9F80430CC
:106AF0009847FEE700C00120AD700DB0EFBEADDEDF
:106B0000F82A0020B04EB14BD6F8884044F4700506
:106B1000C6F888501A68AE4C002042F00101196096
:106B200098601D6825F0847828F480321A605C60D3
:106B30001968A84C21F480224FF000651A60D860D3
:106B4000B560B460D6F88810A348A44B41F4700433
:106B50009842C6F8884007D25E1E321A22F003021D
:106B60009F490432FFF710FE9E489F4DA84207D26E
:106B7000691E0B1A23F0030204320021FFF79EFE68
:106B80009A4E914834689A4A44F4007535603168E9
:106B900041F480633360356845F480713160C668C4
:106BA0004FF6FF0426403243C260FCF703F8FFF7BC
:106BB00097FA8648826802F00C04082C00F03187AE
:106BC0008C4A8D4DFA621560804B8C4A9E68F86A3B
:106BD0008B4D0168C6F30319914499F8B047E14021
:106BE000884C01602B1B002B4FEAA30660DD701E52
:106BF0004FF0010A54F8041B00F00705884756457A
:106C0000D14655DD95B3012D28D0022D20D0032D7E
:106C100018D0042D10D0052D08D0062D42F09384F5
:106C20004B46013354F8040B994680474D460135D5
:106C300054F8041BA94688474A46013254F8043BDD
:106C4000914698474846013054F8045B8146A8476E
:106C50004946013154F8042B894690474D46013589
:106C600054F8043B9847AE42A94621DDC7F8289066
:106C7000A046B96A58F8042B20340831B96290470D
:106C800054F81C5CA847D8F80430984754F8140C02
:106C9000804754F8101C884754F80C2C904754F83F
:106CA000085CA84754F8043C9847B86A8642DFDC81
:106CB000554E564C311B8A100029BA6252DDBD6A0E
:106CC00054F8040B6B1E03F007068047B96A0125D0
:106CD000A94247DD3EB3012E1ED0022E18D0032E4E
:106CE00012D0042E0CD0052E06D0062E42F076834C
:106CF00054F8043B0135984754F8046B0135B0470C
:106D000054F8040B0135804754F8041B01358847BB
:106D100054F8042B0135904754F8043B9847BE6A59
:106D20000135AE421EDDB86A8346A146203459F8CB
:106D3000041B884754F81C2C9047D9F80430984716
:106D400054F8146CB04754F8100C804754F80C1CDD
:106D5000884754F8082C9047083554F8043C984765
:106D6000AB45E2DC72B60025184C3D64266BDFF8BB
:106D7000A48046F001002063216B01F001023A6417
:106D80003B6CFD63236B43F002062663206B00F02F
:106D90000201F963FB6BBD63226B42F004032363C2
:106DA000266BC7F8B85006F0040007F1B0010126C1
:106DB000B8631748BB6BC7F8BC50C7F8B460C7F8D6
:106DC000B060F9F7B5FB27E000ED00E000380240C5
:106DD00010300024000000080000002040000120C6
:106DE000C4EE02084000012058440120003C02404B
:106DF0000003FA05000000200024F400B0ED0008B4
:106E0000C4EE0208C4EE0208C4EE0208C4EE020892
:106E100000000240000802404FF4803383614FF0CD
:106E2000020BC7F8B0B0F9F783FB4FF40032826170
:106E30000423C7F8B030F9F77BFB4FF4802282615E
:106E40004FF4006A40464FF00069C7E92D65C7F866
:106E5000BC50C7F8B0A0F9F76BFBA8F50060C8F804
:106E600018900823C7F8B030C7E92D65C7F8BC50A3
:106E7000F9F75EFB4FF400228261C7F8B0A0F9F782
:106E800057FBC0F818904FF04009C7F8B090F9F7D9
:106E90004FFB4FF4800383614FF0800AC7F8B0A026
:106EA000F9F746FB4FF400024FF4805C8261C7F8AB
:106EB000B0C0F9F73DFB4FF0805383617D63206BD9
:106EC00040F004022263236BC7F8C05003F00400B3
:106ED0007863786BC7F8B46040464FF48068C7E9C0
:106EE0002E56C7F8B080F9F723FBC7F8B0B0F9F712
:106EF0001FFB0422C7F8B020F9F71AFB0823C7F8D4
:106F0000B030F9F715FB1022C7F8B020F9F710FBE5
:106F10002023C7F8B030F9F70BFBC7F8B090F9F7AA
:106F200007FBDFF81C94C7F8B0A0F9F701FB4FF49A
:106F30008072C7F8B020F9F7FBFA4FF40073C7F876
:106F4000B030F9F7F5FAC9F8D857C9F8D0574FF467
:106F500000314FF0806585614FF4802281614FF4EC
:106F600000234FF480154FF40011826183614FF4C8
:106F7000800285614FF4000381614FF080754FF00E
:106F80000071826183618561816199F8010818252A
:106F90004FF080421123C9F8CC57C9F8C827C9F867
:106FA000D43700F0FF05002801F06982DC49D9F8E8
:106FB000C807DC4EDFF88CB3022589F80158F9F7D1
:106FC00027FCD94BC9F87C5001224FF001014AF649
:106FD000C8704FF4FA7489F801189862DC62DA60BC
:106FE0001A604FF000533360002099F8BD10C9F8C3
:106FF00074004FF48274C9E92300C9F88000C9F80D
:107000009400082207234FF400604FF4007AC9E986
:107010001BB4C9F88820C9F89830C9F87800C9F8B5
:1070200084A001F0FF04002901F0AA81D9F86C4086
:10703000022689F8BD60236823F040052560D9E960
:107040001C20D9F87840D9F87C30D9F88050024318
:107050002243D9F88800D9F88C401A432A43D9F83A
:107060009430D9F884500243224305F40070D9F8D3
:107070006C401A4302432260B9F88620D9F8905038
:10708000D9F86C0002F004032B434360C46900216B
:1070900024F400620125C261C9F8C01089F8BD500E
:1070A00099F80131C9F8D81001F1804E0C24C9E9D2
:1070B0003411C9F8E010C9F8E4104FF4E1300EF5CE
:1070C0008831C9F8DC40C9F8C810C9F8CC0003F011
:1070D000FF04002B01F05482D9F8C820D9F8D05011
:1070E000242689F80161D06820F40054D460116925
:1070F000D9F8D46021F4405333431361D9F8D80050
:10710000D468D9F8DC30D9F8E460054324F4164C8F
:107110001D432CF00C0135430D43D5605569D9F85A
:10712000E04025F4407020435061D9F8E410B1F5F7
:10713000004F01F0C5817D4B9A4200F08B8403F52E
:107140008066B24200F08684FFF712F9D9F8CC20AD
:107150004FF0190B940064260BFB00F5B5FBF4F01F
:10716000B0FBF6F10C01FFF703F9D9F8CC205B4630
:10717000950003FB00F0B0FBF5FBFFF7F9F8D9F839
:10718000CC104FF0190A8B000AFB00F0B0FBF3F2B1
:10719000B2FBF6F506FB15B001013231B1FBF6FB8F
:1071A000FFF7E6F8D9F8CC20534603FB00F0910036
:1071B0000BF0F005B0FBF1FAFFF7DAF8D9F8CC30B4
:1071C00019219A0001FB00F0B0FBF2F1B1FBF6F0DF
:1071D00006FB10A31A013232B2FBF6F606F00F01DD
:1071E00029432144D9F8C840A160D9F8C800DFF884
:1071F00058E1046924F490410161466926F02A03AC
:107200004361C568002245F400542026C460C9F8D3
:10721000042189F8016189F8026199F85512444DF9
:10722000C9F82C224FF48043C9E98D225E20FE224A
:10723000C9E986E5C9F82402C9F83022C9F828321C
:10724000C9F8203201F0FF04002901F02582DFF89F
:10725000FC80D9F81852242089F855022A6822F0B7
:1072600001012960FFF784F8D9F81822314BB0FBEF
:10727000F3F65660D9F81C422F4DAC4200F231842F
:10728000013640F6FC7316626100B0FBF1F61E4257
:1072900008BF0426D661D9E98D5005431560D9E9A8
:1072A0008942D9F818621443B460D9E98B310B4391
:1072B000F3603568214B45F0010030602024002642
:1072C000C9F8586289F85542C9F8486289F8566287
:1072D00006F1804CD9F86040C9F828600CF590326E
:1072E0004FF480310125C9F83060C9F83860C9F819
:1072F0004060C9F84C60C9F82C60C9F85060C9F802
:107300002020C9F84830C9F82410C9F83450002C9E
:1073100000F00C85D9F86050EE0640F16E8417E05D
:107320000C08012000E100E00004004000100140D2
:10733000801A060040420F00A08601000100000FE5
:107340004000012000380040005400403811012066
:10735000D9F8200000230124FB6789F85C40066906
:10736000C8F8AC4326F0E0620261016941F00075A3
:107370000561466B26F01F024263416B41F0080530
:107380004563C04889F85C3002260823C8F8A83352
:10739000C8F8B0634FF400628361402580214FF448
:1073A0008053826185618161836199F8550220284B
:1073B00000F0D083B44D4FF0000C4FF0FF0E284684
:1073C000012189F82BC789F828E7FAF7E1FCA9F829
:1073D0002907AC4D4FF480034FF00061AB61A96108
:1073E000FBF70CFB72B6FA6AA84C546062B64FF415
:1073F000803600204FF400334FF48021AE6189F8CD
:10740000320789F81E07AB61A961AE61AB61A96162
:1074100072B6C9F81405C9F8180562B672B6C9F88B
:107420000803C9F80C0362B6FDF7E2FA4FF4002432
:107430004FF400024FF08056AC61AA61AE6198F83B
:10744000B8534DBB9248C9F894070123052188F829
:10745000B833C9F89817AA462C46D9F8946746F865
:107460002A40013599F898275FFA85FA5245F4D8F1
:1074700000258848C9F8240E0523C9F8283EAB46E4
:107480002946D9F8244E44F82B10013599F8286E76
:107490005FFA85FB5E45F4D87F4D804CC9F89C5758
:1074A00005F5E473C9F8A83705F53E7605F5986348
:1074B00005F1980205F59870C9F8B067C9F8BC37AE
:1074C000774E784BC9F8A027C9F8A40705F51871BD
:1074D00005F5647205F58560C9F8EC6FC9F8F83FE9
:1074E000714E724BC9F8AC1705F5AB65C9F8B427F6
:1074F000C9F8B807C9F8C0572663E3636C496D4AF9
:107500006D486E4D6E4E6F4BC9F8E01FC9F8F02FF5
:10751000C9F8F40FC9F8FC5FA66463656A496B4A51
:107520006B486C4D6C4E61600A236263A0632564F6
:10753000666689F8C4376949694A6A486A4D6B4E7C
:107540006B4B6164E2642065A5656A496A4A6B4DCC
:107550006B482166C4F880206A496B4ADFF844E230
:10756000DFF844A2DFF844B2C4E92936674E684B1D
:10757000C8F8F830C4E92B50664D6748C4F8E850A5
:10758000C4E93012C4E9386E6449654A654E664DF7
:10759000C8F8E810C4E93B0AC8F8F420C8F8FC6051
:1075A000C8F8005161486249624A634B634E644DBA
:1075B000C8F80401C8F80C11C8F83821C8F83C31E3
:1075C000C8F84061C8F844515E485F495F4A604B63
:1075D000604E614DC8F84801C8F84C11C8F85021F8
:1075E000C8F85431C8F85861C8F85C515B485C4928
:1075F0005C4A5D4B5D4E5E4DC8F86001C8F868118D
:10760000C8F86C21C8F888315A485B495B4A5C4B22
:10761000C4F8F4B0C8F8AC615A4EC8F8B0515A4D2D
:10762000C8F8B401C8F8B81158485949C8F8C82171
:10763000C8F8CC31574A584BC8F8E861C8F8EC5143
:10764000564E574DC8F8F001C8F8F411C8F8F821A3
:10765000C8F8FC31C8F8AC69C9F8145262B60948D8
:10766000802181610022012689F8102589F81F6791
:10767000FDF768F9FDF7BCF9C7F814807B6989F854
:10768000C66095E0000002406B0701209D020008E3
:10769000E81A0120FC1A0120F414012040100120F6
:1076A0007D1D0008F51E0008851F00082520000824
:1076B0002502000859370008F11E000829020008B9
:1076C000D5200008B9210008211F0008C11F0008AB
:1076D000C9480008AD600008512200081D48000894
:1076E0004121000879210008D94800086D4C0008A4
:1076F000414B0008D12100089D2200083D5100089F
:10770000594E0008DD220008E1220008E5220008A9
:10771000811D0008ED220008092D00082D37000802
:1077200041440008DD1E0008310200080D1F00085A
:10773000111F00085D1F0008B11F0008DD1F0008B1
:10774000012000088120000891200008C1200008C5
:10775000F1200008F944000895210008BD21000827
:107760004D220008350200086D220008CD220008D5
:10777000D1220008D5220008D9220008A925000836
:10778000352D00084D020008E9220008F12200080A
:107790000124000809240008091F0008A93900086D
:1077A000F9270008F12C000805240008192D00080D
:1077B00093F8D859A4F580647C60002D00F01E81F8
:1077C000012D00F02F84022D00F0E28299F8354758
:1077D000002C00F0C980D9F83817D9F82457B9F827
:1077E0003C676B1A9BB2B342C0F0BE80B9F83E57FB
:1077F00031449A1B4C1BA91868BAB1F5004F834657
:1078000003D91444A9F83C371E469822002107F1F9
:10781000B000FFF753F873BA99F834A7A7F8B7B0D8
:107820000526A022A7F8B93087F8B56087F8B6A07A
:1078300087F8B22001E097F8B5600636F1B207F19B
:10784000B000F9F705FA0028F5D0C4F30E040026BD
:10785000002D7BD007F1B0010023AE4203F10200FE
:1078600006F1010262D296B2B24A32F81420CA710D
:10787000013414F4004F4FEA1222A4B218BF0024BE
:1078800083B28A71AE4204F1010293461FFA82FC70
:1078900003F1020006F1010E01F1020246D2A54EEB
:1078A00036F81430D3711BF4004F1FFA8EF64FEAEE
:1078B000132393710CBF6446002483B2AE4202F1DD
:1078C000020A03F1020006F101022FD296B283B23E
:1078D000984A981CB86232F814008AF807000134FC
:1078E00014F4004F4FEA1022A4B218BF00248AF803
:1078F0000620AE4204F1010201F106001FFA82FBEC
:1079000006F1010E01F1080110D28A4E3B8D12F4EE
:10791000004F36F81420C2714FEA12260CBF5C46A5
:107920000024802B86711FFA8EF696D1D9B287F883
:10793000B51001E097F8B5100631C9B207F1B000F3
:10794000F9F786F90028F5D0B54283D8F96A794C61
:107950000D6A281B00234210C9F8242789F83537FF
:10796000C9F8383789F8343799F8295EC5B399F8DA
:107970002B4E99F828CED9F8243E601C5FFA80F887
:10798000C44589F82B8E05F1FF329CBF4FF00008EB
:1079900089F82B8E89F8292E53F8246096F805A0D3
:1079A000D6F88610B244CAF80610B6F88A50AAF87B
:1079B0000A5074790C34E1B23046F9F749F90028DD
:1079C000F7D099F8C407092806D809EB800B0130D5
:1079D000CBF89C6789F8C40799F8293E002B75D02D
:1079E000554DFEF7A9FA2C6924F00400286130BF38
:1079F0007B6993F8D859002D7FF4E2AE4FF4006212
:107A000029464E48FEF75AFF4D48C0F8E450284634
:107A1000FBF7EAFA7A69012682F8D869FCF7E8FFF1
:107A2000D4E6416843684749474C466803F03F0540
:107A3000B1FBF5F2454DFD626368C6F38810C3F3F0
:107A40000146013602FB00F07100B0FBF1F0286046
:107A5000FFF7BAB8FEF7A6FCD9F8CC604FF01908CA
:107A6000B40008FB00F06426B0FBF4F5B5FBF6F3B8
:107A70001C01FEF797FCD9F8CC1042468D0002FBA2
:107A800000F0B0FBF5FAFEF78DFCD9F8CC304FF0E2
:107A9000190B0BFB00F09A00B0FBF2F1B1FBF6F50D
:107AA00006FB15A003013233B3FBF6F202F0F0053A
:107AB000FEF778FCD9F8CC30594601FB00F09A006B
:107AC000B0FBF2FAFEF76EFCFFF778BB99F83027AF
:107AD000012A85D11E4989F831374FF000668E6141
:107AE0007EE74FF49671D9F8205201FB06F64FF469
:107AF0007A73B6FBF3F601361662BDB904EB4401A6
:107B0000B0FBF1F3C3F30B06B6FA86F14E0963003E
:107B10004EB9002D40F07E862344B0FBF3F444F4CC
:107B20000046FFF7B7BB0126FFF7B4BB192104FBE2
:107B300001F1E5E74000002000ED00E0141B01200A
:107B4000302201200024F400003802400000002010
:107B500000080240D9F82C6799F85522202A7FF4B2
:107B600029AC2146BC4833461922FAF75BF9014695
:107B700000287FF41FAC99F85432012B3FF41AAC63
:107B8000D9F8182289F854421368B44823F40063E2
:107B90001360D9F818224FF0220E89F855E289F8BF
:107BA0005652C9F85812C9F84402156845F4806065
:107BB0001060D9F818522A6842F480702860334661
:107BC00022464FF00110FAF72DF968B9D9F81812CA
:107BD000A348A0230B6132462146FAF781FE002814
:107BE00001F00284D9F85832D9F858329D4D4FF03F
:107BF000000B89F854B2FFF7DEBBD9F860309A4821
:107C0000D9F8244023F4885121F0020646F00202FC
:107C1000C9F86020456825F440334360416821433A
:107C20004160D9F82060914C726822F480707060D5
:107C30007568D9F8303045EA03217160726822F026
:107C4000407070607568D9F828301D437560B16860
:107C500021F40062B260B568D9F82C000543B56024
:107C6000D9F84830A342B46824F07061B160B268BA
:107C700000F08A80D9F848000243B260B36823F06C
:107C80004054B460B268D9F84C100A43B260B56889
:107C900025F00200B060B368D9F8384043EA4402E6
:107CA000B260D9F84010002969D0736843F40064C9
:107CB0007460726822F4604171604FF4604595FA17
:107CC000A5F0D9F844407168B0FA80F3621E9A407A
:107CD0000A437260F56AD9F83C3025F47000F0620E
:107CE000F26A5C1E42EA0451F162B56825F4007044
:107CF000B060B368D9F8504043EA4422B260B1683A
:107D000021F48065B560B068D9F8343040EA832446
:107D1000B4600026C9F86460D9F8602022F003013D
:107D200041F00105C9F86050FFF712BB504EC9F889
:107D3000644089F85C40C7F88040726C4D4842F45A
:107D400080737364716CC7F8B05001F480760322BD
:107D5000C7F8806007F1B001C7E92E45D7F8803039
:107D6000C7F8B420F8F7E4FB214612202A46F8F7BA
:107D70009FFA41484FF480240460FFF7CBBA75683E
:107D800025F400607060A5E722F04055B5607EE7FD
:107D9000D9F80803D9F80C13884203D007F1B000D2
:107DA000F9F7A0FF354ED9F82027D6F8EC40A31AF2
:107DB000002B3FF70BADB9F8065099F834077969F5
:107DC0002F4A013500264FF400040228A9F8065076
:107DD00081F8D869946100F04185294902268E61B5
:107DE000FC6AFE6A94F82F2094F82E80746A254964
:107DF000C7F88C10551CB8EB050348BF0333002CA3
:107E0000BCBF04F57F543F34C3F38700A213FF289F
:107E1000FA6100F017850130C5B21B4A1B4B3D6269
:107E20004FF0000A00265FFA8AF007F18D04012165
:107E3000B8617C62B962B346C7F810A0C7E92523D0
:107E40000E4BFE600022C7E92C22C7E92E22C3F8A0
:107E5000E4204FF4007421E0020010000000FFFF56
:107E6000020001006B070120002301400100000F08
:107E7000003802400004024000E100E0302201200E
:107E800000080240010000016CA100086CC100085C
:107E9000614E326922F00401316130BFD9F80853D4
:107EA000D9F80C63B54207F13200F1D0F9F71AFFA7
:107EB0000028EDD0D7F89410B7F93200D7F8B030D9
:107EC000D7F898C00D46013C35F804EBC7F894503C
:107ED0001EFB00FA4AF38F321A44C7F8B0204E88CE
:107EE000D7F8B43016FB00F848F38F31E646194452
:107EF000C7F8B4103EF8046BD7F8B830C7F898E06C
:107F000016FB00F646F38F3A5344C7F8B830BCF876
:107F1000026080FB00C84FEA9C3545EA884A3F4D25
:107F200016FB00F02E46D5F8E4505544C6F8E45050
:107F3000D7F8BC6040F38F303044A4B2C7F8BC001F
:107F4000002CABD105F5807E83FB0353AD0B45EAD6
:107F5000834C80FB0038980B82FB022540EA884A5C
:107F600081FB0118930B880BE24440EA884243EA04
:107F7000854CBD6AFB69FE689444E2449AFBFEFEB0
:107F80007345C8BF0025BD6236B326467C6A07F13B
:107F900090018C428BF0010B25D1BE6AD7F810B04E
:107FA000002E40F07D84386A0BF1010A824500F012
:107FB00049841B4D97F88C2005EB820CDCF8AC4D06
:107FC00094F80280217805EB880E05EB810BDEF832
:107FD000B43DDBF8B42D25E77C6A07F190018C42B3
:107FE0004FF00106D9D025460D4815F8011B7D62DA
:107FF00000EB8108D8F8AC3D03EB0B0E13F80B40F7
:108000009EF8025000EB840A00EB850CDAF8B42DE0
:10801000DCF8B43D12E700BF00ED00E030220120A3
:10802000C0CB0008F86A436A90F82F40058EFC61C7
:10803000002BBCBF03F57F533F339E133D627E622E
:108040000024D9F80823D9F80C138A423FF4BEABB8
:1080500007F1B000F9F746FE00283FF4B7AB99F8F6
:10806000AC0AD9F82087002800F07E8100F1FF3E9D
:108070000EEB8E0509EB850ABD49DAF81068B1F8F8
:10808000E8B0A8EB0602B2F5806F00F24985D9F896
:10809000B43AB84D1E469A1CC9F8B42A36F8041BE7
:1080A000C9F8B46A05EB0B1A5D88B7F9B03015FB57
:1080B00003FEBAF9025011FB03FC4EF38F364FEA70
:1080C0000B11AAF80260A6EB050E0E46A9494CF367
:1080D0008F328D5F8A53D9F8C46AD9F8B81A521B07
:1080E000D9F8C85A3244C9F8C42A8E1C0EEB0502CE
:1080F0000D46C9F8B86AC9F8C82A35F804CBC9F8DA
:10810000B85A49881CFB03F511FB03FEBAF906C0F7
:10811000BAF904104EF38F32AAF80620A2EB0C0E27
:1081200045F38F36D9F8CC2AD9F8BC5AAAF804609E
:10813000761AD9F8D01A1644C9F8CC6A2A460EEB3A
:108140000106A91CC9F8BC1AC9F8D06A32F804CBD8
:10815000C9F8BC2A6D881CFB03FE15FB03F2BAF9B3
:108160000850C7F828804EF38F36AAF80860761BAF
:10817000D9F8D45A42F38F31BAF90A20AAF80A1072
:108180002E44A1EB020CC9F8D46AD9F8C01AD9F868
:10819000D86A0D460CEB06028E1CC9F8C06AC9F8F5
:1081A000D82A35F804EBC9F8C05A49887A691EFB09
:1081B00003F511FB03FC45F38F3683FB03354CF3CA
:1081C0008F3102EB8B0C9A0BBAF90C30AAF80C60C9
:1081D000F61AD9F8DC3A42EA8542BAF90E50AAF802
:1081E0000E103344D9F8E06AC9F8DC3A4D1B2E442E
:1081F000DCF8DC195E4DCCF8DC29521AD5F8E41015
:10820000C9F8E06A114401F58072C5F8E410BA615A
:108210001FFA80FA00F1010E01465D460BE0DCF822
:108220000C180131CCF80C180AF101031FFA83FA7B
:10823000F24551465ADC0AF0010309EB031B01EB3E
:108240008106DBF8CC3ADBF8C48ADBF8D02A09EBEC
:10825000860CDBF8C86A83FB033B9B0B43EA8B432A
:1082600082FB022B920B42EA8B4B88FB0828920B75
:108270005B4442EA884B86FB0662B60B46EA8248BC
:10828000D8444344DCF80488BA6993FBF2F64645C7
:108290005FFA8AFB4FEA8102C1DDB8F1000F02D11B
:1082A000BB6ACCF814380A4409EB820CB96ACCF8E2
:1082B00004680BF10106F2B27245CCF810188CF884
:1082C0000848CCF80C48AFDC02EB8208013209EB1D
:1082D000880BD2B27245CBF80448F5DD0AF10103F0
:1082E0001FFA83FAF245B9625146A4DD00EB80061D
:1082F00009EB86087B6AD8F80428D7F828C093428F
:1083000040F31C840135C5F30800194DA5F8E800B9
:1083100000287FF496AE184999F8B04A99F8B1CA86
:10832000164E0C448C4494F8C03794F8C2A79CF8BD
:10833000C4579CF8C64706EB830B06EB8A0806EB8E
:10834000850E06EB8401DBF8B42DD8F8B40DDEF809
:10835000B43DD1F8B46DC9F8B42AC9F8B80AC9F85F
:10836000BC3AC9F8C06A6BE6014BB3F8E8B08EE6D8
:108370003022012058240120B0ED0008C0CB0008B5
:10838000C149FC6589F8BC400A6BC0482A430A63AE
:108390000B6B2B40FB65FA6DBC650A6B2A430A63C5
:1083A0000B6B2B40BB65BA6D7C650A6B2A430A6375
:1083B0000B6B2B407B657A6D3C650A6B2A430A6325
:1083C0000B6B2B403B653A6DFC640A6C42F48043B6
:1083D0000B64096CC7F8B0A001F48042FA6407F19D
:1083E000B001FB6C0123C7E92D344FF48068C7F856
:1083F000BC30F8F79DF8C0F818A04FF4805BC7F8C0
:10840000B080F8F795F8C0F818804FF0050AC7F863
:10841000B0B0F8F78DF8C0F818B001224FF400534F
:10842000C7E92D54C7E92F2AC7F8B030F8F780F80C
:108430004FF400430122C7F8B030C7F8B450C7F872
:10844000BC20C7F8C0A0C7F8B840F8F771F84FF4DF
:108450008042C7F8B4500125C7F8B020C7F8C0A0C3
:10846000C7F8B840C7F8BC50F8F762F824200122DA
:108470002146F7F71DFF10207060FEF7D7BDBD64E1
:1084800089F800583146266C46F001002064226CC1
:1084900002F00103BB642A461C20BB6CF7F708FFFF
:1084A0007B494FF080560E607D64256C45F00200DC
:1084B0002064246C04F002027A647B6CFEF776BDC3
:1084C00001F1804E0EF5104C624500F0A1800CF5D4
:1084D0008065AA4200F09C80FDF74AFFD9F8CC30B5
:1084E0004FF0190A5A0064260AFB00F0B0FBF2F1C3
:1084F000B1FBF6F4FDF73CFFD9F8CC205346510010
:1085000003FB00F0B0FBF1FAFDF732FF2501D9F8CB
:10851000CC404FF0190B63000BFB00F0B0FBF3F203
:10852000B2FBF6F106FB11A0C4003234B4FBF6F343
:108530005A0002F4F87AFDF71BFFD9F8CC405946EF
:1085400001FB00F06300B0FBF3F4FDF711FFD9F875
:10855000CC1019224B0002FB00F0B0FBF3F2B2FB8F
:10856000F6F006FB1044E1003231B1FBF6F606F0FE
:1085700007032B44D9F8C8505344AB60FEF735BE0F
:10858000414BBC6689F800411A6B42482A431A6382
:10859000196B2940B966BA6E7C661A6B2A431A6356
:1085A000196B294079667A6E3C665A6C42F010016C
:1085B00059645B6CC7F8B46003F010064FF40072A6
:1085C0003E6607F1B00107263B6EC7F8B020C7E949
:1085D0002E45C7F8C0604FF01208F7F7A9FFC7E9AA
:1085E0002F564FF48065C7F8B840C7E92C58F7F705
:1085F0009FFF214622462520F7F75AFE2448D9F846
:10860000C84020214160E3680B43E360FEF764BD8E
:10861000FDF7C8FED9F8CC604FF0190B75000BFBC5
:1086200000F06426B0FBF5F2B2FBF6F10D01FDF7A8
:10863000B9FED9F8CC405B46620003FB00F0B0FB0A
:10864000F2FAFDF7AFFED9F8CC104FF0190B0BFB87
:1086500000F04B00B0FBF3F4B4FBF6F206FB12A003
:10866000C1003231B1FBF6F35C00FDF79BFED9F897
:10867000CC105A4604F4F87A02FB00F04B00B0FB31
:10868000F3F4FDF78FFE62E7003802400004024079
:1086900000E100E0000002407748BC6789F85442DE
:1086A000026BDFF8F88142F002010163036B03F013
:1086B0000205BD67BA6F7C67026B42F0020101637D
:1086C000036B03F002057D677A6F3C67026C42F42E
:1086D00000110164036C03F400153D673A6FFC66FA
:1086E000026B42F400110163006BC7F8B84000F45C
:1086F0000013012540226148FB6607F1B0014FF0ED
:10870000120B4FF0040AC7E92C2BFB6EC7F8C0A070
:10871000C7F8BC50F7F70CFF8023C7E92E45C7F810
:10872000B4B0C7F8C0A008F53A7BC7F8B030F7F787
:10873000FFFE4FF4000340214FF000700322C8E910
:10874000BC14C8E9C4234FF4806A4D4AC8F8EC024F
:108750004FF400115846C8E9BF44C8E9C144C8F8FD
:108760000C43C8F8F8A2C8F8181308F5527BC8F8EB
:10877000E822FAF787F9C9F84C02C8F858A34FF075
:1087800000704FF400034FF400114FF0030A3D4A0C
:10879000C8F84C03C8E9DCA3C8F878133A4BC8F80A
:1087A00048334FF400315846C8E9D444C8E9D744A7
:1087B000C8F86443C8F86C43C8F82023C8F86813A5
:1087C000FAF760F92F48C8F8800321462A462F207F
:1087D000C9F850B2F7F76CFD2C4A4FF400435360D0
:1087E000214622460B20F7F763FD284B30464FF415
:1087F00000611E4619602A462146F7F759FD2146B9
:10880000756002221F204FF00044F7F751FD3460DD
:10881000FEF71FBD192504FB05F5B0FBF5F040F48C
:108820004046FEF737BD1A4E706980F0800242F470
:108830000004B461B9F810500135A9F81050144B78
:1088400002219961124A134E1348C9F804634FF488
:108850000034C9F8F4029461FEF7B8BF99F83537CF
:10886000002B7FF4BAAAD9F82457C9F83857012049
:1088700089F83507FFF7B1BA00380240000402401A
:10888000B8600240580201201060024000E100E0A0
:1088900000080240DB1B0400B9A2010038110120CE
:1088A000B9F80860B86901360628A9F8086006D842
:1088B00009EB4B0ABAF884570135AAF88457D9F85E
:1088C0001C40D9F80813D9F80C33994A23445E1A8E
:1088D000C2F8F060974E984C4FF40030B061FD6ADA
:1088E0009822E86B0021FDF7E9FFA8464FF4897252
:1088F00000219148FDF7E2FFAC634FF400104FF404
:1089000000254FF480144FF480014FF4000298F8D2
:1089100028B0B561B461864DB061B161B261D9F87A
:108920002067C5F8F460002302227E68A9F8083C9D
:10893000FF24C9F8F03AC9F8F43AC9F8E83A89F8D6
:10894000ED3A0420032189F8EE2A0023002289F859
:10895000EC4AC6E9002389F8E5BA89F8F80A89F8EB
:10896000EF1A1B24FAF7BCFBFAF7BAFB631E1FFAD7
:1089700083FA0AF1FF351FFA85F808F1FF3B1FFA69
:108980008BF4FAF7ADFBFAF7ABFBFAF7A9FB601E25
:1089900086B2FAF7A5FB711E1FFA81FAFAF7A0FB5F
:1089A0000AF1FF3295B2FAF79BFB6B1E1FFA83F8B0
:1089B00008F1FF3B1FFA8BF4FAF792FBFAF790FBF2
:1089C000601E84B2002CCFD15A4920268E61C7E99F
:1089D0000844C7E90344C7E9064408225649BC6273
:1089E000A346A246204625462646A446BA604FF036
:1089F0008008FB6891F800E05B0018EA0E0F18BFD2
:108A000043F001039BB2FB605FEA580340F0C4816E
:108A100091F801803B69C8F3801E91F901805B00E9
:108A20004EEA4C0243EAD8731FFA82FC9AB23A61CA
:108A300001314FF02008BB695A000B7818EA030F88
:108A400018BF42F0010292B25FEA5803BA6140F0E7
:108A5000C48191F801E091F901207600CEF38018ED
:108A600046EAD27348EA45059EB2ADB201312023F1
:108A70000A786400134218BF44F001045B08A4B2F2
:108A800040F0C48191F801E091F901804000CEF3FB
:108A9000801242EA4A0340EAD8701FFA83FA80B291
:108AA000013120234FEA4B0291F800B013EA0B0F7B
:108AB00018BF42F001021FFA82FB5A0840F0C2813F
:108AC000BB6A91F801804FEA430E3B6AC8F38012FB
:108AD00042EA430891F901301FFA88F23A624EEAFD
:108AE000D37293B2BB62013120227B6A91F800E01D
:108AF0005B0012EA0E0F18BF43F001039BB25FEA5E
:108B000052087B6240F0C181FA6991F901E053009B
:108B100043EADE7293B2FB6101314FF04008C4E1D9
:108B20005846FAF761FA99F8AC0AFFF7B0BA00BFF5
:108B300030220120000802404C0C0120D8F80C38EB
:108B40003A6A8B498B4EC9F804139342C9F8F46210
:108B50000BD200283FF4D6ABD9F81038ACEB0301A8
:108B60004302803399427FF6CDAB10F0010B824E69
:108B7000824909EB0B0A14BF04234FF48023B3612D
:108B80009AF8B02A0132D3B201EB8B0C022BDCF83D
:108B9000AC2D12BF8AF8B03A00238AF8B04AD65CEE
:108BA000764901EB860A13440135DAF8B42D734E89
:108BB000C5F3080809EBCB0C02EB8801CCF8B41A1A
:108BC0009B7806EB830A6E4BDAF8B42D02EB880132
:108BD0006C4ACCF8B81A0FFA8BF603EBCB0302EB16
:108BE000CB011C805C809C80DC801C825C829C822F
:108BF000DC821C845C849C84DC841C865C869C8671
:108C0000DC86A3F84040A3F84240A3F84440A3F810
:108C10004640A3F85040A3F85240A3F85440A3F8AC
:108C20005640A3F86040A3F86240A3F86440A3F85C
:108C30006640A3F87040A3F87240A3F87440A3F80C
:108C4000764080339942CCD14F4A02EB061B360165
:108C50001F289451CBE90144CBF80C4006D809EB0E
:108C60004008B8F844370133A8F844375FFA8EF16A
:108C7000FE6989F8AC1A01EB810209EB820EB14260
:108C8000CEF80C48FFF43FAB012940F22983421E85
:108C9000D5B209F618033D4E4FF0140C1CFB0534F9
:108CA000A01B3B4DA0F11402900805FB00F0013021
:108CB00010F00702D9F810584FF0000328D0012A0D
:108CC00020D0022A1AD0032A14D0042A0ED0052A52
:108CD00008D0062A02D0336A14365B1B306A421B66
:108CE00014361344306A421B14361344306A421B54
:108CF00014361344306A421B14361344306A421B44
:108D000014361344306A1436421BB44213441ED046
:108D1000306A421B706B1344421BB06C1344421BFD
:108D2000F06D1344421B306F1344421BD6F884008D
:108D30001344421BD6F898001344421BD6F8AC00EB
:108D4000A0361344B442A0EB05021344E0D1B3FBB8
:108D5000F1F6D9F810487B69013104EB012A0D497D
:108D600056440225C1F8EC6083F8D859FEF72EBDB1
:108D7000DB1B0400B9A2010000080240C0CB0008C0
:108D80005824012058440120040B012044080120EC
:108D9000CDCCCC0C3022012013EA0E0F3B694FEAF8
:108DA000430318BF43F001039BB23B615FEA9803A2
:108DB00040F098824B78BA69C3F3801E4EEA4208AD
:108DC00091F901E04FEA4C0C1FFA88F34CEADE728D
:108DD000BB611FFA82FC013120230A78760013421E
:108DE00018BF46F001065B08B6B240F0998291F8D0
:108DF00001E091F901206D00CEF3801845EAD273AD
:108E000048EA44049DB2A4B2013120230A7840000C
:108E1000134218BF40F001005B0880B240F0998215
:108E20004FEA4A0391F801A091F90180CAF3801E2C
:108E30004EEA4B0243EAD8731FFA82FB1FFA83FA09
:108E400001312022BB6A91F800E05B0012EA0E0FAC
:108E500018BF43F001039BB25208BB6240F09A82F4
:108E60003A6A4B784FEA42087A6AC3F3801E4EEAA8
:108E700042039AB291F901307A6248EAD3781FFA34
:108E800088F23A6201314FF02008FA6953000A78FB
:108E900018EA020F18BF43F001039BB25FEA5808BB
:108EA000FB6102D101314FF08008BA68531E13F004
:108EB000FF02BA607FF49DADD7E9068E3969A7F845
:108EC0009610A7F89C60A7F89E50BE6A3D6AA7F866
:108ED000A040A7F8A2007C6AF868A7F8A86007F18C
:108EE000320207F1B001A7F898C0A7F89A80A7F856
:108EF000A4A0A7F8A6B0A7F8AA50A7F8AC40A7F876
:108F0000AEE0A7F89400F9F7BFFB07F1960600283A
:108F10003FF489AC7A8E9AB1FB6AB9F80E50D96BDE
:108F2000AD4891F888C055FA82F49444A9F80E40EF
:108F300081F888C0426982F0400A4AF48003836164
:108F4000B7F8960007F1B20107F132020236F9F7DD
:108F50009BFB00283FF467AC7D8E9DB1FC6AB9F89D
:108F60000E20E06B90F8888052FA85FBA8449A4D59
:108F700080F88880A9F80EB06B6983F0400444F44F
:108F80008000A861FA6A0231354692460E4635F8ED
:108F9000020B07F132023146F9F776FB00283FF465
:108FA00042AC798E99B1DAF83C40B9F80EC094F829
:108FB000888089485CFA81FB8844A9F80EB084F85F
:108FC0008880436983F0400242F480018161023667
:108FD000288807F132023146F9F756FB00283FF4A2
:108FE00022AC7C8E9CB1DAF83C00B9F80EC090F847
:108FF0008880794A5CFA84FBA044A9F80EB080F816
:109000008880536983F0400141F48004946168884A
:1090100007F13202B11CF9F737FB00283FF403AC2B
:10902000788E98B1DAF83C20B9F80EC092F88880B2
:1090300069495CFA80FB8044A9F80EB082F8888008
:109040004B6983F0400444F480008861A88807F1EC
:109050003202311D0635F9F717FB00283FF4E3AB68
:109060007A8E9AB1DAF83C10B9F80EC091F888807F
:10907000594C5CFA82FB9044A9F80EB081F88880C4
:10908000636983F0400040F48002A26107F1B001FF
:10909000A94206F106067FF47AAF0020C7F88C00DB
:1090A00007F1AE05C7F88F00044607F18C0184462E
:1090B00003E0382C1FFA8AFC50D035F802AFCAF30F
:1090C000C00E04F007004EEA4C0C07280FFA8CFB88
:1090D00014BF1FFA8BF00020CAF3800848EA40034F
:1090E00004F1010604F102001FFA80FEB2B202F0A0
:1090F00007061AB2734608BF01F801BB072E03F03A
:109100000706BE62BE6A0ABF01F8012B1FFA82FE83
:109110004FF0000ECAF3400242EA4E00072E0FFA4B
:1091200080FB04F1030314BF1FFA8BF600260AF03C
:1091300001021FFA83F842EA460008F0070608BF5A
:1091400001F801BB0434072E0FFA80FAA4B2B0D1A3
:10915000382C01F801AB4FF0000CAED197F98C0020
:1091600097F88C30002807F18C02C0F2AA835E00C9
:10917000F4B2600014F0800F18BF80F0D500C3B2C5
:109180005E0013F0800F18BF86F0D506F4B26100C0
:1091900014F0800F18BF81F0D501CDB215F0800F0B
:1091A0004FEA450018BF80F0D500C3B213F0800F1E
:1091B0004FEA430618BF86F0D506F4B2610014F0FA
:1091C000800F18BF81F0D501CDB2290600F174835C
:1091D0006800C4B23DE000BF000802405900CCB2B4
:1091E000630014F0800F18BF83F0D503DEB2710066
:1091F00016F0800F18BF81F0D501CCB2650014F0D5
:10920000800F18BF85F0D505E8B2430010F0800F3D
:1092100018BF83F0D503DEB216F0800F4FEA460187
:1092200018BF81F0D501CCB214F0800F4FEA44058D
:1092300018BF85F0D505E8B210F0800F4FEA400363
:1092400007F1920618BF83F0D5039642DCB200F016
:109250008281517861404C0011F0800F18BF84F07A
:10926000D504E5B2680015F0800F18BF80F0D50076
:10927000C3B25E0013F0800F18BF86F0D506F1B2BE
:109280004C0011F0800F18BF84F0D504E5B26800DF
:1092900015F0800F18BF80F0D500C3B25E0013F048
:1092A000800F18BF86F0D506F1B24C0011F0800F88
:1092B00018BF84F0D504E5B215F0800F4FEA4500E1
:1092C00018BF80F0D5009678C3B2734001321C06F7
:1092D00002F1010282D55D0085F0D500C4B27FE7BE
:1092E000002334E513EA0E0F4FEA4C0318BF43F096
:1092F00001035FEAD8081FFA83FC7FF49CABBA69CC
:1093000091F801E0530091F90120CEF3801843EA6F
:10931000D2739AB248EA4606B6B2BA610131202346
:109320000A786D00134218BF45F001055B08ADB225
:109330007FF49EAB91F801E091F901206400CEF337
:10934000801844EAD27348EA40009CB280B20131EE
:1093500020234FEA4A0291F800A013EA0A0F18BF2F
:1093600042F001025B081FFA82FA7FF49BAB91F88E
:1093700001E0BA6ACEF3801848EA42039AB291F942
:109380000130BA624FEA4B0B4BEAD3721FFA82FBF1
:10939000013120223B6A91F800805B0012EA080F3D
:1093A00018BF43F001039BB252083B627FF49DABB0
:1093B0007B6A91F801804FEA430EFB69C8F3801283
:1093C00091F9018042EA430293B24EEAD872FB61FE
:1093D00093B27B6201314FF0200866E554F8042B0C
:1093E00090470225FDF784BCD9F81852C7F88800C9
:1093F0006A69C7F88820A969C7F888103046D7F885
:109400008830F8F737FD38B9D9F818321861304686
:10941000F8F730FD014660B1D9F85842042C7EF4CB
:10942000E3ABD9F81822166846F400701060FEF716
:10943000DBBBD9F81802056845F480720260334638
:1094400022464FF00110F8F7EDFC00287EF4CCAB7B
:109450002146D9F81842BC48A12323613246F9F7C6
:109460003FFA00287EF4BEABD9F818120020C7F8E6
:1094700084004D69C7F884508A69C7F88420304653
:10948000D7F88430F9F7F4F9002858D1D9F8184200
:109490002369616989F8283711F0040133D0236901
:1094A00089F8293701463346A8480122F8F7BAFC63
:1094B00000287DF47FAFD9F81802016841F40075E7
:1094C0000560D9F8184299F82807226989F82A27EF
:1094D00026699F4D89F82B674FF0000A2023FF284B
:1094E00089F8553289F854A289F856A27DF463AF01
:1094F00001212846F8F74CFCB9F8291781427DF480
:109500005AAFFDF766BF914833460122F8F78AFC4F
:1095100000287DF44FAF3346D9F818628B48356880
:1095200025F480623260D9F81842266989F82967E3
:109530000122F8F777FC0028BDD0FDF73BBFD9F832
:109540005832FDF737BF54F8042B4FF0020890470C
:10955000C146FDF765BB34B1B9F80C300133A9F849
:109560000C30FFF76CB9FA6A7A4ED56BD7F88C10CD
:10957000B7F89000A8804FF400132960B3616A79AE
:10958000002A00F0DF800232D500F96A486B90F8BB
:1095900000E090F801B075446B1E93FBFEF61BFBD8
:1095A00006F2703295B2B5F5096F3FF648A999F801
:1095B000F81A6818431E93FBF1F8A8F11C0A1FFA69
:1095C0008AF6002E43D0721E012502F00708F9F733
:1095D00087FDAE423BD941460FFA88F019B3012806
:1095E0001BD0022816D0032811D004280CD005283F
:1095F00007D0062802D0F9F773FD0225F9F770FDB0
:109600000135F9F76DFD0135F9F76AFD0135F9F717
:1096100067FD0135F9F764FD01350135F9F760FDA6
:10962000ABB29E4213D90835F9F75AFDF9F758FD48
:10963000F9F756FDF9F754FDF9F752FDF9F750FD2A
:10964000F9F74EFDF9F74CFDAAB29642EBD8FAF7BE
:10965000A9FA00283FF4F3A83F48D9F82017D0F81A
:10966000F45099F8F86AD9F8F00A4A1B3346D9F849
:10967000F41AF8F70DFFFB6AB9F8088CDD6B79680E
:1096800085F886000023D1E900014246FCF7AAFED6
:10969000002982460B4661DBB0F1004F71F10002F8
:1096A0004FF0010B0EDB4FEA9A0242EA837ABAF1DD
:1096B000004F4FEAA3034FEA4B0073F100025FFA39
:1096C00080FBF0DA990341EA9A4000234FEA8A3A94
:1096D0004FF080419A0842EA81739A454FEAA1010E
:1096E00070EB0102F6DB53EA010228D01A46002390
:1096F0003C62BB6294087C62BC6A12EB030C41EBD7
:10970000040EE24570EB0E040BDBBAEB0C0ABC6AEC
:1097100060EB0E00921841EB010CD3184CEB0402E5
:10972000BA627C6A44EA8172BC6A5B08891043EAC7
:10973000C4736410BC6252EA0104DBD13C6A8BFB47
:1097400003BE0EE0254620E70200010004000100F0
:109750006B07012000080240302201204FF0FF3B40
:10976000DE46A6FB0BA006FB0E021AEB0A0C42EB30
:1097700002011CEB0A0342EB0100C10041EA5370F5
:10978000DB0013EB0A0142EB0002CB00D0006FF4C8
:10979000FF7B40EA51725B4572F1FF3116DB002A14
:1097A00004DA40F2FF141B1942F10002590A41EA9F
:1097B000C25E1EF500504FEA622444F1000A830B9A
:1097C00043EA8A42FF2A28BFFF22D4B2F96A85F809
:1097D00087403E4C91F82E00D4F8F02099F8E5BA75
:1097E000D9F8E83A99F8EC4AC5F88C200430A2EB95
:1097F000402C0BFB08F106FB03F3B3FBF1F06B7994
:1098000099F8ED1AC5F890C085F8890085F88A4066
:1098100085F88B100BB10233DB00F86A446B94F8C7
:1098200000806078434403F1FF3E9EFBF8F300FBA9
:1098300003F3711E70330BFB0314B4FBF6F602EB5B
:10984000462A7A69C5F894A0D2F8AC4954B12846A2
:109850001F4D696981F0080C4CF40023AB61A047EF
:10986000FE6AF063B9F80A0099F83447194D0130DF
:109870004FF40022A9F80A004FF48011AA614FF4B6
:1098800000134FF480064FF400000222032CA9615C
:10989000AB61AE61A861AA617EF4D4AF99F8354797
:1098A000002C7EF4CFAFD9F82457C9F838570121DE
:1098B00089F83517FEF7C6BF6B0083F0D506F4B202
:1098C000C7E4590081F0D505ECB252E43022012002
:0898D000000002400008024004
:1098D800AAAA000001000101010201030104010517
:1098E8000106010701080109010A010B010C010D1C
:1098F800010E010F0110011101120080000000008B
:109908000408000009260008892600080B1000003A
:1099180049260008152700080D000B00080007005D
:109928000400020001000E00D506B30500048F03F1
:109938000002000180007F004000200010000800A5
:109948000400020001006907AA0066001E00FF006B
:10995800AAAA66661E1EFE01FFFF0000000610167A
:1099680000061016000000405A2E212CEC3FDDFCAA
:10997800CD298ACFBBF94FC08CCDA1D8B2C064091C
:1099880026DB53347C0CC53E12363D22143E74F05F
:109998008B1F51C86CEDC2C2D6C63AE3BEC38F1541
:1099A80011E6823A7D18203BB63B0817DA39A3E462
:1099B80013143BC3D5E18FC752C2EFEE1BC9E72092
:1099C800FBF1713E8E2336350E3FF10A6733E1D93C
:1099D800D5077CC067D787CE2DC04BFB95D0FA2A18
:1099E8006EFEFB3F412D412DFB3F6EFEFA2A95D0BE
:1099F8004BFB2DC087CE67D77CC0D507E1D967332D
:109A0800F10A0E3F36358E23713EFBF1E7201BC964
:109A1800EFEE52C28FC7D5E13BC31314A3E4DA3982
:109A28000817B63B203B7D18823A11E68F15BEC356
:109A38003AE3D6C6C2C26CED51C88B1F74F0143E0F
:109A48003D221236C53E7C0C533426DB6409B2C075
:109A5800A1D88CCD4FC0BBF98ACFCD29DDFCEC3F16
:109A6800212C5A2E00400000212CA6D1DDFC14C068
:109A78008ACF33D64FC04506A1D8743264094E3F09
:109A88005334DA24C53E84F33D22EEC974F0ECC1A8
:109A980051C875E0C2C294123AE32A398F15423C84
:109AA800823AEF19203B83E708174AC4A3E426C685
:109AB8003BC3EDEB8FC72B1EEFEEAE3DE720E5363F
:109AC800713E050E363572DCF10AF2C0E1D999CC47
:109AD8007CC02BF887CE99284BFBD33FFA2A6B2FF3
:109AE800FB3F9201412DBFD26EFE05C095D006D531
:109AF8002DC0B50467D77931D507843F67331F2652
:109B08000E3F0FF58E23CACAFBF18FC11BC919DF9F
:109B180052C21111D5E171381314C53CDA395D1BF5
:109B2800B63BF8E87D18E0C411E67EC5BEC371EA0D
:109B3800D6C6C61C6CED3E3D8B1FAF37143E8C0F4E
:109B48001236C3DD7C0C3BC126DBADCBB2C09CF624
:109B58008CCD5F27BBF9B13FCD297630EC3F23038D
:109B68005A2EDFD3000000C0A6D1DFD314C02303D0
:109B780033D676304506B13F74325F274E3F9CF6A8
:109B8800DA24ADCB84F33BC1EEC9C3DDECC18C0F45
:109B980075E0AF3794123E3D2A39C61C423C71EA43
:109BA800EF197EC583E7E0C44AC4F8E826C65D1B02
:109BB800EDEBC53C2B1E7138AE3D1111E53619DFB2
:109BC800050E8FC172DCCACAF2C00FF599CC1F26E8
:109BD8002BF8843F99287931D33FB5046B2F06D5EC
:109BE800920105C0BFD2BFD205C0920106D56B2F26
:109BF800B504D33F79319928843F2BF81F2699CC97
:109C08000FF5F2C0CACA72DC8FC1050E19DFE5363E
:109C18001111AE3D71382B1EC53CEDEB5D1B26C600
:109C2800F8E84AC4E0C483E77EC5EF1971EA423C0C
:109C3800C61C2A393E3D9412AF3775E08C0FECC133
:109C4800C3DDEEC93BC184F3ADCBDA249CF64E3FAD
:109C58005F277432B13F4506763033D6230314C0EC
:109C6800DFD3A6D100C00000DFD35A2E2303EC3F78
:109C78007630CD29B13FBBF95F278CCD9CF6B2C0B9
:109C8800ADCB26DB3BC17C0CC3DD12368C0F143EFA
:109C9800AF378B1F3E3D6CEDC61CD6C671EABEC3FE
:109CA8007EC511E6E0C47D18F8E8B63B5D1BDA39DD
:109CB800C53C13147138D5E1111152C219DF1BC903
:109CC8008FC1FBF1CACA8E230FF50E3F1F266733DB
:109CD800843FD507793167D7B5042DC006D595D00F
:109CE80005C06EFEBFD2412D9201FB3F6B2FFA2AB1
:109CF800D33F4BFB992887CE2BF87CC099CCE1D970
:109D0800F2C0F10A72DC3635050E713EE536E72001
:109D1800AE3DEFEE2B1E8FC7EDEB3BC326C6A3E48B
:109D28004AC4081783E7203BEF19823A423C8F1553
:109D38002A393AE39412C2C275E051C8ECC174F0F2
:109D4800EEC93D2284F3C53EDA2453344E3F6409FC
:109D58007432A1D845064FC033D68ACF14C0DDFC73
:109D6800A6D1212C000000405A2E212CEC3FDDFC0E
:109D7800CD298ACFBBF94FC08CCDA1D8B2C0640918
:109D880026DB53347C0CC53E12363D22143E74F05B
:109D98008B1F51C86CEDC2C2D6C63AE3BEC38F153D
:109DA80011E6823A7D18203BB63B0817DA39A3E45E
:109DB80013143BC3D5E18FC752C2EFEE1BC9E7208E
:109DC800FBF1713E8E2336350E3FF10A6733E1D938
:109DD800D5077CC067D787CE2DC04BFB95D0FA2A14
:109DE8006EFEFB3F412D412DFB3F6EFEFA2A95D0BA
:109DF8004BFB2DC087CE67D77CC0D507E1D9673329
:109E0800F10A0E3F36358E23713EFBF1E7201BC960
:109E1800EFEE52C28FC7D5E13BC31314A3E4DA397E
:109E28000817B63B203B7D18823A11E68F15BEC352
:109E38003AE3D6C6C2C26CED51C88B1F74F0143E0B
:109E48003D221236C53E7C0C533426DB6409B2C071
:109E5800A1D88CCD4FC0BBF98ACFCD29DDFCEC3F12
:109E6800212C5A2E00400000212CA6D1DDFC14C064
:109E78008ACF33D64FC04506A1D8743264094E3F05
:109E88005334DA24C53E84F33D22EEC974F0ECC1A4
:109E980051C875E0C2C294123AE32A398F15423C80
:109EA800823AEF19203B83E708174AC4A3E426C681
:109EB8003BC3EDEB8FC72B1EEFEEAE3DE720E5363B
:109EC800713E050E363572DCF10AF2C0E1D999CC43
:109ED8007CC02BF887CE99284BFBD33FFA2A6B2FEF
:109EE800FB3F9201412DBFD26EFE05C095D006D52D
:109EF8002DC0B50467D77931D507843F67331F264E
:109F08000E3F0FF58E23CACAFBF18FC11BC919DF9B
:109F180052C21111D5E171381314C53CDA395D1BF1
:109F2800B63BF8E87D18E0C411E67EC5BEC371EA09
:109F3800D6C6C61C6CED3E3D8B1FAF37143E8C0F4A
:109F48001236C3DD7C0C3BC126DBADCBB2C09CF620
:109F58008CCD5F27BBF9B13FCD297630EC3F230389
:109F68005A2EDFD3000000C0A6D1DFD314C02303CC
:109F780033D676304506B13F74325F274E3F9CF6A4
:109F8800DA24ADCB84F33BC1EEC9C3DDECC18C0F41
:109F980075E0AF3794123E3D2A39C61C423C71EA3F
:109FA800EF197EC583E7E0C44AC4F8E826C65D1BFE
:109FB800EDEBC53C2B1E7138AE3D1111E53619DFAE
:109FC800050E8FC172DCCACAF2C00FF599CC1F26E4
:109FD8002BF8843F99287931D33FB5046B2F06D5E8
:109FE800920105C0BFD2BFD205C0920106D56B2F22
:109FF800B504D33F79319928843F2BF81F2699CC93
:10A008000FF5F2C0CACA72DC8FC1050E19DFE5363A
:10A018001111AE3D71382B1EC53CEDEB5D1B26C6FC
:10A02800F8E84AC4E0C483E77EC5EF1971EA423C08
:10A03800C61C2A393E3D9412AF3775E08C0FECC12F
:10A04800C3DDEEC93BC184F3ADCBDA249CF64E3FA9
:10A058005F277432B13F4506763033D6230314C0E8
:10A06800DFD3A6D100C00000DFD35A2E2303EC3F74
:10A078007630CD29B13FBBF95F278CCD9CF6B2C0B5
:10A08800ADCB26DB3BC17C0CC3DD12368C0F143EF6
:10A09800AF378B1F3E3D6CEDC61CD6C671EABEC3FA
:10A0A8007EC511E6E0C47D18F8E8B63B5D1BDA39D9
:10A0B800C53C13147138D5E1111152C219DF1BC9FF
:10A0C8008FC1FBF1CACA8E230FF50E3F1F266733D7
:10A0D800843FD507793167D7B5042DC006D595D00B
:10A0E80005C06EFEBFD2412D9201FB3F6B2FFA2AAD
:10A0F800D33F4BFB992887CE2BF87CC099CCE1D96C
:10A10800F2C0F10A72DC3635050E713EE536E720FD
:10A11800AE3DEFEE2B1E8FC7EDEB3BC326C6A3E487
:10A128004AC4081783E7203BEF19823A423C8F154F
:10A138002A393AE39412C2C275E051C8ECC174F0EE
:10A14800EEC93D2284F3C53EDA2453344E3F6409F8
:10A158007432A1D845064FC033D68ACF14C0DDFC6F
:10A16800A6D1212C00000040DA395D1B793167D770
:10A1780074F0ECC13BC184F3E1D967332B1E71380D
:10A18800EC3FDDFC7D18E0C406D595D0C2C2941220
:10A198009CF64E3F36358E23E53619DFBBF94FC0A6
:10A1A800BEC371EABFD2412D8F15423CB13F45066F
:10A1B800E7201BC972DCCACAB2C064096CED3E3D17
:10A1C8006B2FFA2A203B83E7230314C08FC7D5E1FE
:10A1D80099CC1F267C0CC53E143E8C0F992887CE3F
:10A1E800A3E426C600C00000A3E4DA39992879312F
:10A1F800143E74F07C0C3BC199CCE1D98FC72B1E5F
:10A208002303EC3F203B7D186B2F06D56CEDC2C2B3
:10A21800B2C09CF672DC3635E720E536B13FBBF9B3
:10A228008F15BEC3BFD2BFD2BEC38F15BBF9B13F16
:10A23800E536E720363572DC9CF6B2C0C2C26CED5A
:10A2480006D56B2F7D18203BEC3F23032B1E8FC7B1
:10A25800E1D999CC3BC17C0C74F0143E7931992832
:10A26800DA39A3E4000000C026C6A3E487CE992803
:10A278008C0F143EC53E7C0C1F2699CCD5E18FC7A8
:10A2880014C0230383E7203BFA2A6B2F3E3D6CED75
:10A298006409B2C0CACA72DC1BC9E7204506B13FCF
:10A2A800423C8F15412DBFD271EABEC34FC0BBF9E6
:10A2B80019DFE5368E2336354E3F9CF69412C2C21E
:10A2C80095D006D5E0C47D18DDFCEC3F71382B1E17
:10A2D8006733E1D984F33BC1ECC174F067D77931B6
:10A2E8005D1BDA39004000005D1B26C667D787CEA4
:10A2F800ECC18C0F84F3C53E67331F267138D5E156
:10A30800DDFC14C0E0C483E795D0FA2A94123E3DE0
:10A318004E3F64098E23CACA19DF1BC94FC04506C0
:10A3280071EA423C412D412D423C71EA45064FC03D
:10A338001BC919DFCACA8E2364094E3F3E3D9412D9
:10A34800FA2A95D083E7E0C414C0DDFCD5E1713862
:10A358001F266733C53E84F38C0FECC187CE67D7C1
:10A3680026C65D1B00000040DA395D1B793167D7CE
:10A3780074F0ECC13BC184F3E1D967332B1E71380B
:10A38800EC3FDDFC7D18E0C406D595D0C2C294121E
:10A398009CF64E3F36358E23E53619DFBBF94FC0A4
:10A3A800BEC371EABFD2412D8F15423CB13F45066D
:10A3B800E7201BC972DCCACAB2C064096CED3E3D15
:10A3C8006B2FFA2A203B83E7230314C08FC7D5E1FC
:10A3D80099CC1F267C0CC53E143E8C0F992887CE3D
:10A3E800A3E426C600C00000A3E4DA39992879312D
:10A3F800143E74F07C0C3BC199CCE1D98FC72B1E5D
:10A408002303EC3F203B7D186B2F06D56CEDC2C2B1
:10A41800B2C09CF672DC3635E720E536B13FBBF9B1
:10A428008F15BEC3BFD2BFD2BEC38F15BBF9B13F14
:10A43800E536E720363572DC9CF6B2C0C2C26CED58
:10A4480006D56B2F7D18203BEC3F23032B1E8FC7AF
:10A45800E1D999CC3BC17C0C74F0143E7931992830
:10A46800DA39A3E4000000C026C6A3E487CE992801
:10A478008C0F143EC53E7C0C1F2699CCD5E18FC7A6
:10A4880014C0230383E7203BFA2A6B2F3E3D6CED73
:10A498006409B2C0CACA72DC1BC9E7204506B13FCD
:10A4A800423C8F15412DBFD271EABEC34FC0BBF9E4
:10A4B80019DFE5368E2336354E3F9CF69412C2C21C
:10A4C80095D006D5E0C47D18DDFCEC3F71382B1E15
:10A4D8006733E1D984F33BC1ECC174F067D77931B4
:10A4E8005D1BDA39004000005D1B26C667D787CEA2
:10A4F800ECC18C0F84F3C53E67331F267138D5E154
:10A50800DDFC14C0E0C483E795D0FA2A94123E3DDE
:10A518004E3F64098E23CACA19DF1BC94FC04506BE
:10A5280071EA423C412D412D423C71EA45064FC03B
:10A538001BC919DFCACA8E2364094E3F3E3D9412D7
:10A54800FA2A95D083E7E0C414C0DDFCD5E1713860
:10A558001F266733C53E84F38C0FECC187CE67D7BF
:10A5680026C65D1B00000040DA395D1B793167D7CC
:10A5780074F0ECC13BC184F3E1D967332B1E713809
:10A58800EC3FDDFC7D18E0C406D595D0C2C294121C
:10A598009CF64E3F36358E23E53619DFBBF94FC0A2
:10A5A800BEC371EABFD2412D8F15423CB13F45066B
:10A5B800E7201BC972DCCACAB2C064096CED3E3D13
:10A5C8006B2FFA2A203B83E7230314C08FC7D5E1FA
:10A5D80099CC1F267C0CC53E143E8C0F992887CE3B
:10A5E800A3E426C600C00000A3E4DA39992879312B
:10A5F800143E74F07C0C3BC199CCE1D98FC72B1E5B
:10A608002303EC3F203B7D186B2F06D56CEDC2C2AF
:10A61800B2C09CF672DC3635E720E536B13FBBF9AF
:10A628008F15BEC3BFD2BFD2BEC38F15BBF9B13F12
:10A63800E536E720363572DC9CF6B2C0C2C26CED56
:10A6480006D56B2F7D18203BEC3F23032B1E8FC7AD
:10A65800E1D999CC3BC17C0C74F0143E793199282E
:10A66800DA39A3E4000000C026C6A3E487CE9928FF
:10A678008C0F143EC53E7C0C1F2699CCD5E18FC7A4
:10A6880014C0230383E7203BFA2A6B2F3E3D6CED71
:10A698006409B2C0CACA72DC1BC9E7204506B13FCB
:10A6A800423C8F15412DBFD271EABEC34FC0BBF9E2
:10A6B80019DFE5368E2336354E3F9CF69412C2C21A
:10A6C80095D006D5E0C47D18DDFCEC3F71382B1E13
:10A6D8006733E1D984F33BC1ECC174F067D77931B2
:10A6E8005D1BDA39004000005D1B26C667D787CEA0
:10A6F800ECC18C0F84F3C53E67331F267138D5E152
:10A70800DDFC14C0E0C483E795D0FA2A94123E3DDC
:10A718004E3F64098E23CACA19DF1BC94FC04506BC
:10A7280071EA423C412D412D423C71EA45064FC039
:10A738001BC919DFCACA8E2364094E3F3E3D9412D5
:10A74800FA2A95D083E7E0C414C0DDFCD5E171385E
:10A758001F266733C53E84F38C0FECC187CE67D7BD
:10A7680026C65D1B00000040DA395D1B793167D7CA
:10A7780074F0ECC13BC184F3E1D967332B1E713807
:10A78800EC3FDDFC7D18E0C406D595D0C2C294121A
:10A798009CF64E3F36358E23E53619DFBBF94FC0A0
:10A7A800BEC371EABFD2412D8F15423CB13F450669
:10A7B800E7201BC972DCCACAB2C064096CED3E3D11
:10A7C8006B2FFA2A203B83E7230314C08FC7D5E1F8
:10A7D80099CC1F267C0CC53E143E8C0F992887CE39
:10A7E800A3E426C600C00000A3E4DA399928793129
:10A7F800143E74F07C0C3BC199CCE1D98FC72B1E59
:10A808002303EC3F203B7D186B2F06D56CEDC2C2AD
:10A81800B2C09CF672DC3635E720E536B13FBBF9AD
:10A828008F15BEC3BFD2BFD2BEC38F15BBF9B13F10
:10A83800E536E720363572DC9CF6B2C0C2C26CED54
:10A8480006D56B2F7D18203BEC3F23032B1E8FC7AB
:10A85800E1D999CC3BC17C0C74F0143E793199282C
:10A86800DA39A3E4000000C026C6A3E487CE9928FD
:10A878008C0F143EC53E7C0C1F2699CCD5E18FC7A2
:10A8880014C0230383E7203BFA2A6B2F3E3D6CED6F
:10A898006409B2C0CACA72DC1BC9E7204506B13FC9
:10A8A800423C8F15412DBFD271EABEC34FC0BBF9E0
:10A8B80019DFE5368E2336354E3F9CF69412C2C218
:10A8C80095D006D5E0C47D18DDFCEC3F71382B1E11
:10A8D8006733E1D984F33BC1ECC174F067D77931B0
:10A8E8005D1BDA39004000005D1B26C667D787CE9E
:10A8F800ECC18C0F84F3C53E67331F267138D5E150
:10A90800DDFC14C0E0C483E795D0FA2A94123E3DDA
:10A918004E3F64098E23CACA19DF1BC94FC04506BA
:10A9280071EA423C412D412D423C71EA45064FC037
:10A938001BC919DFCACA8E2364094E3F3E3D9412D3
:10A94800FA2A95D083E7E0C414C0DDFCD5E171385C
:10A958001F266733C53E84F38C0FECC187CE67D7BB
:10A9680026C65D1B0000004079319928C53E84F356
:10A978002B1E8FC783E7E0C4C2C26CEDCACA8E2300
:10A98800BBF9B13F412D412DB13FBBF98E23CACA56
:10A998006CEDC2C2E0C483E78FC72B1E84F3C53EAB
:10A9A8009928793100400000992887CE84F33BC16B
:10A9B8008FC7D5E1E0C47D186CED3E3D8E2336355A
:10A9C800B13F4506412DBFD2BBF94FC0CACA72DCA0
:10A9D800C2C2941283E7203B2B1E7138C53E7C0C03
:10A9E800793167D7000000C087CE67D73BC17C0CA0
:10A9F800D5E171387D18203B3E3D9412363572DC26
:10AA080045064FC0BFD2BFD24FC0450672DC3635AF
:10AA180094123E3D203B7D187138D5E17C0C3BC13A
:10AA280067D787CE00C0000067D779317C0CC53E58
:10AA380071382B1E203B83E79412C2C272DCCACA4B
:10AA48004FC0BBF9BFD2412D4506B13F36358E23E5
:10AA58003E3D6CED7D18E0C4D5E18FC73BC184F362
:10AA680087CE99280000004079319928C53E84F3A3
:10AA78002B1E8FC783E7E0C4C2C26CEDCACA8E23FF
:10AA8800BBF9B13F412D412DB13FBBF98E23CACA55
:10AA98006CEDC2C2E0C483E78FC72B1E84F3C53EAA
:10AAA8009928793100400000992887CE84F33BC16A
:10AAB8008FC7D5E1E0C47D186CED3E3D8E23363559
:10AAC800B13F4506412DBFD2BBF94FC0CACA72DC9F
:10AAD800C2C2941283E7203B2B1E7138C53E7C0C02
:10AAE800793167D7000000C087CE67D73BC17C0C9F
:10AAF800D5E171387D18203B3E3D9412363572DC25
:10AB080045064FC0BFD2BFD24FC0450672DC3635AE
:10AB180094123E3D203B7D187138D5E17C0C3BC139
:10AB280067D787CE00C0000067D779317C0CC53E57
:10AB380071382B1E203B83E79412C2C272DCCACA4A
:10AB48004FC0BBF9BFD2412D4506B13F36358E23E4
:10AB58003E3D6CED7D18E0C4D5E18FC73BC184F361
:10AB680087CE99280000004079319928C53E84F3A2
:10AB78002B1E8FC783E7E0C4C2C26CEDCACA8E23FE
:10AB8800BBF9B13F412D412DB13FBBF98E23CACA54
:10AB98006CEDC2C2E0C483E78FC72B1E84F3C53EA9
:10ABA8009928793100400000992887CE84F33BC169
:10ABB8008FC7D5E1E0C47D186CED3E3D8E23363558
:10ABC800B13F4506412DBFD2BBF94FC0CACA72DC9E
:10ABD800C2C2941283E7203B2B1E7138C53E7C0C01
:10ABE800793167D7000000C087CE67D73BC17C0C9E
:10ABF800D5E171387D18203B3E3D9412363572DC24
:10AC080045064FC0BFD2BFD24FC0450672DC3635AD
:10AC180094123E3D203B7D187138D5E17C0C3BC138
:10AC280067D787CE00C0000067D779317C0CC53E56
:10AC380071382B1E203B83E79412C2C272DCCACA49
:10AC48004FC0BBF9BFD2412D4506B13F36358E23E3
:10AC58003E3D6CED7D18E0C4D5E18FC73BC184F360
:10AC680087CE99280000004079319928C53E84F3A1
:10AC78002B1E8FC783E7E0C4C2C26CEDCACA8E23FD
:10AC8800BBF9B13F412D412DB13FBBF98E23CACA53
:10AC98006CEDC2C2E0C483E78FC72B1E84F3C53EA8
:10ACA8009928793100400000992887CE84F33BC168
:10ACB8008FC7D5E1E0C47D186CED3E3D8E23363557
:10ACC800B13F4506412DBFD2BBF94FC0CACA72DC9D
:10ACD800C2C2941283E7203B2B1E7138C53E7C0C00
:10ACE800793167D7000000C087CE67D73BC17C0C9D
:10ACF800D5E171387D18203B3E3D9412363572DC23
:10AD080045064FC0BFD2BFD24FC0450672DC3635AC
:10AD180094123E3D203B7D187138D5E17C0C3BC137
:10AD280067D787CE00C0000067D779317C0CC53E55
:10AD380071382B1E203B83E79412C2C272DCCACA48
:10AD48004FC0BBF9BFD2412D4506B13F36358E23E2
:10AD58003E3D6CED7D18E0C4D5E18FC73BC184F35F
:10AD680087CE99280000004079319928C53E84F3A0
:10AD78002B1E8FC783E7E0C4C2C26CEDCACA8E23FC
:10AD8800BBF9B13F412D412DB13FBBF98E23CACA52
:10AD98006CEDC2C2E0C483E78FC72B1E84F3C53EA7
:10ADA8009928793100400000992887CE84F33BC167
:10ADB8008FC7D5E1E0C47D186CED3E3D8E23363556
:10ADC800B13F4506412DBFD2BBF94FC0CACA72DC9C
:10ADD800C2C2941283E7203B2B1E7138C53E7C0CFF
:10ADE800793167D7000000C087CE67D73BC17C0C9C
:10ADF800D5E171387D18203B3E3D9412363572DC22
:10AE080045064FC0BFD2BFD24FC0450672DC3635AB
:10AE180094123E3D203B7D187138D5E17C0C3BC136
:10AE280067D787CE00C0000067D779317C0CC53E54
:10AE380071382B1E203B83E79412C2C272DCCACA47
:10AE48004FC0BBF9BFD2412D4506B13F36358E23E1
:10AE58003E3D6CED7D18E0C4D5E18FC73BC184F35E
:10AE680087CE99280000004079319928C53E84F39F
:10AE78002B1E8FC783E7E0C4C2C26CEDCACA8E23FB
:10AE8800BBF9B13F412D412DB13FBBF98E23CACA51
:10AE98006CEDC2C2E0C483E78FC72B1E84F3C53EA6
:10AEA8009928793100400000992887CE84F33BC166
:10AEB8008FC7D5E1E0C47D186CED3E3D8E23363555
:10AEC800B13F4506412DBFD2BBF94FC0CACA72DC9B
:10AED800C2C2941283E7203B2B1E7138C53E7C0CFE
:10AEE800793167D7000000C087CE67D73BC17C0C9B
:10AEF800D5E171387D18203B3E3D9412363572DC21
:10AF080045064FC0BFD2BFD24FC0450672DC3635AA
:10AF180094123E3D203B7D187138D5E17C0C3BC135
:10AF280067D787CE00C0000067D779317C0CC53E53
:10AF380071382B1E203B83E79412C2C272DCCACA46
:10AF48004FC0BBF9BFD2412D4506B13F36358E23E0
:10AF58003E3D6CED7D18E0C4D5E18FC73BC184F35D
:10AF680087CE99280000004079319928C53E84F39E
:10AF78002B1E8FC783E7E0C4C2C26CEDCACA8E23FA
:10AF8800BBF9B13F412D412DB13FBBF98E23CACA50
:10AF98006CEDC2C2E0C483E78FC72B1E84F3C53EA5
:10AFA8009928793100400000992887CE84F33BC165
:10AFB8008FC7D5E1E0C47D186CED3E3D8E23363554
:10AFC800B13F4506412DBFD2BBF94FC0CACA72DC9A
:10AFD800C2C2941283E7203B2B1E7138C53E7C0CFD
:10AFE800793167D7000000C087CE67D73BC17C0C9A
:10AFF800D5E171387D18203B3E3D9412363572DC20
:10B0080045064FC0BFD2BFD24FC0450672DC3635A9
:10B0180094123E3D203B7D187138D5E17C0C3BC134
:10B0280067D787CE00C0000067D779317C0CC53E52
:10B0380071382B1E203B83E79412C2C272DCCACA45
:10B048004FC0BBF9BFD2412D4506B13F36358E23DF
:10B058003E3D6CED7D18E0C4D5E18FC73BC184F35C
:10B0680087CE99280000004079319928C53E84F39D
:10B078002B1E8FC783E7E0C4C2C26CEDCACA8E23F9
:10B08800BBF9B13F412D412DB13FBBF98E23CACA4F
:10B098006CEDC2C2E0C483E78FC72B1E84F3C53EA4
:10B0A8009928793100400000992887CE84F33BC164
:10B0B8008FC7D5E1E0C47D186CED3E3D8E23363553
:10B0C800B13F4506412DBFD2BBF94FC0CACA72DC99
:10B0D800C2C2941283E7203B2B1E7138C53E7C0CFC
:10B0E800793167D7000000C087CE67D73BC17C0C99
:10B0F800D5E171387D18203B3E3D9412363572DC1F
:10B1080045064FC0BFD2BFD24FC0450672DC3635A8
:10B1180094123E3D203B7D187138D5E17C0C3BC133
:10B1280067D787CE00C0000067D779317C0CC53E51
:10B1380071382B1E203B83E79412C2C272DCCACA44
:10B148004FC0BBF9BFD2412D4506B13F36358E23DE
:10B158003E3D6CED7D18E0C4D5E18FC73BC184F35B
:10B1680087CE99280000004012363D22DA39A3E440
:10B17800D5077CC087CE67D73BC3131474F0143E41
:10B18800212C5A2EC53E84F308174AC4E1D999CC1C
:10B198002DC0B504D5E171388B1FAF37EC3F2303C1
:10B1A800DA24ADCB83E7E0C4F2C00FF506D56B2FE8
:10B1B8001111AE3D3E3D9412763033D69CF6B2C0A6
:10B1C8007EC511E6CACA8E239201FB3FE536E72009
:10B1D8002A393AE345064FC08CCDA1D8BEC38F1596
:10B1E800FBF1713E412D412D713EFBF18F15BEC320
:10B1F800A1D88CCD4FC045063AE32A39E720E53679
:10B20800FB3F92018E23CACA11E67EC5B2C09CF6E6
:10B2180033D6763094123E3DAE3D11116B2F06D5D4
:10B228000FF5F2C0E0C483E7ADCBDA242303EC3F8B
:10B23800AF378B1F7138D5E1B5042DC099CCE1D952
:10B248004AC4081784F3C53E5A2E212C143E74F0C4
:10B2580013143BC367D787CE7CC0D507A3E4DA397C
:10B268003D221236004000003D22EEC9A3E426C666
:10B278007CC02BF867D779311314C53C143E8C0F6A
:10B288005A2EDFD384F33BC14AC4F8E899CC1F2671
:10B29800B504D33F71382B1EAF3775E0230314C0B4
:10B2A800ADCB26DBE0C47D180FF50E3F6B2FFA2AD5
:10B2B800AE3DEFEE9412C2C233D68ACFB2C0640953
:10B2C80011E6823A8E233635FB3F6EFEE7201BC916
:10B2D8003AE3D6C64FC0BBF9A1D874328F15423CA9
:10B2E800713E050E412DBFD2FBF18FC1BEC371EA7D
:10B2F8008CCD5F274506B13F2A39C61CE53619DFD4
:10B30800920105C0CACA72DC7EC5EF199CF64E3F91
:10B318007630CD293E3D6CED111152C206D595D03F
:10B32800F2C0F10A83E7203BDA245334EC3FDDFC1A
:10B338008B1F51C8D5E18FC72DC04BFBE1D96733AF
:10B348000817B63BC53E7C0C212CA6D174F0ECC185
:10B358003BC3EDEB87CE9928D507843FDA395D1BCF
:10B368001236C3DD000000C0EEC9C3DD26C65D1B72
:10B378002BF8843F79319928C53CEDEB8C0FECC153
:10B38800DFD3A6D13BC17C0CF8E8B63B1F26673358
:10B39800D33F4BFB2B1E8FC775E051C814C0DDFC93
:10B3A80026DB53347D18203B0E3FF10AFA2A95D04C
:10B3B800EFEE52C2C2C26CED8ACFCD2964094E3F6E
:10B3C800823AEF19363572DC6EFE05C01BC919DFEB
:10B3D800D6C6C61CBBF9B13F74325F27423C71EA3E
:10B3E800050E8FC1BFD2BFD28FC1050E71EA423C94
:10B3F8005F277432B13FBBF9C61CD6C619DF1BC91B
:10B4080005C06EFE72DC3635EF19823A4E3F64098C
:10B41800CD298ACF6CEDC2C252C2EFEE95D0FA2A7E
:10B42800F10A0E3F203B7D18533426DBDDFC14C0A7
:10B4380051C875E08FC72B1E4BFBD33F67331F26C0
:10B44800B63BF8E87C0C3BC1A6D1DFD3ECC18C0F2E
:10B45800EDEBC53C99287931843F2BF85D1B26C656
:10B46800C3DDEEC900C00000C3DD12365D1BDA394A
:10B47800843FD507992887CEEDEB3BC3ECC174F028
:10B48800A6D1212C7C0CC53EB63B08176733E1D901
:10B498004BFB2DC08FC7D5E151C88B1FDDFCEC3F9E
:10B4A8005334DA24203B83E7F10AF2C095D006D55D
:10B4B80052C211116CED3E3DCD2976304E3F9CF6BF
:10B4C800EF197EC572DCCACA05C0920119DFE536DC
:10B4D800C61C2A39B13F45065F278CCD71EABEC329
:10B4E8008FC1FBF1BFD2412D050E713E423C8F1535
:10B4F8007432A1D8BBF94FC0D6C63AE31BC9E720BE
:10B508006EFEFB3F36358E23823A11E66409B2C0DF
:10B518008ACF33D6C2C29412EFEEAE3DFA2A6B2F11
:10B528000E3F0FF57D18E0C426DBADCB14C0230316
:10B5380075E0AF372B1E7138D33FB5041F2699CC61
:10B54800F8E84AC43BC184F3DFD35A2E8C0F143E6B
:10B55800C53C1314793167D72BF87CC026C6A3E401
:10B56800EEC93D220000004012363D22DA39A3E43C
:10B57800D5077CC087CE67D73BC3131474F0143E3D
:10B58800212C5A2EC53E84F308174AC4E1D999CC18
:10B598002DC0B504D5E171388B1FAF37EC3F2303BD
:10B5A800DA24ADCB83E7E0C4F2C00FF506D56B2FE4
:10B5B8001111AE3D3E3D9412763033D69CF6B2C0A2
:10B5C8007EC511E6CACA8E239201FB3FE536E72005
:10B5D8002A393AE345064FC08CCDA1D8BEC38F1592
:10B5E800FBF1713E412D412D713EFBF18F15BEC31C
:10B5F800A1D88CCD4FC045063AE32A39E720E53675
:10B60800FB3F92018E23CACA11E67EC5B2C09CF6E2
:10B6180033D6763094123E3DAE3D11116B2F06D5D0
:10B628000FF5F2C0E0C483E7ADCBDA242303EC3F87
:10B63800AF378B1F7138D5E1B5042DC099CCE1D94E
:10B648004AC4081784F3C53E5A2E212C143E74F0C0
:10B6580013143BC367D787CE7CC0D507A3E4DA3978
:10B668003D221236004000003D22EEC9A3E426C662
:10B678007CC02BF867D779311314C53C143E8C0F66
:10B688005A2EDFD384F33BC14AC4F8E899CC1F266D
:10B69800B504D33F71382B1EAF3775E0230314C0B0
:10B6A800ADCB26DBE0C47D180FF50E3F6B2FFA2AD1
:10B6B800AE3DEFEE9412C2C233D68ACFB2C064094F
:10B6C80011E6823A8E233635FB3F6EFEE7201BC912
:10B6D8003AE3D6C64FC0BBF9A1D874328F15423CA5
:10B6E800713E050E412DBFD2FBF18FC1BEC371EA79
:10B6F8008CCD5F274506B13F2A39C61CE53619DFD0
:10B70800920105C0CACA72DC7EC5EF199CF64E3F8D
:10B718007630CD293E3D6CED111152C206D595D03B
:10B72800F2C0F10A83E7203BDA245334EC3FDDFC16
:10B738008B1F51C8D5E18FC72DC04BFBE1D96733AB
:10B748000817B63BC53E7C0C212CA6D174F0ECC181
:10B758003BC3EDEB87CE9928D507843FDA395D1BCB
:10B768001236C3DD000000C0EEC9C3DD26C65D1B6E
:10B778002BF8843F79319928C53CEDEB8C0FECC14F
:10B78800DFD3A6D13BC17C0CF8E8B63B1F26673354
:10B79800D33F4BFB2B1E8FC775E051C814C0DDFC8F
:10B7A80026DB53347D18203B0E3FF10AFA2A95D048
:10B7B800EFEE52C2C2C26CED8ACFCD2964094E3F6A
:10B7C800823AEF19363572DC6EFE05C01BC919DFE7
:10B7D800D6C6C61CBBF9B13F74325F27423C71EA3A
:10B7E800050E8FC1BFD2BFD28FC1050E71EA423C90
:10B7F8005F277432B13FBBF9C61CD6C619DF1BC917
:10B8080005C06EFE72DC3635EF19823A4E3F640988
:10B81800CD298ACF6CEDC2C252C2EFEE95D0FA2A7A
:10B82800F10A0E3F203B7D18533426DBDDFC14C0A3
:10B8380051C875E08FC72B1E4BFBD33F67331F26BC
:10B84800B63BF8E87C0C3BC1A6D1DFD3ECC18C0F2A
:10B85800EDEBC53C99287931843F2BF85D1B26C652
:10B86800C3DDEEC900C00000C3DD12365D1BDA3946
:10B87800843FD507992887CEEDEB3BC3ECC174F024
:10B88800A6D1212C7C0CC53EB63B08176733E1D9FD
:10B898004BFB2DC08FC7D5E151C88B1FDDFCEC3F9A
:10B8A8005334DA24203B83E7F10AF2C095D006D559
:10B8B80052C211116CED3E3DCD2976304E3F9CF6BB
:10B8C800EF197EC572DCCACA05C0920119DFE536D8
:10B8D800C61C2A39B13F45065F278CCD71EABEC325
:10B8E8008FC1FBF1BFD2412D050E713E423C8F1531
:10B8F8007432A1D8BBF94FC0D6C63AE31BC9E720BA
:10B908006EFEFB3F36358E23823A11E66409B2C0DB
:10B918008ACF33D6C2C29412EFEEAE3DFA2A6B2F0D
:10B928000E3F0FF57D18E0C426DBADCB14C0230312
:10B9380075E0AF372B1E7138D33FB5041F2699CC5D
:10B94800F8E84AC43BC184F3DFD35A2E8C0F143E67
:10B95800C53C1314793167D72BF87CC026C6A3E4FD
:10B96800EEC93D220000004000400000000000C079
:10B9780000C000000000004000400000000000C0BF
:10B9880000C000000000004000400000000000C0AF
:10B9980000C000000000004000400000000000C09F
:10B9A80000C000000000004000400000000000C08F
:10B9B80000C000000000004000400000000000C07F
:10B9C80000C000000000004000400000000000C06F
:10B9D80000C000000000004000400000000000C05F
:10B9E80000C000000000004000400000000000C04F
:10B9F80000C000000000004000400000000000C03F
:10BA080000C000000000004000400000000000C02E
:10BA180000C000000000004000400000000000C01E
:10BA280000C000000000004000400000000000C00E
:10BA380000C000000000004000400000000000C0FE
:10BA480000C000000000004000400000000000C0EE
:10BA580000C000000000004000400000000000C0DE
:10BA680000C000000000004000400000000000C0CE
:10BA780000C000000000004000400000000000C0BE
:10BA880000C000000000004000400000000000C0AE
:10BA980000C000000000004000400000000000C09E
:10BAA80000C000000000004000400000000000C08E
:10BAB80000C000000000004000400000000000C07E
:10BAC80000C000000000004000400000000000C06E
:10BAD80000C000000000004000400000000000C05E
:10BAE80000C000000000004000400000000000C04E
:10BAF80000C000000000004000400000000000C03E
:10BB080000C000000000004000400000000000C02D
:10BB180000C000000000004000400000000000C01D
:10BB280000C000000000004000400000000000C00D
:10BB380000C000000000004000400000000000C0FD
:10BB480000C000000000004000400000000000C0ED
:10BB580000C000000000004000400000000000C0DD
:10BB680000C000000000004000400000000000C0CD
:10BB780000C000000000004000400000000000C0BD
:10BB880000C000000000004000400000000000C0AD
:10BB980000C000000000004000400000000000C09D
:10BBA80000C000000000004000400000000000C08D
:10BBB80000C000000000004000400000000000C07D
:10BBC80000C000000000004000400000000000C06D
:10BBD80000C000000000004000400000000000C05D
:10BBE80000C000000000004000400000000000C04D
:10BBF80000C000000000004000400000000000C03D
:10BC080000C000000000004000400000000000C02C
:10BC180000C000000000004000400000000000C01C
:10BC280000C000000000004000400000000000C00C
:10BC380000C000000000004000400000000000C0FC
:10BC480000C000000000004000400000000000C0EC
:10BC580000C000000000004000400000000000C0DC
:10BC680000C000000000004000400000000000C0CC
:10BC780000C000000000004000400000000000C0BC
:10BC880000C000000000004000400000000000C0AC
:10BC980000C000000000004000400000000000C09C
:10BCA80000C000000000004000400000000000C08C
:10BCB80000C000000000004000400000000000C07C
:10BCC80000C000000000004000400000000000C06C
:10BCD80000C000000000004000400000000000C05C
:10BCE80000C000000000004000400000000000C04C
:10BCF80000C000000000004000400000000000C03C
:10BD080000C000000000004000400000000000C02B
:10BD180000C000000000004000400000000000C01B
:10BD280000C000000000004000400000000000C00B
:10BD380000C000000000004000400000000000C0FB
:10BD480000C000000000004000400000000000C0EB
:10BD580000C000000000004000400000000000C0DB
:10BD680000C000000000004000400000000000C0CB
:10BD780000C000000000004000400000000000C0BB
:10BD880000C000000000004000400000000000C0AB
:10BD980000C000000000004000400000000000C09B
:10BDA80000C000000000004000400000000000C08B
:10BDB80000C000000000004000400000000000C07B
:10BDC80000C000000000004000400000000000C06B
:10BDD80000C000000000004000400000000000C05B
:10BDE80000C000000000004000400000000000C04B
:10BDF80000C000000000004000400000000000C03B
:10BE080000C000000000004000400000000000C02A
:10BE180000C000000000004000400000000000C01A
:10BE280000C000000000004000400000000000C00A
:10BE380000C000000000004000400000000000C0FA
:10BE480000C000000000004000400000000000C0EA
:10BE580000C000000000004000400000000000C0DA
:10BE680000C000000000004000400000000000C0CA
:10BE780000C000000000004000400000000000C0BA
:10BE880000C000000000004000400000000000C0AA
:10BE980000C000000000004000400000000000C09A
:10BEA80000C000000000004000400000000000C08A
:10BEB80000C000000000004000400000000000C07A
:10BEC80000C000000000004000400000000000C06A
:10BED80000C000000000004000400000000000C05A
:10BEE80000C000000000004000400000000000C04A
:10BEF80000C000000000004000400000000000C03A
:10BF080000C000000000004000400000000000C029
:10BF180000C000000000004000400000000000C019
:10BF280000C000000000004000400000000000C009
:10BF380000C000000000004000400000000000C0F9
:10BF480000C000000000004000400000000000C0E9
:10BF580000C000000000004000400000000000C0D9
:10BF680000C000000000004000400000000000C0C9
:10BF780000C000000000004000400000000000C0B9
:10BF880000C000000000004000400000000000C0A9
:10BF980000C000000000004000400000000000C099
:10BFA80000C000000000004000400000000000C089
:10BFB80000C000000000004000400000000000C079
:10BFC80000C000000000004000400000000000C069
:10BFD80000C000000000004000400000000000C059
:10BFE80000C000000000004000400000000000C049
:10BFF80000C000000000004000400000000000C039
:10C0080000C000000000004000400000000000C028
:10C0180000C000000000004000400000000000C018
:10C0280000C000000000004000400000000000C008
:10C0380000C000000000004000400000000000C0F8
:10C0480000C000000000004000400000000000C0E8
:10C0580000C000000000004000400000000000C0D8
:10C0680000C000000000004000400000000000C0C8
:10C0780000C000000000004000400000000000C0B8
:10C0880000C000000000004000400000000000C0A8
:10C0980000C000000000004000400000000000C098
:10C0A80000C000000000004000400000000000C088
:10C0B80000C000000000004000400000000000C078
:10C0C80000C000000000004000400000000000C068
:10C0D80000C000000000004000400000000000C058
:10C0E80000C000000000004000400000000000C048
:10C0F80000C000000000004000400000000000C038
:10C1080000C000000000004000400000000000C027
:10C1180000C000000000004000400000000000C017
:10C1280000C000000000004000400000000000C007
:10C1380000C000000000004000400000000000C0F7
:10C1480000C000000000004000400000000000C0E7
:10C1580000C000000000004000400000000000C0D7
:10C1680000C0000000000040C53C13141F2699CCF5
:10C1780026DBADCBC2C294126EFEFB3F423C8F154C
:10C188005F278CCD72DCCACA52C21111DDFCEC3FAC
:10C19800B63B0817992887CEC3DDEEC9ECC18C0FD2
:10C1A8004BFBD33F203B7D18CD298ACF19DF1BC914
:10C1B8008FC1050EBBF9B13F823AEF19FA2A95D023
:10C1C80075E051C83BC17C0C2BF8843FDA395D1B04
:10C1D800212CA6D1D5E18FC7F2C0F10A9CF64E3FBB
:10C1E8002A39C61C412DBFD23AE3D6C6B2C064096B
:10C1F8000FF50E3F71382B1E5A2EDFD3A3E426C647
:10C208007CC0D50784F3C53EAF378B1F6B2F06D58F
:10C2180011E67EC54FC04506FBF1713EE536E720C5
:10C22800763033D683E7E0C42DC0B50474F0143EED
:10C2380012363D22793167D7F8E84AC414C023037F
:10C24800EFEEAE3D36358E237432A1D871EABEC307
:10C2580005C092016CED3E3D5334DA246733E1D9D1
:10C26800EDEB3BC300C00000EDEBC53C67331F2678
:10C27800533426DB6CEDC2C205C06EFE71EA423C47
:10C2880074325F27363572DCEFEE52C214C0DDFC23
:10C29800F8E8B63B793199281236C3DD74F0ECC161
:10C2A8002DC04BFB83E7203B7630CD29E53619DFDF
:10C2B800FBF18FC14FC0BBF911E6823A6B2FFA2A06
:10C2C800AF3775E084F33BC17CC02BF8A3E4DA39BF
:10C2D8005A2E212C7138D5E10FF5F2C0B2C09CF668
:10C2E8003AE32A39412D412D2A393AE39CF6B2C066
:10C2F800F2C00FF5D5E17138212C5A2EDA39A3E4B2
:10C308002BF87CC03BC184F375E0AF37FA2A6B2F5A
:10C31800823A11E6BBF94FC08FC1FBF119DFE53650
:10C32800CD297630203B83E74BFB2DC0ECC174F060
:10C33800C3DD123699287931B63BF8E8DDFC14C024
:10C3480052C2EFEE72DC36355F277432423C71EA36
:10C358006EFE05C0C2C26CED26DB53341F26673360
:10C36800C53CEDEB000000C03BC3EDEBE1D9673302
:10C37800DA2453343E3D6CED920105C0BEC371EA28
:10C38800A1D874328E233635AE3DEFEE230314C0A8
:10C398004AC4F8E867D779313D221236143E74F062
:10C3A800B5042DC0E0C483E733D67630E720E53600
:10C3B800713EFBF145064FC07EC511E606D56B2FD1
:10C3C8008B1FAF37C53E84F3D5077CC026C6A3E4D0
:10C3D800DFD35A2E2B1E71380E3F0FF56409B2C0F9
:10C3E800D6C63AE3BFD2412DC61C2A394E3F9CF629
:10C3F800F10AF2C08FC7D5E1A6D1212C5D1BDA392D
:10C40800843F2BF87C0C3BC151C875E095D0FA2AC3
:10C41800EF19823AB13FBBF9050E8FC11BC919DF6D
:10C428008ACFCD297D18203BD33F4BFB8C0FECC125
:10C43800EEC9C3DD87CE99280817B63BEC3FDDFC73
:10C44800111152C2CACA72DC8CCD5F278F15423CCB
:10C45800FB3F6EFE9412C2C2ADCB26DB99CC1F26E1
:10C468001314C53C0040000013143BC399CCE1D918
:10C47800ADCBDA2494123E3DFB3F92018F15BEC32B
:10C488008CCDA1D8CACA8E231111AE3DEC3F23032F
:10C4980008174AC487CE67D7EEC93D228C0F143ED1
:10C4A800D33FB5047D18E0C48ACF33D61BC9E72033
:10C4B800050E713EB13F4506EF197EC595D006D5EC
:10C4C80051C88B1F7C0CC53E843FD5075D1B26C613
:10C4D800A6D1DFD38FC72B1EF10A0E3F4E3F64094A
:10C4E800C61CD6C6BFD2BFD2D6C6C61C64094E3F2C
:10C4F8000E3FF10A2B1E8FC7DFD3A6D126C65D1BC0
:10C50800D507843FC53E7C0C8B1F51C806D595D0F6
:10C518007EC5EF194506B13F713E050EE7201BC9E0
:10C5280033D68ACFE0C47D18B504D33F143E8C0FB0
:10C538003D22EEC967D787CE4AC408172303EC3FCC
:10C54800AE3D11118E23CACAA1D88CCDBEC38F159A
:10C558009201FB3F3E3D9412DA24ADCBE1D999CC50
:10C568003BC3131400000040C53C13141F2699CC8C
:10C5780026DBADCBC2C294126EFEFB3F423C8F1548
:10C588005F278CCD72DCCACA52C21111DDFCEC3FA8
:10C59800B63B0817992887CEC3DDEEC9ECC18C0FCE
:10C5A8004BFBD33F203B7D18CD298ACF19DF1BC910
:10C5B8008FC1050EBBF9B13F823AEF19FA2A95D01F
:10C5C80075E051C83BC17C0C2BF8843FDA395D1B00
:10C5D800212CA6D1D5E18FC7F2C0F10A9CF64E3FB7
:10C5E8002A39C61C412DBFD23AE3D6C6B2C0640967
:10C5F8000FF50E3F71382B1E5A2EDFD3A3E426C643
:10C608007CC0D50784F3C53EAF378B1F6B2F06D58B
:10C6180011E67EC54FC04506FBF1713EE536E720C1
:10C62800763033D683E7E0C42DC0B50474F0143EE9
:10C6380012363D22793167D7F8E84AC414C023037B
:10C64800EFEEAE3D36358E237432A1D871EABEC303
:10C6580005C092016CED3E3D5334DA246733E1D9CD
:10C66800EDEB3BC300C00000EDEBC53C67331F2674
:10C67800533426DB6CEDC2C205C06EFE71EA423C43
:10C6880074325F27363572DCEFEE52C214C0DDFC1F
:10C69800F8E8B63B793199281236C3DD74F0ECC15D
:10C6A8002DC04BFB83E7203B7630CD29E53619DFDB
:10C6B800FBF18FC14FC0BBF911E6823A6B2FFA2A02
:10C6C800AF3775E084F33BC17CC02BF8A3E4DA39BB
:10C6D8005A2E212C7138D5E10FF5F2C0B2C09CF664
:10C6E8003AE32A39412D412D2A393AE39CF6B2C062
:10C6F800F2C00FF5D5E17138212C5A2EDA39A3E4AE
:10C708002BF87CC03BC184F375E0AF37FA2A6B2F56
:10C71800823A11E6BBF94FC08FC1FBF119DFE5364C
:10C72800CD297630203B83E74BFB2DC0ECC174F05C
:10C73800C3DD123699287931B63BF8E8DDFC14C020
:10C7480052C2EFEE72DC36355F277432423C71EA32
:10C758006EFE05C0C2C26CED26DB53341F2667335C
:10C76800C53CEDEB000000C03BC3EDEBE1D96733FE
:10C77800DA2453343E3D6CED920105C0BEC371EA24
:10C78800A1D874328E233635AE3DEFEE230314C0A4
:10C798004AC4F8E867D779313D221236143E74F05E
:10C7A800B5042DC0E0C483E733D67630E720E536FC
:10C7B800713EFBF145064FC07EC511E606D56B2FCD
:10C7C8008B1FAF37C53E84F3D5077CC026C6A3E4CC
:10C7D800DFD35A2E2B1E71380E3F0FF56409B2C0F5
:10C7E800D6C63AE3BFD2412DC61C2A394E3F9CF625
:10C7F800F10AF2C08FC7D5E1A6D1212C5D1BDA3929
:10C80800843F2BF87C0C3BC151C875E095D0FA2ABF
:10C81800EF19823AB13FBBF9050E8FC11BC919DF69
:10C828008ACFCD297D18203BD33F4BFB8C0FECC121
:10C83800EEC9C3DD87CE99280817B63BEC3FDDFC6F
:10C84800111152C2CACA72DC8CCD5F278F15423CC7
:10C85800FB3F6EFE9412C2C2ADCB26DB99CC1F26DD
:10C868001314C53C0040000013143BC399CCE1D914
:10C87800ADCBDA2494123E3DFB3F92018F15BEC327
:10C888008CCDA1D8CACA8E231111AE3DEC3F23032B
:10C8980008174AC487CE67D7EEC93D228C0F143ECD
:10C8A800D33FB5047D18E0C48ACF33D61BC9E7202F
:10C8B800050E713EB13F4506EF197EC595D006D5E8
:10C8C80051C88B1F7C0CC53E843FD5075D1B26C60F
:10C8D800A6D1DFD38FC72B1EF10A0E3F4E3F640946
:10C8E800C61CD6C6BFD2BFD2D6C6C61C64094E3F28
:10C8F8000E3FF10A2B1E8FC7DFD3A6D126C65D1BBC
:10C90800D507843FC53E7C0C8B1F51C806D595D0F2
:10C918007EC5EF194506B13F713E050EE7201BC9DC
:10C9280033D68ACFE0C47D18B504D33F143E8C0FAC
:10C938003D22EEC967D787CE4AC408172303EC3FC8
:10C94800AE3D11118E23CACAA1D88CCDBEC38F1596
:10C958009201FB3F3E3D9412DA24ADCBE1D999CC4C
:10C968003BC3131400000040D33FB5046409B2C0B0
:10C978008FC1FBF16CED3E3DB63B08175D1B26C62B
:10C9880051C875E072DC363574325F27FA2A95D0C3
:10C99800DFD3A6D187CE9928DA245334E53619DFB8
:10C9A8003AE3D6C6E0C47D181314C53C143E74F0AF
:10C9B8000FF5F2C04FC045069201FB3FEC3F230341
:10C9C800D5077CC03BC184F3EFEEAE3D423C8F15EA
:10C9D800EF197EC58FC7D5E1C3DD123667331F2631
:10C9E800CD298ACFBFD2BFD28ACFCD291F266733A0
:10C9F8001236C3DDD5E18FC77EC5EF198F15423CCE
:10CA0800AE3DEFEE84F33BC17CC0D5072303EC3F7A
:10CA1800FB3F920145064FC0F2C00FF574F0143E7B
:10CA2800C53C13147D18E0C4D6C63AE319DFE536D1
:10CA38005334DA24992887CEA6D1DFD395D0FA2AA1
:10CA48005F277432363572DC75E051C826C65D1B27
:10CA58000817B63B3E3D6CEDFBF18FC1B2C06409CF
:10CA6800B504D33F00400000B5042DC0B2C09CF609
:10CA7800FBF1713E3E3D941208174AC426C6A3E452
:10CA880075E0AF3736358E235F278CCD95D006D528
:10CA9800A6D1212C99287931533426DB19DF1BC9FB
:10CAA800D6C6C61C7D18203BC53CEDEB74F0ECC126
:10CAB800F2C0F10A4506B13FFB3F6EFE230314C0E6
:10CAC8007CC02BF884F3C53EAE3D11118F15BEC353
:10CAD8007EC511E6D5E1713812363D221F2699CC64
:10CAE8008ACF33D6BFD2412DCD2976306733E1D9ED
:10CAF800C3DDEEC98FC72B1EEF19823A423C71EA9B
:10CB0800EFEE52C23BC17C0CD507843FEC3FDDFC05
:10CB1800920105C04FC0BBF90FF50E3F143E8C0FB4
:10CB280013143BC3E0C483E73AE32A39E536E72028
:10CB3800DA24ADCB87CE67D7DFD35A2EFA2A6B2FEC
:10CB48007432A1D872DCCACA51C88B1F5D1BDA398E
:10CB5800B63BF8E86CEDC2C28FC1050E64094E3FC2
:10CB6800D33F4BFB000000C02DC04BFB9CF64E3F53
:10CB7800713E050E9412C2C24AC4F8E8A3E4DA3939
:10CB8800AF378B1F8E23CACA8CCDA1D806D56B2F81
:10CB9800212C5A2E793167D726DBADCB1BC9E7206C
:10CBA800C61C2A39203B83E7EDEB3BC3ECC18C0F55
:10CBB800F10A0E3FB13FBBF96EFE05C014C0DDFCA3
:10CBC8002BF8843FC53E7C0C111152C2BEC371EADA
:10CBD80011E6823A71382B1E3D22EEC999CCE1D973
:10CBE80033D67630412D412D763033D6E1D999CCE4
:10CBF800EEC93D222B1E7138823A11E671EABEC396
:10CC080052C211117C0CC53E843F2BF8DDFC14C0C8
:10CC180005C06EFEBBF9B13F0E3FF10A8C0FECC1A7
:10CC28003BC3EDEB83E7203B2A39C61CE7201BC931
:10CC3800ADCB26DB67D779315A2E212C6B2F06D541
:10CC4800A1D88CCDCACA8E238B1FAF37DA39A3E49B
:10CC5800F8E84AC4C2C29412050E713E4E3F9CF6D3
:10CC68004BFB2DC000C000004BFBD33F4E3F640977
:10CC7800050E8FC1C2C26CEDF8E8B63BDA395D1B10
:10CC88008B1F51C8CACA72DCA1D874326B2FFA2A1A
:10CC98005A2EDFD367D787CEADCBDA24E720E53627
:10CCA8002A393AE383E7E0C43BC313148C0F143EDC
:10CCB8000E3F0FF5BBF94FC005C09201DDFCEC3FFC
:10CCC800843FD5077C0C3BC152C2EFEE71EA423C6F
:10CCD800823AEF192B1E8FC7EEC9C3DDE1D967333E
:10CCE8007630CD29412DBFD233D68ACF99CC1F2695
:10CCF8003D2212367138D5E111E67EC5BEC38F15C7
:10CD08001111AE3DC53E84F32BF87CC014C023033B
:10CD18006EFEFB3FB13F4506F10AF2C0ECC174F06C
:10CD2800EDEBC53C203B7D18C61CD6C61BC919DFD8
:10CD380026DB533479319928212CA6D106D595D0F4
:10CD48008CCD5F278E233635AF3775E0A3E426C632
:10CD58004AC4081794123E3D713EFBF19CF6B2C0DE
:10CD68002DC0B50400000040D33FB5046409B2C02B
:10CD78008FC1FBF16CED3E3DB63B08175D1B26C627
:10CD880051C875E072DC363574325F27FA2A95D0BF
:10CD9800DFD3A6D187CE9928DA245334E53619DFB4
:10CDA8003AE3D6C6E0C47D181314C53C143E74F0AB
:10CDB8000FF5F2C04FC045069201FB3FEC3F23033D
:10CDC800D5077CC03BC184F3EFEEAE3D423C8F15E6
:10CDD800EF197EC58FC7D5E1C3DD123667331F262D
:10CDE800CD298ACFBFD2BFD28ACFCD291F2667339C
:10CDF8001236C3DDD5E18FC77EC5EF198F15423CCA
:10CE0800AE3DEFEE84F33BC17CC0D5072303EC3F76
:10CE1800FB3F920145064FC0F2C00FF574F0143E77
:10CE2800C53C13147D18E0C4D6C63AE319DFE536CD
:10CE38005334DA24992887CEA6D1DFD395D0FA2A9D
:10CE48005F277432363572DC75E051C826C65D1B23
:10CE58000817B63B3E3D6CEDFBF18FC1B2C06409CB
:10CE6800B504D33F00400000B5042DC0B2C09CF605
:10CE7800FBF1713E3E3D941208174AC426C6A3E44E
:10CE880075E0AF3736358E235F278CCD95D006D524
:10CE9800A6D1212C99287931533426DB19DF1BC9F7
:10CEA800D6C6C61C7D18203BC53CEDEB74F0ECC122
:10CEB800F2C0F10A4506B13FFB3F6EFE230314C0E2
:10CEC8007CC02BF884F3C53EAE3D11118F15BEC34F
:10CED8007EC511E6D5E1713812363D221F2699CC60
:10CEE8008ACF33D6BFD2412DCD2976306733E1D9E9
:10CEF800C3DDEEC98FC72B1EEF19823A423C71EA97
:10CF0800EFEE52C23BC17C0CD507843FEC3FDDFC01
:10CF1800920105C04FC0BBF90FF50E3F143E8C0FB0
:10CF280013143BC3E0C483E73AE32A39E536E72024
:10CF3800DA24ADCB87CE67D7DFD35A2EFA2A6B2FE8
:10CF48007432A1D872DCCACA51C88B1F5D1BDA398A
:10CF5800B63BF8E86CEDC2C28FC1050E64094E3FBE
:10CF6800D33F4BFB000000C02DC04BFB9CF64E3F4F
:10CF7800713E050E9412C2C24AC4F8E8A3E4DA3935
:10CF8800AF378B1F8E23CACA8CCDA1D806D56B2F7D
:10CF9800212C5A2E793167D726DBADCB1BC9E72068
:10CFA800C61C2A39203B83E7EDEB3BC3ECC18C0F51
:10CFB800F10A0E3FB13FBBF96EFE05C014C0DDFC9F
:10CFC8002BF8843FC53E7C0C111152C2BEC371EAD6
:10CFD80011E6823A71382B1E3D22EEC999CCE1D96F
:10CFE80033D67630412D412D763033D6E1D999CCE0
:10CFF800EEC93D222B1E7138823A11E671EABEC392
:10D0080052C211117C0CC53E843F2BF8DDFC14C0C4
:10D0180005C06EFEBBF9B13F0E3FF10A8C0FECC1A3
:10D028003BC3EDEB83E7203B2A39C61CE7201BC92D
:10D03800ADCB26DB67D779315A2E212C6B2F06D53D
:10D04800A1D88CCDCACA8E238B1FAF37DA39A3E497
:10D05800F8E84AC4C2C29412050E713E4E3F9CF6CF
:10D068004BFB2DC000C000004BFBD33F4E3F640973
:10D07800050E8FC1C2C26CEDF8E8B63BDA395D1B0C
:10D088008B1F51C8CACA72DCA1D874326B2FFA2A16
:10D098005A2EDFD367D787CEADCBDA24E720E53623
:10D0A8002A393AE383E7E0C43BC313148C0F143ED8
:10D0B8000E3F0FF5BBF94FC005C09201DDFCEC3FF8
:10D0C800843FD5077C0C3BC152C2EFEE71EA423C6B
:10D0D800823AEF192B1E8FC7EEC9C3DDE1D967333A
:10D0E8007630CD29412DBFD233D68ACF99CC1F2691
:10D0F8003D2212367138D5E111E67EC5BEC38F15C3
:10D108001111AE3DC53E84F32BF87CC014C0230337
:10D118006EFEFB3FB13F4506F10AF2C0ECC174F068
:10D12800EDEBC53C203B7D18C61CD6C61BC919DFD4
:10D1380026DB533479319928212CA6D106D595D0F0
:10D148008CCD5F278E233635AF3775E0A3E426C62E
:10D158004AC4081794123E3D713EFBF19CF6B2C0DA
:10D168002DC0B50400000040C53E7C0C7D18E0C40D
:10D17800CACA72DCBFD2412D8E233635203B83E7E5
:10D1880084F33BC100C0000084F3C53E203B7D18FA
:10D198008E23CACABFD2BFD2CACA8E237D18203BEB
:10D1A800C53E84F3000000C03BC184F383E7203B05
:10D1B80036358E23412DBFD272DCCACAE0C47D1831
:10D1C8007C0CC53E004000007C0C3BC1E0C483E7FA
:10D1D80072DC3635412D412D363572DC83E7E0C4EB
:10D1E8003BC17C0C00000040C53E7C0C7D18E0C4AF
:10D1F800CACA72DCBFD2412D8E233635203B83E765
:10D2080084F33BC100C0000084F3C53E203B7D1879
:10D218008E23CACABFD2BFD2CACA8E237D18203B6A
:10D22800C53E84F3000000C03BC184F383E7203B84
:10D2380036358E23412DBFD272DCCACAE0C47D18B0
:10D248007C0CC53E004000007C0C3BC1E0C483E779
:10D2580072DC3635412D412D363572DC83E7E0C46A
:10D268003BC17C0C00000040C53E7C0C7D18E0C42E
:10D27800CACA72DCBFD2412D8E233635203B83E7E4
:10D2880084F33BC100C0000084F3C53E203B7D18F9
:10D298008E23CACABFD2BFD2CACA8E237D18203BEA
:10D2A800C53E84F3000000C03BC184F383E7203B04
:10D2B80036358E23412DBFD272DCCACAE0C47D1830
:10D2C8007C0CC53E004000007C0C3BC1E0C483E7F9
:10D2D80072DC3635412D412D363572DC83E7E0C4EA
:10D2E8003BC17C0C00000040C53E7C0C7D18E0C4AE
:10D2F800CACA72DCBFD2412D8E233635203B83E764
:10D3080084F33BC100C0000084F3C53E203B7D1878
:10D318008E23CACABFD2BFD2CACA8E237D18203B69
:10D32800C53E84F3000000C03BC184F383E7203B83
:10D3380036358E23412DBFD272DCCACAE0C47D18AF
:10D348007C0CC53E004000007C0C3BC1E0C483E778
:10D3580072DC3635412D412D363572DC83E7E0C469
:10D368003BC17C0C00000040C53E7C0C7D18E0C42D
:10D37800CACA72DCBFD2412D8E233635203B83E7E3
:10D3880084F33BC100C0000084F3C53E203B7D18F8
:10D398008E23CACABFD2BFD2CACA8E237D18203BE9
:10D3A800C53E84F3000000C03BC184F383E7203B03
:10D3B80036358E23412DBFD272DCCACAE0C47D182F
:10D3C8007C0CC53E004000007C0C3BC1E0C483E7F8
:10D3D80072DC3635412D412D363572DC83E7E0C4E9
:10D3E8003BC17C0C00000040C53E7C0C7D18E0C4AD
:10D3F800CACA72DCBFD2412D8E233635203B83E763
:10D4080084F33BC100C0000084F3C53E203B7D1877
:10D418008E23CACABFD2BFD2CACA8E237D18203B68
:10D42800C53E84F3000000C03BC184F383E7203B82
:10D4380036358E23412DBFD272DCCACAE0C47D18AE
:10D448007C0CC53E004000007C0C3BC1E0C483E777
:10D4580072DC3635412D412D363572DC83E7E0C468
:10D468003BC17C0C00000040C53E7C0C7D18E0C42C
:10D47800CACA72DCBFD2412D8E233635203B83E7E2
:10D4880084F33BC100C0000084F3C53E203B7D18F7
:10D498008E23CACABFD2BFD2CACA8E237D18203BE8
:10D4A800C53E84F3000000C03BC184F383E7203B02
:10D4B80036358E23412DBFD272DCCACAE0C47D182E
:10D4C8007C0CC53E004000007C0C3BC1E0C483E7F7
:10D4D80072DC3635412D412D363572DC83E7E0C4E8
:10D4E8003BC17C0C00000040C53E7C0C7D18E0C4AC
:10D4F800CACA72DCBFD2412D8E233635203B83E762
:10D5080084F33BC100C0000084F3C53E203B7D1876
:10D518008E23CACABFD2BFD2CACA8E237D18203B67
:10D52800C53E84F3000000C03BC184F383E7203B81
:10D5380036358E23412DBFD272DCCACAE0C47D18AD
:10D548007C0CC53E004000007C0C3BC1E0C483E776
:10D5580072DC3635412D412D363572DC83E7E0C467
:10D568003BC17C0C00000040C53E7C0C7D18E0C42B
:10D57800CACA72DCBFD2412D8E233635203B83E7E1
:10D5880084F33BC100C0000084F3C53E203B7D18F6
:10D598008E23CACABFD2BFD2CACA8E237D18203BE7
:10D5A800C53E84F3000000C03BC184F383E7203B01
:10D5B80036358E23412DBFD272DCCACAE0C47D182D
:10D5C8007C0CC53E004000007C0C3BC1E0C483E7F6
:10D5D80072DC3635412D412D363572DC83E7E0C4E7
:10D5E8003BC17C0C00000040C53E7C0C7D18E0C4AB
:10D5F800CACA72DCBFD2412D8E233635203B83E761
:10D6080084F33BC100C0000084F3C53E203B7D1875
:10D618008E23CACABFD2BFD2CACA8E237D18203B66
:10D62800C53E84F3000000C03BC184F383E7203B80
:10D6380036358E23412DBFD272DCCACAE0C47D18AC
:10D648007C0CC53E004000007C0C3BC1E0C483E775
:10D6580072DC3635412D412D363572DC83E7E0C466
:10D668003BC17C0C00000040C53E7C0C7D18E0C42A
:10D67800CACA72DCBFD2412D8E233635203B83E7E0
:10D6880084F33BC100C0000084F3C53E203B7D18F5
:10D698008E23CACABFD2BFD2CACA8E237D18203BE6
:10D6A800C53E84F3000000C03BC184F383E7203B00
:10D6B80036358E23412DBFD272DCCACAE0C47D182C
:10D6C8007C0CC53E004000007C0C3BC1E0C483E7F5
:10D6D80072DC3635412D412D363572DC83E7E0C4E6
:10D6E8003BC17C0C00000040C53E7C0C7D18E0C4AA
:10D6F800CACA72DCBFD2412D8E233635203B83E760
:10D7080084F33BC100C0000084F3C53E203B7D1874
:10D718008E23CACABFD2BFD2CACA8E237D18203B65
:10D72800C53E84F3000000C03BC184F383E7203B7F
:10D7380036358E23412DBFD272DCCACAE0C47D18AB
:10D748007C0CC53E004000007C0C3BC1E0C483E774
:10D7580072DC3635412D412D363572DC83E7E0C465
:10D768003BC17C0C00000040C53E7C0C7D18E0C429
:10D77800CACA72DCBFD2412D8E233635203B83E7DF
:10D7880084F33BC100C0000084F3C53E203B7D18F4
:10D798008E23CACABFD2BFD2CACA8E237D18203BE5
:10D7A800C53E84F3000000C03BC184F383E7203BFF
:10D7B80036358E23412DBFD272DCCACAE0C47D182B
:10D7C8007C0CC53E004000007C0C3BC1E0C483E7F4
:10D7D80072DC3635412D412D363572DC83E7E0C4E5
:10D7E8003BC17C0C00000040C53E7C0C7D18E0C4A9
:10D7F800CACA72DCBFD2412D8E233635203B83E75F
:10D8080084F33BC100C0000084F3C53E203B7D1873
:10D818008E23CACABFD2BFD2CACA8E237D18203B64
:10D82800C53E84F3000000C03BC184F383E7203B7E
:10D8380036358E23412DBFD272DCCACAE0C47D18AA
:10D848007C0CC53E004000007C0C3BC1E0C483E773
:10D8580072DC3635412D412D363572DC83E7E0C464
:10D868003BC17C0C00000040C53E7C0C7D18E0C428
:10D87800CACA72DCBFD2412D8E233635203B83E7DE
:10D8880084F33BC100C0000084F3C53E203B7D18F3
:10D898008E23CACABFD2BFD2CACA8E237D18203BE4
:10D8A800C53E84F3000000C03BC184F383E7203BFE
:10D8B80036358E23412DBFD272DCCACAE0C47D182A
:10D8C8007C0CC53E004000007C0C3BC1E0C483E7F3
:10D8D80072DC3635412D412D363572DC83E7E0C4E4
:10D8E8003BC17C0C00000040C53E7C0C7D18E0C4A8
:10D8F800CACA72DCBFD2412D8E233635203B83E75E
:10D9080084F33BC100C0000084F3C53E203B7D1872
:10D918008E23CACABFD2BFD2CACA8E237D18203B63
:10D92800C53E84F3000000C03BC184F383E7203B7D
:10D9380036358E23412DBFD272DCCACAE0C47D18A9
:10D948007C0CC53E004000007C0C3BC1E0C483E772
:10D9580072DC3635412D412D363572DC83E7E0C463
:10D968003BC17C0C70F5000874F5000820E602083D
:10D978006C99000820DE020820D602086CA900086D
:10D9880038DA000838E2000820CE020820C602086B
:10D998006CB1000820BE020820B6020820AE0208BA
:10D9A80020A602086CA10008209E02082096020802
:10D9B800208E0208208602086CC10008207E02081A
:10D9C80020760208206E0208206602086CD1000842
:10D9D800205E020820560208204E0208204602084F
:10D9E8006CC90008203E0208203602086CB90008FD
:10D9F800202E020820260208201E020820160208EF
:10DA0800200E02082006020820FE010820F6010860
:10DA180020EE010820E6010820DE010820D60108D2
:10DA280020CE010820C6010820BE010820B6010842
:10DA38000000004074325F27143E74F0EF197EC571
:10DA4800D5E18FC7F2C00FF595D0FA2AB504D33FB8
:10DA580036358E23C53CEDEB8F15BEC3C3DDEEC94D
:10DA68004FC0BBF9DFD35A2E64094E3FAF378B1F27
:10DA7800203B83E7111152C2E1D999CC05C06EFE53
:10DA880067D77931050E713EDA395D1B2A393AE3D9
:10DA98007C0C3BC133D68ACF14C0230326DB533416
:10DAA80094123E3DB63B0817E53619DFD5077CC012
:10DAB800BFD2BFD27CC0D50719DFE5360817B63B01
:10DAC8003E3D9412533426DB230314C08ACF33D649
:10DAD8003BC17C0C3AE32A395D1BDA39713E050EED
:10DAE800793167D76EFE05C099CCE1D952C21111C0
:10DAF80083E7203B8B1FAF374E3F64095A2EDFD395
:10DB0800BBF94FC0EEC9C3DDBEC38F15EDEBC53CF5
:10DB18008E233635D33FB504FA2A95D00FF5F2C0D7
:10DB28008FC7D5E17EC5EF1974F0143E5F277432B4
:10DB3800004000005F278CCD74F0ECC17EC511E673
:10DB48008FC72B1E0FF50E3FFA2A6B2FD33F4BFBC7
:10DB58008E23CACAEDEB3BC3BEC371EAEEC93D22B0
:10DB6800BBF9B13F5A2E212C4E3F9CF68B1F51C852
:10DB780083E7E0C452C2EFEE99CC1F266EFEFB3F4E
:10DB880079319928713EFBF15D1B26C63AE3D6C66A
:10DB98003BC184F38ACFCD292303EC3F5334DA24E5
:10DBA8003E3D6CED08174AC419DF1BC97CC02BF831
:10DBB800BFD2412DD507843FE536E720B63BF8E8CC
:10DBC8009412C2C226DBADCB14C0DDFC33D676304E
:10DBD8007C0CC53E2A39C61CDA39A3E4050E8FC170
:10DBE80067D787CE05C09201E1D967331111AE3DE1
:10DBF800203B7D18AF3775E06409B2C0DFD3A6D1EA
:10DC08004FC04506C3DD12368F15423CC53C131480
:10DC1800363572DCB5042DC095D006D5F2C0F10AB0
:10DC2800D5E17138EF19823A143E8C0F7432A1D8BD
:10DC3800000000C08CCDA1D8ECC18C0F11E6823A4F
:10DC48002B1E71380E3FF10A6B2F06D54BFB2DC0EA
:10DC5800CACA72DC3BC3131471EA423C3D22123635
:10DC6800B13F4506212CA6D19CF6B2C051C875E03B
:10DC7800E0C47D18EFEEAE3D1F266733FB3F9201EF
:10DC8800992887CEFBF18FC126C6A3E4D6C6C61C49
:10DC980084F3C53ECD297630EC3FDDFCDA24ADCBEC
:10DCA8006CEDC2C24AC4F8E81BC9E7202BF8843FD0
:10DCB800412D412D843F2BF8E7201BC9F8E84AC4C1
:10DCC800C2C26CEDADCBDA24DDFCEC3F7630CD2959
:10DCD800C53E84F3C61CD6C6A3E426C68FC1FBF195
:10DCE80087CE99289201FB3F67331F26AE3DEFEEA2
:10DCF8007D18E0C475E051C8B2C09CF6A6D1212CAD
:10DD08004506B13F12363D22423C71EA13143BC32B
:10DD180072DCCACA2DC04BFB06D56B2FF10A0E3F29
:10DD280071382B1E823A11E68C0FECC1A1D88CCD2C
:10DD380000C00000A1D874328C0F143E823AEF194B
:10DD48007138D5E1F10AF2C006D595D02DC0B504D9
:10DD580072DC36351314C53C423C8F151236C3DDD0
:10DD680045064FC0A6D1DFD3B2C0640975E0AF370E
:10DD78007D18203BAE3D11116733E1D9920105C0F2
:10DD880087CE67D78FC1050EA3E4DA39C61C2A39B6
:10DD9800C53E7C0C763033D6DDFC14C0ADCB26DB1B
:10DDA800C2C29412F8E8B63BE720E536843FD507AF
:10DDB800412DBFD22BF87CC01BC919DF4AC40817F4
:10DDC8006CED3E3DDA245334EC3F2303CD298ACF52
:10DDD80084F33BC1D6C63AE326C65D1BFBF1713E10
:10DDE80099287931FB3F6EFE1F2699CCEFEE52C27F
:10DDF800E0C483E751C88B1F9CF64E3F212C5A2E56
:10DE0800B13FBBF93D22EEC971EABEC33BC3EDEB9E
:10DE1800CACA8E234BFBD33F6B2FFA2A0E3F0FF54E
:10DE28002B1E8FC711E67EC5ECC174F08CCD5F2721
:10DE38000000004074325F27143E74F0EF197EC56D
:10DE4800D5E18FC7F2C00FF595D0FA2AB504D33FB4
:10DE580036358E23C53CEDEB8F15BEC3C3DDEEC949
:10DE68004FC0BBF9DFD35A2E64094E3FAF378B1F23
:10DE7800203B83E7111152C2E1D999CC05C06EFE4F
:10DE880067D77931050E713EDA395D1B2A393AE3D5
:10DE98007C0C3BC133D68ACF14C0230326DB533412
:10DEA80094123E3DB63B0817E53619DFD5077CC00E
:10DEB800BFD2BFD27CC0D50719DFE5360817B63BFD
:10DEC8003E3D9412533426DB230314C08ACF33D645
:10DED8003BC17C0C3AE32A395D1BDA39713E050EE9
:10DEE800793167D76EFE05C099CCE1D952C21111BC
:10DEF80083E7203B8B1FAF374E3F64095A2EDFD391
:10DF0800BBF94FC0EEC9C3DDBEC38F15EDEBC53CF1
:10DF18008E233635D33FB504FA2A95D00FF5F2C0D3
:10DF28008FC7D5E17EC5EF1974F0143E5F277432B0
:10DF3800004000005F278CCD74F0ECC17EC511E66F
:10DF48008FC72B1E0FF50E3FFA2A6B2FD33F4BFBC3
:10DF58008E23CACAEDEB3BC3BEC371EAEEC93D22AC
:10DF6800BBF9B13F5A2E212C4E3F9CF68B1F51C84E
:10DF780083E7E0C452C2EFEE99CC1F266EFEFB3F4A
:10DF880079319928713EFBF15D1B26C63AE3D6C666
:10DF98003BC184F38ACFCD292303EC3F5334DA24E1
:10DFA8003E3D6CED08174AC419DF1BC97CC02BF82D
:10DFB800BFD2412DD507843FE536E720B63BF8E8C8
:10DFC8009412C2C226DBADCB14C0DDFC33D676304A
:10DFD8007C0CC53E2A39C61CDA39A3E4050E8FC16C
:10DFE80067D787CE05C09201E1D967331111AE3DDD
:10DFF800203B7D18AF3775E06409B2C0DFD3A6D1E6
:10E008004FC04506C3DD12368F15423CC53C13147C
:10E01800363572DCB5042DC095D006D5F2C0F10AAC
:10E02800D5E17138EF19823A143E8C0F7432A1D8B9
:10E03800000000C08CCDA1D8ECC18C0F11E6823A4B
:10E048002B1E71380E3FF10A6B2F06D54BFB2DC0E6
:10E05800CACA72DC3BC3131471EA423C3D22123631
:10E06800B13F4506212CA6D19CF6B2C051C875E037
:10E07800E0C47D18EFEEAE3D1F266733FB3F9201EB
:10E08800992887CEFBF18FC126C6A3E4D6C6C61C45
:10E0980084F3C53ECD297630EC3FDDFCDA24ADCBE8
:10E0A8006CEDC2C24AC4F8E81BC9E7202BF8843FCC
:10E0B800412D412D843F2BF8E7201BC9F8E84AC4BD
:10E0C800C2C26CEDADCBDA24DDFCEC3F7630CD2955
:10E0D800C53E84F3C61CD6C6A3E426C68FC1FBF191
:10E0E80087CE99289201FB3F67331F26AE3DEFEE9E
:10E0F8007D18E0C475E051C8B2C09CF6A6D1212CA9
:10E108004506B13F12363D22423C71EA13143BC327
:10E1180072DCCACA2DC04BFB06D56B2FF10A0E3F25
:10E1280071382B1E823A11E68C0FECC1A1D88CCD28
:10E1380000C00000A1D874328C0F143E823AEF1947
:10E148007138D5E1F10AF2C006D595D02DC0B504D5
:10E1580072DC36351314C53C423C8F151236C3DDCC
:10E1680045064FC0A6D1DFD3B2C0640975E0AF370A
:10E178007D18203BAE3D11116733E1D9920105C0EE
:10E1880087CE67D78FC1050EA3E4DA39C61C2A39B2
:10E19800C53E7C0C763033D6DDFC14C0ADCB26DB17
:10E1A800C2C29412F8E8B63BE720E536843FD507AB
:10E1B800412DBFD22BF87CC01BC919DF4AC40817F0
:10E1C8006CED3E3DDA245334EC3F2303CD298ACF4E
:10E1D80084F33BC1D6C63AE326C65D1BFBF1713E0C
:10E1E80099287931FB3F6EFE1F2699CCEFEE52C27B
:10E1F800E0C483E751C88B1F9CF64E3F212C5A2E52
:10E20800B13FBBF93D22EEC971EABEC33BC3EDEB9A
:10E21800CACA8E234BFBD33F6B2FFA2A0E3F0FF54A
:10E228002B1E8FC711E67EC5ECC174F08CCD5F271D
:10E238000000004067331F263E3D6CED8F15BEC3BE
:10E2480072DCCACA14C0DDFC67D779318C0F143E62
:10E25800203B7D18E53619DF45064FC095D006D519
:10E268003BC17C0CA3E4DA392B1E71384E3F64099C
:10E27800412DBFD29CF6B2C08FC7D5E126C65D1B23
:10E2880084F3C53EFA2A6B2FB13FBBF9E7201BC9BF
:10E2980083E7E0C4ECC174F087CE99282303EC3FF0
:10E2A80036358E23423C71EA9412C2C2E1D999CC28
:10E2B80000C00000E1D9673394123E3D423C8F15FF
:10E2C800363572DC230314C087CE67D7ECC18C0FB8
:10E2D80083E7203BE720E536B13F4506FA2A95D08B
:10E2E80084F33BC126C6A3E48FC72B1E9CF64E3F82
:10E2F800412D412D4E3F9CF62B1E8FC7A3E426C609
:10E308003BC184F395D0FA2A4506B13FE536E720AC
:10E31800203B83E78C0FECC167D787CE14C023035B
:10E3280072DC36358F15423C3E3D94126733E1D995
:10E33800000000C099CCE1D9C2C2941271EA423CF3
:10E348008E233635EC3F2303992887CE74F0ECC131
:10E35800E0C483E71BC9E720BBF9B13F6B2FFA2A5A
:10E36800C53E84F35D1B26C6D5E18FC7B2C09CF6B7
:10E37800BFD2412D64094E3F71382B1EDA39A3E410
:10E388007C0C3BC106D595D04FC0450619DFE53654
:10E398007D18203B143E8C0F793167D7DDFC14C003
:10E3A800CACA72DCBEC38F156CED3E3D1F266733AB
:10E3B800004000001F2699CC6CEDC2C2BEC371EAB2
:10E3C800CACA8E23DDFCEC3F79319928143E74F0DB
:10E3D8007D18E0C419DF1BC94FC0BBF906D56B2FE8
:10E3E8007C0CC53EDA395D1B7138D5E16409B2C0D1
:10E3F800BFD2BFD2B2C06409D5E171385D1BDA392A
:10E40800C53E7C0C6B2F06D5BBF94FC01BC919DF65
:10E41800E0C47D1874F0143E99287931EC3FDDFC96
:10E428008E23CACA71EABEC3C2C26CED99CC1F263C
:10E438000000004067331F263E3D6CED8F15BEC3BC
:10E4480072DCCACA14C0DDFC67D779318C0F143E60
:10E45800203B7D18E53619DF45064FC095D006D517
:10E468003BC17C0CA3E4DA392B1E71384E3F64099A
:10E47800412DBFD29CF6B2C08FC7D5E126C65D1B21
:10E4880084F3C53EFA2A6B2FB13FBBF9E7201BC9BD
:10E4980083E7E0C4ECC174F087CE99282303EC3FEE
:10E4A80036358E23423C71EA9412C2C2E1D999CC26
:10E4B80000C00000E1D9673394123E3D423C8F15FD
:10E4C800363572DC230314C087CE67D7ECC18C0FB6
:10E4D80083E7203BE720E536B13F4506FA2A95D089
:10E4E80084F33BC126C6A3E48FC72B1E9CF64E3F80
:10E4F800412D412D4E3F9CF62B1E8FC7A3E426C607
:10E508003BC184F395D0FA2A4506B13FE536E720AA
:10E51800203B83E78C0FECC167D787CE14C0230359
:10E5280072DC36358F15423C3E3D94126733E1D993
:10E53800000000C099CCE1D9C2C2941271EA423CF1
:10E548008E233635EC3F2303992887CE74F0ECC12F
:10E55800E0C483E71BC9E720BBF9B13F6B2FFA2A58
:10E56800C53E84F35D1B26C6D5E18FC7B2C09CF6B5
:10E57800BFD2412D64094E3F71382B1EDA39A3E40E
:10E588007C0C3BC106D595D04FC0450619DFE53652
:10E598007D18203B143E8C0F793167D7DDFC14C001
:10E5A800CACA72DCBEC38F156CED3E3D1F266733A9
:10E5B800004000001F2699CC6CEDC2C2BEC371EAB0
:10E5C800CACA8E23DDFCEC3F79319928143E74F0D9
:10E5D8007D18E0C419DF1BC94FC0BBF906D56B2FE6
:10E5E8007C0CC53EDA395D1B7138D5E16409B2C0CF
:10E5F800BFD2BFD2B2C06409D5E171385D1BDA3928
:10E60800C53E7C0C6B2F06D5BBF94FC01BC919DF63
:10E61800E0C47D1874F0143E99287931EC3FDDFC94
:10E628008E23CACA71EABEC3C2C26CED99CC1F263A
:10E638000000004067331F263E3D6CED8F15BEC3BA
:10E6480072DCCACA14C0DDFC67D779318C0F143E5E
:10E65800203B7D18E53619DF45064FC095D006D515
:10E668003BC17C0CA3E4DA392B1E71384E3F640998
:10E67800412DBFD29CF6B2C08FC7D5E126C65D1B1F
:10E6880084F3C53EFA2A6B2FB13FBBF9E7201BC9BB
:10E6980083E7E0C4ECC174F087CE99282303EC3FEC
:10E6A80036358E23423C71EA9412C2C2E1D999CC24
:10E6B80000C00000E1D9673394123E3D423C8F15FB
:10E6C800363572DC230314C087CE67D7ECC18C0FB4
:10E6D80083E7203BE720E536B13F4506FA2A95D087
:10E6E80084F33BC126C6A3E48FC72B1E9CF64E3F7E
:10E6F800412D412D4E3F9CF62B1E8FC7A3E426C605
:10E708003BC184F395D0FA2A4506B13FE536E720A8
:10E71800203B83E78C0FECC167D787CE14C0230357
:10E7280072DC36358F15423C3E3D94126733E1D991
:10E73800000000C099CCE1D9C2C2941271EA423CEF
:10E748008E233635EC3F2303992887CE74F0ECC12D
:10E75800E0C483E71BC9E720BBF9B13F6B2FFA2A56
:10E76800C53E84F35D1B26C6D5E18FC7B2C09CF6B3
:10E77800BFD2412D64094E3F71382B1EDA39A3E40C
:10E788007C0C3BC106D595D04FC0450619DFE53650
:10E798007D18203B143E8C0F793167D7DDFC14C0FF
:10E7A800CACA72DCBEC38F156CED3E3D1F266733A7
:10E7B800004000001F2699CC6CEDC2C2BEC371EAAE
:10E7C800CACA8E23DDFCEC3F79319928143E74F0D7
:10E7D8007D18E0C419DF1BC94FC0BBF906D56B2FE4
:10E7E8007C0CC53EDA395D1B7138D5E16409B2C0CD
:10E7F800BFD2BFD2B2C06409D5E171385D1BDA3926
:10E80800C53E7C0C6B2F06D5BBF94FC01BC919DF61
:10E81800E0C47D1874F0143E99287931EC3FDDFC92
:10E828008E23CACA71EABEC3C2C26CED99CC1F2638
:10E838000000004067331F263E3D6CED8F15BEC3B8
:10E8480072DCCACA14C0DDFC67D779318C0F143E5C
:10E85800203B7D18E53619DF45064FC095D006D513
:10E868003BC17C0CA3E4DA392B1E71384E3F640996
:10E87800412DBFD29CF6B2C08FC7D5E126C65D1B1D
:10E8880084F3C53EFA2A6B2FB13FBBF9E7201BC9B9
:10E8980083E7E0C4ECC174F087CE99282303EC3FEA
:10E8A80036358E23423C71EA9412C2C2E1D999CC22
:10E8B80000C00000E1D9673394123E3D423C8F15F9
:10E8C800363572DC230314C087CE67D7ECC18C0FB2
:10E8D80083E7203BE720E536B13F4506FA2A95D085
:10E8E80084F33BC126C6A3E48FC72B1E9CF64E3F7C
:10E8F800412D412D4E3F9CF62B1E8FC7A3E426C603
:10E908003BC184F395D0FA2A4506B13FE536E720A6
:10E91800203B83E78C0FECC167D787CE14C0230355
:10E9280072DC36358F15423C3E3D94126733E1D98F
:10E93800000000C099CCE1D9C2C2941271EA423CED
:10E948008E233635EC3F2303992887CE74F0ECC12B
:10E95800E0C483E71BC9E720BBF9B13F6B2FFA2A54
:10E96800C53E84F35D1B26C6D5E18FC7B2C09CF6B1
:10E97800BFD2412D64094E3F71382B1EDA39A3E40A
:10E988007C0C3BC106D595D04FC0450619DFE5364E
:10E998007D18203B143E8C0F793167D7DDFC14C0FD
:10E9A800CACA72DCBEC38F156CED3E3D1F266733A5
:10E9B800004000001F2699CC6CEDC2C2BEC371EAAC
:10E9C800CACA8E23DDFCEC3F79319928143E74F0D5
:10E9D8007D18E0C419DF1BC94FC0BBF906D56B2FE2
:10E9E8007C0CC53EDA395D1B7138D5E16409B2C0CB
:10E9F800BFD2BFD2B2C06409D5E171385D1BDA3924
:10EA0800C53E7C0C6B2F06D5BBF94FC01BC919DF5F
:10EA1800E0C47D1874F0143E99287931EC3FDDFC90
:10EA28008E23CACA71EABEC3C2C26CED99CC1F2636
:10EA380001000201000201000201000200030102BC
:10EA480001030100020302000306080B0D10121552
:10EA5800171A1C1F0205070A0C0F111416191B1E82
:10EA680088EE02088CEE020898EE0208A0EE020872
:10EA7800ACEE020805004F008400AA00C400D700CD
:10EA8800E400EE00F400F900FC00000000402C3720
:10EA9800D72F7428A622981ED41A9F183F168A14B6
:10EAA80035133C12C0116811FC10CA105710F70F2B
:10EAB800BC0FA80F920F670F740F200FCC0E470ED4
:10EAC800DD0D590DAD0C2D0C800BC90A140A550922
:10EAD800B2083D08EE07D107B907C307B907C00751
:10EAE800AE0789076907B6079F070B0809080040A2
:10EAF800CB377F30CB2ADB26CF224120E21D231CD7
:10EB0800001B901A631B9B1C6B1D291EC61D1C1B1A
:10EB1800D117CC145A129610720FEB0EE20E8D0F0D
:10EB2800DB10741255138814BE159416471500117E
:10EB3800FE0DD50B1D0AF2081A086A070507DD063F
:10EB4800DB06FB06F8064D07B0074C080709A009C5
:10EB58000040DA3C403AB33912372636413597300F
:10EB6800812AB52681244A24BB24A2252324E8200F
:10EB7800F21D6A1BFC18641600141F121010200ED8
:10EB88004C0C9B0A48096908AE070E07890621063E
:10EB98007505A3042204F203CA03910366033E0326
:10EBA8001503EF02D102B7029F028D027B026202B7
:10EBB80056020040BC3B153807355832CC2F772D0C
:10EBC8004C2B4C296A27A425F6236322F3209C1F8B
:10EBD8004F1E0B1DCB1B921A6019431833172F16A3
:10EBE80036154E147513A212DB1122118110FB0F7A
:10EBF800800F780EDA0D630DEA0C5F0CD50B4B0B0A
:10EC0800C80A4F0AE10979091609BA086208120800
:10EC1800CB078907C83E603A233C953F00409536AC
:10EC2800012C2924F71D6518D3141C134413CF1481
:10EC3800BE158A17C617B31611154413A6110A1064
:10EC4800790E130D860B380A11091B08E9079C0772
:10EC58004507E80686068206AB06E7062507570736
:10EC68007C073A07BC064606A50584059505CC052C
:10EC78006D069E063607000044ED000878B10108CD
:10EC880078AD010878A9010878A5010878A10108DC
:10EC9800789D01087899010878950108789101080C
:10ECA800788D01087889010878850108788101083C
:10ECB800787D01087879010878750108787101086C
:10ECC800786D01087869010878650108786101089C
:10ECD800785D0108785901087855010878510108CC
:10ECE800784D0108784901087845010878410108FC
:10ECF800783D01087839010878350108783101082C
:10ED0800782D01087829010878250108782101085B
:10ED1800781D01087819010878150108781101088B
:10ED2800780D0108780901087805010878010108BB
:10ED380078FD000878F9000878F500080000412DF2
:10ED48000040412D0000BFD200C0BFD20000412DBD
:10ED58000040412D0000BFD200C0BFD20000412DAD
:10ED68000040412D0000BFD200C0BFD20000412D9D
:10ED78000040412D0000BFD200C0BFD20000412D8D
:10ED88000040412D0000BFD200C0BFD20000412D7D
:10ED98000040412D0000BFD200C0BFD20000412D6D
:10EDA8000040412D0000BFD200C0BFD20000412D5D
:10EDB8000040412D0000BFD200C0BFD20000412D4D
:10EDC8000040412D0000BFD200C0BFD20000412D3D
:10EDD8000040412D0000BFD200C0BFD20000412D2D
:10EDE8000040412D0000BFD200C0BFD20000412D1D
:10EDF8000040412D0000BFD200C0BFD20000412D0D
:10EE08000040412D0000BFD200C0BFD20000412DFC
:10EE18000040412D0000BFD200C0BFD20000412DEC
:10EE28000040412D0000BFD200C0BFD20000412DDC
:10EE38000040412D0000BFD200C0BFD20000412DCC
:10EE48000040412D0000BFD200C0BFD20000412DBC
:10EE58000040412D0000BFD200C0BFD20000412DAC
:10EE68000040412D0000BFD200C0BFD20000412D9C
:10EE78000040412D0000BFD200C0BFD20000412D8C
:10EE88000040412D0000BFD200C0BFD20000412D7C
:10EE98000040412D0000BFD200C0BFD20000412D6C
:10EEA8000040412D0000BFD200C0BFD20000412D5C
:10EEB8000040412D0000BFD200C0BFD20000412D4C
:10EEC8000040412D0000BFD200C0BFD20000412D3C
:10EED8000040412D0000BFD200C0BFD20000412D2C
:10EEE8000040412D0000BFD200C0BFD20000412D1C
:10EEF8000040412D0000BFD200C0BFD20000412D0C
:10EF08000040412D0000BFD200C0BFD20000412DFB
:10EF18000040412D0000BFD200C0BFD20000412DEB
:10EF28000040412D0000BFD200C0BFD20000412DDB
:10EF38000040412D0000BFD200C0BFD20000412DCB
:10EF48000040412D0000BFD200C0BFD20000412DBB
:10EF58000040412D0000BFD200C0BFD20000412DAB
:10EF68000040412D0000BFD200C0BFD20000412D9B
:10EF78000040412D0000BFD200C0BFD20000412D8B
:10EF88000040412D0000BFD200C0BFD20000412D7B
:10EF98000040412D0000BFD200C0BFD20000412D6B
:10EFA8000040412D0000BFD200C0BFD20000412D5B
:10EFB8000040412D0000BFD200C0BFD20000412D4B
:10EFC8000040412D0000BFD200C0BFD20000412D3B
:10EFD8000040412D0000BFD200C0BFD20000412D2B
:10EFE8000040412D0000BFD200C0BFD20000412D1B
:10EFF8000040412D0000BFD200C0BFD20000412D0B
:10F008000040412D0000BFD200C0BFD20000412DFA
:10F018000040412D0000BFD200C0BFD20000412DEA
:10F028000040412D0000BFD200C0BFD20000412DDA
:10F038000040412D0000BFD200C0BFD20000412DCA
:10F048000040412D0000BFD200C0BFD20000412DBA
:10F058000040412D0000BFD200C0BFD20000412DAA
:10F068000040412D0000BFD200C0BFD20000412D9A
:10F078000040412D0000BFD200C0BFD20000412D8A
:10F088000040412D0000BFD200C0BFD20000412D7A
:10F098000040412D0000BFD200C0BFD20000412D6A
:10F0A8000040412D0000BFD200C0BFD20000412D5A
:10F0B8000040412D0000BFD200C0BFD20000412D4A
:10F0C8000040412D0000BFD200C0BFD20000412D3A
:10F0D8000040412D0000BFD200C0BFD20000412D2A
:10F0E8000040412D0000BFD200C0BFD20000412D1A
:10F0F8000040412D0000BFD200C0BFD20000412D0A
:10F108000040412D0000BFD200C0BFD20000412DF9
:10F118000040412D0000BFD200C0BFD20000412DE9
:10F128000040412D0000BFD200C0BFD20000412DD9
:10F138000040412D0000BFD200C0BFD200006409CA
:10F1480094125D1B8E23FA2A7931E536203B143E52
:10F15800B13FEC3FC53E423C71386733412D1F2615
:10F168002B1E8F157C0C2303BBF974F083E719DF82
:10F1780067D795D0CACA26C6C2C2B2C000C0B2C03C
:10F18800C2C226C6CACA95D067D719DF83E774F00A
:10F19800BBF923037C0C8F152B1E1F26412D6733CB
:10F1A8007138423CC53EEC3FB13F143E203BE5364A
:10F1B8007931FA2A8E235D1B9412640900009CF6AB
:10F1C8006CEDA3E472DC06D587CE1BC9E0C4ECC1A4
:10F1D8004FC014C03BC1BEC38FC799CCBFD2E1D9C1
:10F1E800D5E171EA84F3DDFC45068C0F7D18E72034
:10F1F80099286B2F3635DA393E3D4E3F00404E3F59
:10F208003E3DDA3936356B2F9928E7207D188C0F6B
:10F218004506DDFC84F371EAD5E1E1D9BFD299CC8A
:10F228008FC7BEC33BC114C04FC0ECC1E0C41BC9EB
:10F2380087CE06D572DCA3E46CED9CF60000640969
:10F2480094125D1B8E23FA2A7931E536203B143E51
:10F25800B13FEC3FC53E423C71386733412D1F2614
:10F268002B1E8F157C0C2303BBF974F083E719DF81
:10F2780067D795D0CACA26C6C2C2B2C000C0B2C03B
:10F28800C2C226C6CACA95D067D719DF83E774F009
:10F29800BBF923037C0C8F152B1E1F26412D6733CA
:10F2A8007138423CC53EEC3FB13F143E203BE53649
:10F2B8007931FA2A8E235D1B9412640900009CF6AA
:10F2C8006CEDA3E472DC06D587CE1BC9E0C4ECC1A3
:10F2D8004FC014C03BC1BEC38FC799CCBFD2E1D9C0
:10F2E800D5E171EA84F3DDFC45068C0F7D18E72033
:10F2F80099286B2F3635DA393E3D4E3F00404E3F58
:10F308003E3DDA3936356B2F9928E7207D188C0F6A
:10F318004506DDFC84F371EAD5E1E1D9BFD299CC89
:10F328008FC7BEC33BC114C04FC0ECC1E0C41BC9EA
:10F3380087CE06D572DCA3E46CED9CF60000640968
:10F3480094125D1B8E23FA2A7931E536203B143E50
:10F35800B13FEC3FC53E423C71386733412D1F2613
:10F368002B1E8F157C0C2303BBF974F083E719DF80
:10F3780067D795D0CACA26C6C2C2B2C000C0B2C03A
:10F38800C2C226C6CACA95D067D719DF83E774F008
:10F39800BBF923037C0C8F152B1E1F26412D6733C9
:10F3A8007138423CC53EEC3FB13F143E203BE53648
:10F3B8007931FA2A8E235D1B9412640900009CF6A9
:10F3C8006CEDA3E472DC06D587CE1BC9E0C4ECC1A2
:10F3D8004FC014C03BC1BEC38FC799CCBFD2E1D9BF
:10F3E800D5E171EA84F3DDFC45068C0F7D18E72032
:10F3F80099286B2F3635DA393E3D4E3F00404E3F57
:10F408003E3DDA3936356B2F9928E7207D188C0F69
:10F418004506DDFC84F371EAD5E1E1D9BFD299CC88
:10F428008FC7BEC33BC114C04FC0ECC1E0C41BC9E9
:10F4380087CE06D572DCA3E46CED9CF60000640967
:10F4480094125D1B8E23FA2A7931E536203B143E4F
:10F45800B13FEC3FC53E423C71386733412D1F2612
:10F468002B1E8F157C0C2303BBF974F083E719DF7F
:10F4780067D795D0CACA26C6C2C2B2C000C0B2C039
:10F48800C2C226C6CACA95D067D719DF83E774F007
:10F49800BBF923037C0C8F152B1E1F26412D6733C8
:10F4A8007138423CC53EEC3FB13F143E203BE53647
:10F4B8007931FA2A8E235D1B9412640900009CF6A8
:10F4C8006CEDA3E472DC06D587CE1BC9E0C4ECC1A1
:10F4D8004FC014C03BC1BEC38FC799CCBFD2E1D9BE
:10F4E800D5E171EA84F3DDFC45068C0F7D18E72031
:10F4F80099286B2F3635DA393E3D4E3F00404E3F56
:10F508003E3DDA3936356B2F9928E7207D188C0F68
:10F518004506DDFC84F371EAD5E1E1D9BFD299CC87
:10F528008FC7BEC33BC114C04FC0ECC1E0C41BC9E8
:10F5380087CE06D572DCA3E46CED9CF601000001D1
:10F548005CEA000850EA0008000000000102030419
:10F55800010203040607080900000000000000007B
:10F5680001020304060708090104201D0E091318E7
:10F578000000203BBFD283E7004083E7BFD2203B97
:10F588000000E0C4412D7D1800C07D18412DE0C465
:10F598000000203BBFD283E7004083E7BFD2203B77
:10F5A8000000E0C4412D7D1800C07D18412DE0C445
:10F5B8000000203BBFD283E7004083E7BFD2203B57
:10F5C8000000E0C4412D7D1800C07D18412DE0C425
:10F5D8000000203BBFD283E7004083E7BFD2203B37
:10F5E8000000E0C4412D7D1800C07D18412DE0C405
:10F5F8000000203BBFD283E7004083E7BFD2203B17
:10F608000000E0C4412D7D1800C07D18412DE0C4E4
:10F618000000203BBFD283E7004083E7BFD2203BF6
:10F628000000E0C4412D7D1800C07D18412DE0C4C4
:10F638000000203BBFD283E7004083E7BFD2203BD6
:10F648000000E0C4412D7D1800C07D18412DE0C4A4
:10F658000000203BBFD283E7004083E7BFD2203BB6
:10F668000000E0C4412D7D1800C07D18412DE0C484
:10F678000000203BBFD283E7004083E7BFD2203B96
:10F688000000E0C4412D7D1800C07D18412DE0C464
:10F698000000203BBFD283E7004083E7BFD2203B76
:10F6A8000000E0C4412D7D1800C07D18412DE0C444
:10F6B8000000203BBFD283E7004083E7BFD2203B56
:10F6C8000000E0C4412D7D1800C07D18412DE0C424
:10F6D8000000203BBFD283E7004083E7BFD2203B36
:10F6E8000000E0C4412D7D1800C07D18412DE0C404
:10F6F8000000203BBFD283E7004083E7BFD2203B16
:10F708000000E0C4412D7D1800C07D18412DE0C4E3
:10F718000000203BBFD283E7004083E7BFD2203BF5
:10F728000000E0C4412D7D1800C07D18412DE0C4C3
:10F738000000203BBFD283E7004083E7BFD2203BD5
:10F748000000E0C4412D7D1800C07D18412DE0C4A3
:10F758000000203BBFD283E7004083E7BFD2203BB5
:10F768000000E0C4412D7D1800C07D18412DE0C483
:10F778000000203BBFD283E7004083E7BFD2203B95
:10F788000000E0C4412D7D1800C07D18412DE0C463
:10F798000000203BBFD283E7004083E7BFD2203B75
:10F7A8000000E0C4412D7D1800C07D18412DE0C443
:10F7B8000000203BBFD283E7004083E7BFD2203B55
:10F7C8000000E0C4412D7D1800C07D18412DE0C423
:10F7D8000000203BBFD283E7004083E7BFD2203B35
:10F7E8000000E0C4412D7D1800C07D18412DE0C403
:10F7F8000000203BBFD283E7004083E7BFD2203B15
:10F808000000E0C4412D7D1800C07D18412DE0C4E2
:10F818000000203BBFD283E7004083E7BFD2203BF4
:10F828000000E0C4412D7D1800C07D18412DE0C4C2
:10F838000000203BBFD283E7004083E7BFD2203BD4
:10F848000000E0C4412D7D1800C07D18412DE0C4A2
:10F858000000203BBFD283E7004083E7BFD2203BB4
:10F868000000E0C4412D7D1800C07D18412DE0C482
:10F878000000203BBFD283E7004083E7BFD2203B94
:10F888000000E0C4412D7D1800C07D18412DE0C462
:10F898000000203BBFD283E7004083E7BFD2203B74
:10F8A8000000E0C4412D7D1800C07D18412DE0C442
:10F8B8000000203BBFD283E7004083E7BFD2203B54
:10F8C8000000E0C4412D7D1800C07D18412DE0C422
:10F8D8000000203BBFD283E7004083E7BFD2203B34
:10F8E8000000E0C4412D7D1800C07D18412DE0C402
:10F8F8000000203BBFD283E7004083E7BFD2203B14
:10F908000000E0C4412D7D1800C07D18412DE0C4E1
:10F918000000203BBFD283E7004083E7BFD2203BF3
:10F928000000E0C4412D7D1800C07D18412DE0C4C1
:10F938000000203BBFD283E7004083E7BFD2203BD3
:10F948000000E0C4412D7D1800C07D18412DE0C4A1
:10F958000000203BBFD283E7004083E7BFD2203BB3
:10F968000000E0C4412D7D1800C07D18412DE0C481
:10F978000000B63B06D53AE3B13FEFEE99CC12361C
:10F988007C0CF2C0E7205F27C2C2B504DA39A6D1E1
:10F9980083E7FB3F71EA8ACF7138D507ECC1DA24D7
:10F9A8008E238FC16409AF3787CEEDEBEC3F11E6AC
:10F9B800BFD2823A23033BC399288B1FB2C0050EDE
:10F9C8003635ADCB74F0843FD5E133D6423C6EFE7C
:10F9D800E0C4212C5D1B2DC0941274321BC90FF595
:10F9E800C53EC3DDE1D9AE3DBBF9D6C66B2F0817BE
:10F9F80000C008176B2FD6C6BBF9AE3DE1D9C3DDF1
:10FA0800C53E0FF51BC9743294122DC05D1B212C05
:10FA1800E0C46EFE423C33D6D5E1843F74F0ADCBF2
:10FA28003635050EB2C08B1F99283BC32303823A93
:10FA3800BFD211E6EC3FEDEB87CEAF3764098FC13B
:10FA48008E23DA24ECC1D50771388ACF71EAFB3FDF
:10FA580083E7A6D1DA39B504C2C25F27E720F2C02E
:10FA68007C0C123699CCEFEEB13F3AE306D5B63BA3
:10FA780000004AC4FA2AC61C4FC011116733EEC9E8
:10FA880084F30E3F19DFA1D83E3D4BFB26C65A2E04
:10FA98007D1805C08F1576308FC72BF8143E26DBEE
:10FAA80072DC713E9CF651C87931131414C0EF19F9
:10FAB800412D7EC5DDFCC53C67D775E04E3FFBF1A7
:10FAC800CACA53348C0F7CC02B1ECD29BEC39201E9
:10FAD800203BDFD3A3E4D33F6CED8CCDE536F10AB0
:10FAE8003BC13D221F2652C245062A3995D0F8E867
:10FAF8000040F8E895D02A39450652C21F263D2213
:10FB08003BC1F10AE5368CCD6CEDD33FA3E4DFD3DE
:10FB1800203B9201BEC3CD292B1E7CC08C0F5334D1
:10FB2800CACAFBF14E3F75E067D7C53CDDFC7EC510
:10FB3800412DEF1914C01314793151C89CF6713E48
:10FB480072DC26DB143E2BF88FC776308F1505C084
:10FB58007D185A2E26C64BFB3E3DA1D819DF0E3F15
:10FB680084F3EEC9673311114FC0C61CFA2A4AC480
:10FB78000000B63B06D53AE3B13FEFEE99CC12361A
:10FB88007C0CF2C0E7205F27C2C2B504DA39A6D1DF
:10FB980083E7FB3F71EA8ACF7138D507ECC1DA24D5
:10FBA8008E238FC16409AF3787CEEDEBEC3F11E6AA
:10FBB800BFD2823A23033BC399288B1FB2C0050EDC
:10FBC8003635ADCB74F0843FD5E133D6423C6EFE7A
:10FBD800E0C4212C5D1B2DC0941274321BC90FF593
:10FBE800C53EC3DDE1D9AE3DBBF9D6C66B2F0817BC
:10FBF80000C008176B2FD6C6BBF9AE3DE1D9C3DDEF
:10FC0800C53E0FF51BC9743294122DC05D1B212C03
:10FC1800E0C46EFE423C33D6D5E1843F74F0ADCBF0
:10FC28003635050EB2C08B1F99283BC32303823A91
:10FC3800BFD211E6EC3FEDEB87CEAF3764098FC139
:10FC48008E23DA24ECC1D50771388ACF71EAFB3FDD
:10FC580083E7A6D1DA39B504C2C25F27E720F2C02C
:10FC68007C0C123699CCEFEEB13F3AE306D5B63BA1
:10FC780000004AC4FA2AC61C4FC011116733EEC9E6
:10FC880084F30E3F19DFA1D83E3D4BFB26C65A2E02
:10FC98007D1805C08F1576308FC72BF8143E26DBEC
:10FCA80072DC713E9CF651C87931131414C0EF19F7
:10FCB800412D7EC5DDFCC53C67D775E04E3FFBF1A5
:10FCC800CACA53348C0F7CC02B1ECD29BEC39201E7
:10FCD800203BDFD3A3E4D33F6CED8CCDE536F10AAE
:10FCE8003BC13D221F2652C245062A3995D0F8E865
:10FCF8000040F8E895D02A39450652C21F263D2211
:10FD08003BC1F10AE5368CCD6CEDD33FA3E4DFD3DC
:10FD1800203B9201BEC3CD292B1E7CC08C0F5334CF
:10FD2800CACAFBF14E3F75E067D7C53CDDFC7EC50E
:10FD3800412DEF1914C01314793151C89CF6713E46
:10FD480072DC26DB143E2BF88FC776308F1505C082
:10FD58007D185A2E26C64BFB3E3DA1D819DF0E3F13
:10FD680084F3EEC9673311114FC0C61CFA2A4AC47E
:10FD78000000423C67D719DFC53E9CF68FC76B2F42
:10FD88007D1814C094126733CACA74F0B13FA3E453
:10FD9800BFD2DA394506ECC18E231F26C2C223031F
:10FDA800203B06D5D5E14E3F84F31BC979318F1529
:10FDB80000C08F1579311BC984F34E3FD5E106D5B4
:10FDC800203B2303C2C21F268E23ECC14506DA3925
:10FDD800BFD2A3E4B13F74F0CACA6733941214C007
:10FDE8007D186B2F8FC79CF6C53E19DF67D7423C3D
:10FDF8000000BEC39928E7203BC16409713895D03B
:10FE080083E7EC3F6CED99CC36358C0F4FC05D1B0A
:10FE1800412D26C6BBF9143E72DCE1D93E3DDDFC1E
:10FE2800E0C4FA2A2B1EB2C07C0CE53687CE71EAF4
:10FE3800004071EA87CEE5367C0CB2C02B1EFA2A48
:10FE4800E0C4DDFC3E3DE1D972DC143EBBF926C6B8
:10FE5800412D5D1B4FC08C0F363599CC6CEDEC3FB6
:10FE680083E795D0713864093BC1E7209928BEC360
:10FE78000000423C67D719DFC53E9CF68FC76B2F41
:10FE88007D1814C094126733CACA74F0B13FA3E452
:10FE9800BFD2DA394506ECC18E231F26C2C223031E
:10FEA800203B06D5D5E14E3F84F31BC979318F1528
:10FEB80000C08F1579311BC984F34E3FD5E106D5B3
:10FEC800203B2303C2C21F268E23ECC14506DA3924
:10FED800BFD2A3E4B13F74F0CACA6733941214C006
:10FEE8007D186B2F8FC79CF6C53E19DF67D7423C3C
:10FEF8000000BEC39928E7203BC16409713895D03A
:10FF080083E7EC3F6CED99CC36358C0F4FC05D1B09
:10FF1800412D26C6BBF9143E72DCE1D93E3DDDFC1D
:10FF2800E0C4FA2A2B1EB2C07C0CE53687CE71EAF3
:10FF3800004071EA87CEE5367C0CB2C02B1EFA2A47
:10FF4800E0C4DDFC3E3DE1D972DC143EBBF926C6B7
:10FF5800412D5D1B4FC08C0F363599CC6CEDEC3FB5
:10FF680083E795D0713864093BC1E7209928BEC35F
:10FF78000000423C67D719DFC53E9CF68FC76B2F40
:10FF88007D1814C094126733CACA74F0B13FA3E451
:10FF9800BFD2DA394506ECC18E231F26C2C223031D
:10FFA800203B06D5D5E14E3F84F31BC979318F1527
:10FFB80000C08F1579311BC984F34E3FD5E106D5B2
:10FFC800203B2303C2C21F268E23ECC14506DA3923
:10FFD800BFD2A3E4B13F74F0CACA6733941214C005
:10FFE8007D186B2F8FC79CF6C53E19DF67D7423C3B
:08FFF8000000BEC39928E720B8
:020000040801F1
:100000003BC16409713895D083E7EC3F6CED99CC26
:1000100036358C0F4FC05D1B412D26C6BBF9143EF3
:1000200072DCE1D93E3DDDFCE0C4FA2A2B1EB2C0F1
:100030007C0CE53687CE71EA004071EA87CEE53662
:100040007C0CB2C02B1EFA2AE0C4DDFC3E3DE1D997
:1000500072DC143EBBF926C6412D5D1B4FC08C0FD0
:10006000363599CC6CEDEC3F83E795D07138640957
:100070003BC1E7209928BEC30000423C67D719DF87
:10008000C53E9CF68FC76B2F7D1814C09412673342
:10009000CACA74F0B13FA3E4BFD2DA394506ECC155
:1000A0008E231F26C2C22303203B06D5D5E14E3F37
:1000B00084F31BC979318F1500C08F1579311BC9A5
:1000C00084F34E3FD5E106D5203B2303C2C21F2651
:1000D0008E23ECC14506DA39BFD2A3E4B13F74F0F8
:1000E000CACA6733941214C07D186B2F8FC79CF651
:1000F000C53E19DF67D7423C0000BEC39928E72000
:100100003BC16409713895D083E7EC3F6CED99CC25
:1001100036358C0F4FC05D1B412D26C6BBF9143EF2
:1001200072DCE1D93E3DDDFCE0C4FA2A2B1EB2C0F0
:100130007C0CE53687CE71EA004071EA87CEE53661
:100140007C0CB2C02B1EFA2AE0C4DDFC3E3DE1D996
:1001500072DC143EBBF926C6412D5D1B4FC08C0FCF
:10016000363599CC6CEDEC3F83E795D07138640956
:100170003BC1E7209928BEC30000C53CE1D926DB7E
:100180003E3D6EFEBEC35F278E2352C22303B63BA5
:1001900067D7C3DD143E4BFBE0C4CD29E7208FC1F8
:1001A0004506823A06D575E0C53E2BF826C6212CB9
:1001B0002B1EF2C064092A39BFD23AE34E3F0FF535
:1001C0008FC75A2E5D1B7CC07C0CAF3795D011E6D3
:1001D000B13FFBF11BC976307D182DC08C0F123654
:1001E00087CEF8E8EC3FEFEECACA74328F1505C02F
:1001F0009412533499CCEDEB0040EDEB99CC533491
:10020000941205C08F157432CACAEFEEEC3FF8E8BD
:1002100087CE12368C0F2DC07D1876301BC9FBF1AE
:10022000B13F11E695D0AF377C0C7CC05D1B5A2ED8
:100230008FC70FF54E3F3AE3BFD22A396409F2C0A7
:100240002B1E212C26C62BF8C53E75E006D5823A1A
:1002500045068FC1E720CD29E0C44BFB143EC3DD2A
:1002600067D7B63B230352C28E235F27BEC36EFE01
:100270003E3D26DBE1D9C53C00003BC31F26DA2406
:10028000C2C29201423CA1D872DCAE3DDDFC4AC440
:1002900099283D22ECC1B504203B33D619DF713ECD
:1002A000BBF97EC5FA2A8B1F3BC1D507DA39DFD3EC
:1002B000D5E10E3F9CF6D6C6412DC61CB2C0F10A50
:1002C0007138A6D1A3E4843F84F351C86B2FEF1992
:1002D0004FC0050EE5368ACF83E7D33F74F0EEC9F1
:1002E0007931081714C0111136358CCD71EAFB3FF6
:1002F0006CEDADCB6733131400C013146733ADCB73
:100300006CEDFB3F71EA8CCD3635111114C0081726
:100310007931EEC974F0D33F83E78ACFE536050E15
:100320004FC0EF196B2F51C884F3843FA3E4A6D1CB
:100330007138F10AB2C0C61C412DD6C69CF60E3FDC
:10034000D5E1DFD3DA39D5073BC18B1FFA2A7EC549
:10035000BBF9713E19DF33D6203BB504ECC13D2219
:1003600099284AC4DDFCAE3D72DCA1D8423C920122
:10037000C2C2DA241F263BC30000C53CE1D926DBFC
:100380003E3D6EFEBEC35F278E2352C22303B63BA3
:1003900067D7C3DD143E4BFBE0C4CD29E7208FC1F6
:1003A0004506823A06D575E0C53E2BF826C6212CB7
:1003B0002B1EF2C064092A39BFD23AE34E3F0FF533
:1003C0008FC75A2E5D1B7CC07C0CAF3795D011E6D1
:1003D000B13FFBF11BC976307D182DC08C0F123652
:1003E00087CEF8E8EC3FEFEECACA74328F1505C02D
:1003F0009412533499CCEDEB0040EDEB99CC53348F
:10040000941205C08F157432CACAEFEEEC3FF8E8BB
:1004100087CE12368C0F2DC07D1876301BC9FBF1AC
:10042000B13F11E695D0AF377C0C7CC05D1B5A2ED6
:100430008FC70FF54E3F3AE3BFD22A396409F2C0A5
:100440002B1E212C26C62BF8C53E75E006D5823A18
:1004500045068FC1E720CD29E0C44BFB143EC3DD28
:1004600067D7B63B230352C28E235F27BEC36EFEFF
:100470003E3D26DBE1D9C53C00003BC31F26DA2404
:10048000C2C29201423CA1D872DCAE3DDDFC4AC43E
:1004900099283D22ECC1B504203B33D619DF713ECB
:1004A000BBF97EC5FA2A8B1F3BC1D507DA39DFD3EA
:1004B000D5E10E3F9CF6D6C6412DC61CB2C0F10A4E
:1004C0007138A6D1A3E4843F84F351C86B2FEF1990
:1004D0004FC0050EE5368ACF83E7D33F74F0EEC9EF
:1004E0007931081714C0111136358CCD71EAFB3FF4
:1004F0006CEDADCB6733131400C013146733ADCB71
:100500006CEDFB3F71EA8CCD3635111114C0081724
:100510007931EEC974F0D33F83E78ACFE536050E13
:100520004FC0EF196B2F51C884F3843FA3E4A6D1C9
:100530007138F10AB2C0C61C412DD6C69CF60E3FDA
:10054000D5E1DFD3DA39D5073BC18B1FFA2A7EC547
:10055000BBF9713E19DF33D6203BB504ECC13D2217
:1005600099284AC4DDFCAE3D72DCA1D8423C920120
:10057000C2C2DA241F263BC300003E3D72DC67D7AF
:10058000203B45063BC12B1E412D8FC784F3B13F55
:1005900083E787CE3635941200C09412363587CE65
:1005A00083E7B13F84F38FC7412D2B1E3BC1450626
:1005B000203B67D772DC3E3D0000C2C28E239928E3
:1005C000E0C4BBF9C53ED5E1BFD271387C0C4FC049
:1005D0007D187931CACA6CED00406CEDCACA793118
:1005E0007D184FC07C0C7138BFD2D5E1C53EBBF938
:1005F000E0C499288E23C2C200003E3D72DC67D75A
:10060000203B45063BC12B1E412D8FC784F3B13FD4
:1006100083E787CE3635941200C09412363587CEE4
:1006200083E7B13F84F38FC7412D2B1E3BC14506A5
:10063000203B67D772DC3E3D0000C2C28E23992862
:10064000E0C4BBF9C53ED5E1BFD271387C0C4FC0C8
:100650007D187931CACA6CED00406CEDCACA793197
:100660007D184FC07C0C7138BFD2D5E1C53EBBF9B7
:10067000E0C499288E23C2C200003E3D72DC67D7D9
:10068000203B45063BC12B1E412D8FC784F3B13F54
:1006900083E787CE3635941200C09412363587CE64
:1006A00083E7B13F84F38FC7412D2B1E3BC1450625
:1006B000203B67D772DC3E3D0000C2C28E239928E2
:1006C000E0C4BBF9C53ED5E1BFD271387C0C4FC048
:1006D0007D187931CACA6CED00406CEDCACA793117
:1006E0007D184FC07C0C7138BFD2D5E1C53EBBF937
:1006F000E0C499288E23C2C200003E3D72DC67D759
:10070000203B45063BC12B1E412D8FC784F3B13FD3
:1007100083E787CE3635941200C09412363587CEE3
:1007200083E7B13F84F38FC7412D2B1E3BC14506A4
:10073000203B67D772DC3E3D0000C2C28E23992861
:10074000E0C4BBF9C53ED5E1BFD271387C0C4FC0C7
:100750007D187931CACA6CED00406CEDCACA793196
:100760007D184FC07C0C7138BFD2D5E1C53EBBF9B6
:10077000E0C499288E23C2C200003E3D72DC67D7D8
:10078000203B45063BC12B1E412D8FC784F3B13F53
:1007900083E787CE3635941200C09412363587CE63
:1007A00083E7B13F84F38FC7412D2B1E3BC1450624
:1007B000203B67D772DC3E3D0000C2C28E239928E1
:1007C000E0C4BBF9C53ED5E1BFD271387C0C4FC047
:1007D0007D187931CACA6CED00406CEDCACA793116
:1007E0007D184FC07C0C7138BFD2D5E1C53EBBF936
:1007F000E0C499288E23C2C200003E3D72DC67D758
:10080000203B45063BC12B1E412D8FC784F3B13FD2
:1008100083E787CE3635941200C09412363587CEE2
:1008200083E7B13F84F38FC7412D2B1E3BC14506A3
:10083000203B67D772DC3E3D0000C2C28E23992860
:10084000E0C4BBF9C53ED5E1BFD271387C0C4FC0C6
:100850007D187931CACA6CED00406CEDCACA793195
:100860007D184FC07C0C7138BFD2D5E1C53EBBF9B5
:10087000E0C499288E23C2C200003E3D72DC67D7D7
:10088000203B45063BC12B1E412D8FC784F3B13F52
:1008900083E787CE3635941200C09412363587CE62
:1008A00083E7B13F84F38FC7412D2B1E3BC1450623
:1008B000203B67D772DC3E3D0000C2C28E239928E0
:1008C000E0C4BBF9C53ED5E1BFD271387C0C4FC046
:1008D0007D187931CACA6CED00406CEDCACA793115
:1008E0007D184FC07C0C7138BFD2D5E1C53EBBF935
:1008F000E0C499288E23C2C200003E3D72DC67D757
:10090000203B45063BC12B1E412D8FC784F3B13FD1
:1009100083E787CE3635941200C09412363587CEE1
:1009200083E7B13F84F38FC7412D2B1E3BC14506A2
:10093000203B67D772DC3E3D0000C2C28E2399285F
:10094000E0C4BBF9C53ED5E1BFD271387C0C4FC0C5
:100950007D187931CACA6CED00406CEDCACA793194
:100960007D184FC07C0C7138BFD2D5E1C53EBBF9B4
:10097000E0C499288E23C2C20000AE3D19DFDFD348
:100980007138050E14C0131436358ACFA3E40E3F18
:10099000BBF94AC41F265F27E0C42BF84E3F11E67F
:1009A00087CE53348F152DC07C0C2A3906D5C3DD74
:1009B0003E3D9201ECC18B1F412D51C874F0FB3FAD
:1009C0006CEDEEC96B2FC61C3BC1B504423C26DB67
:1009D00067D7823A64097CC07D18743299CCF8E8F4
:1009E000B13F0FF526C6CD298E233BC3DDFC713EFA
:1009F000D5E1A6D1E536111100C01111E536A6D119
:100A0000D5E1713EDDFC3BC38E23CD2926C60FF513
:100A1000B13FF8E899CC74327D187CC06409823A01
:100A200067D726DB423CB5043BC1C61C6B2FEEC921
:100A30006CEDFB3F74F051C8412D8B1FECC192014E
:100A40003E3DC3DD06D52A397C0C2DC08F155334AD
:100A500087CE11E64E3F2BF8E0C45F271F264AC41D
:100A6000BBF90E3FA3E48ACF3635131414C0050E2C
:100A70007138DFD319DFAE3D000052C2E720212CD0
:100A80008FC7FBF1EC3FEDEBCACA76305D1BF2C0BD
:100A90004506B63BE1D9A1D8203BD507B2C0EF1936
:100AA0007931ADCB71EAD33F84F3D6C6FA2A3D2221
:100AB000C2C26EFE143E75E0BFD2AF378C0F05C0C8
:100AC0009412123695D03AE3C53E4BFBBEC3DA24EE
:100AD00099287EC59CF6843F83E78CCD6733081741
:100AE0004FC0F10ADA3933D672DCC53C23038FC11B
:100AF0002B1E5A2E1BC9EFEE0040EFEE1BC95A2EDB
:100B00002B1E8FC12303C53C72DC33D6DA39F10AC0
:100B10004FC0081767338CCD83E7843F9CF67EC5B2
:100B20009928DA24BEC34BFBC53E3AE395D0123672
:100B3000941205C08C0FAF37BFD275E0143E6EFE25
:100B4000C2C23D22FA2AD6C684F3D33F71EAADCBA6
:100B50007931EF19B2C0D507203BA1D8E1D9B63B16
:100B60004506F2C05D1B7630CACAEDEBEC3FFBF1E7
:100B70008FC7212CE72052C20000AE3D19DFDFD322
:100B80007138050E14C0131436358ACFA3E40E3F16
:100B9000BBF94AC41F265F27E0C42BF84E3F11E67D
:100BA00087CE53348F152DC07C0C2A3906D5C3DD72
:100BB0003E3D9201ECC18B1F412D51C874F0FB3FAB
:100BC0006CEDEEC96B2FC61C3BC1B504423C26DB65
:100BD00067D7823A64097CC07D18743299CCF8E8F2
:100BE000B13F0FF526C6CD298E233BC3DDFC713EF8
:100BF000D5E1A6D1E536111100C01111E536A6D117
:100C0000D5E1713EDDFC3BC38E23CD2926C60FF511
:100C1000B13FF8E899CC74327D187CC06409823AFF
:100C200067D726DB423CB5043BC1C61C6B2FEEC91F
:100C30006CEDFB3F74F051C8412D8B1FECC192014C
:100C40003E3DC3DD06D52A397C0C2DC08F155334AB
:100C500087CE11E64E3F2BF8E0C45F271F264AC41B
:100C6000BBF90E3FA3E48ACF3635131414C0050E2A
:100C70007138DFD319DFAE3D000052C2E720212CCE
:100C80008FC7FBF1EC3FEDEBCACA76305D1BF2C0BB
:100C90004506B63BE1D9A1D8203BD507B2C0EF1934
:100CA0007931ADCB71EAD33F84F3D6C6FA2A3D221F
:100CB000C2C26EFE143E75E0BFD2AF378C0F05C0C6
:100CC0009412123695D03AE3C53E4BFBBEC3DA24EC
:100CD00099287EC59CF6843F83E78CCD673308173F
:100CE0004FC0F10ADA3933D672DCC53C23038FC119
:100CF0002B1E5A2E1BC9EFEE0040EFEE1BC95A2ED9
:100D00002B1E8FC12303C53C72DC33D6DA39F10ABE
:100D10004FC0081767338CCD83E7843F9CF67EC5B0
:100D20009928DA24BEC34BFBC53E3AE395D0123670
:100D3000941205C08C0FAF37BFD275E0143E6EFE23
:100D4000C2C23D22FA2AD6C684F3D33F71EAADCBA4
:100D50007931EF19B2C0D507203BA1D8E1D9B63B14
:100D60004506F2C05D1B7630CACAEDEBEC3FFBF1E5
:100D70008FC7212CE72052C20000143ED5E195D048
:100D800036358F154FC06409203BE1D967D7DA3972
:100D90007C0C14C09412E536BFD219DF3E3D23030C
:100DA0003BC15D1B793199CC83E74E3FBBF9BEC394
:100DB0008E23FA2A8FC774F0004074F08FC7FA2A86
:100DC0008E23BEC3BBF94E3F83E799CC79315D1BBF
:100DD0003BC123033E3D19DFBFD2E536941214C058
:100DE0007C0CDA3967D7E1D9203B64094FC08F15F5
:100DF000363595D0D5E1143E0000ECC12B1E6B2F8B
:100E0000CACA71EAB13F9CF6E0C41F26992826C6DB
:100E100084F3EC3F6CED1BC9412DE720C2C2DDFC21
:100E2000C53EA3E487CE67337D18B2C04506423C79
:100E300072DC06D571388C0F00C08C0F713806D566
:100E400072DC423C4506B2C07D18673387CEA3E40E
:100E5000C53EDDFCC2C2E720412D1BC96CEDEC3F55
:100E600084F326C699281F26E0C49CF6B13F71EA98
:100E7000CACA6B2F2B1EECC10000143ED5E195D0E1
:100E800036358F154FC06409203BE1D967D7DA3971
:100E90007C0C14C09412E536BFD219DF3E3D23030B
:100EA0003BC15D1B793199CC83E74E3FBBF9BEC393
:100EB0008E23FA2A8FC774F0004074F08FC7FA2A85
:100EC0008E23BEC3BBF94E3F83E799CC79315D1BBE
:100ED0003BC123033E3D19DFBFD2E536941214C057
:100EE0007C0CDA3967D7E1D9203B64094FC08F15F4
:100EF000363595D0D5E1143E0000ECC12B1E6B2F8A
:100F0000CACA71EAB13F9CF6E0C41F26992826C6DA
:100F100084F3EC3F6CED1BC9412DE720C2C2DDFC20
:100F2000C53EA3E487CE67337D18B2C04506423C78
:100F300072DC06D571388C0F00C08C0F713806D565
:100F400072DC423C4506B2C07D18673387CEA3E40D
:100F5000C53EDDFCC2C2E720412D1BC96CEDEC3F54
:100F600084F326C699281F26E0C49CF6B13F71EA97
:100F7000CACA6B2F2B1EECC10000143ED5E195D0E0
:100F800036358F154FC06409203BE1D967D7DA3970
:100F90007C0C14C09412E536BFD219DF3E3D23030A
:100FA0003BC15D1B793199CC83E74E3FBBF9BEC392
:100FB0008E23FA2A8FC774F0004074F08FC7FA2A84
:100FC0008E23BEC3BBF94E3F83E799CC79315D1BBD
:100FD0003BC123033E3D19DFBFD2E536941214C056
:100FE0007C0CDA3967D7E1D9203B64094FC08F15F3
:100FF000363595D0D5E1143E0000ECC12B1E6B2F89
:10100000CACA71EAB13F9CF6E0C41F26992826C6D9
:1010100084F3EC3F6CED1BC9412DE720C2C2DDFC1F
:10102000C53EA3E487CE67337D18B2C04506423C77
:1010300072DC06D571388C0F00C08C0F713806D564
:1010400072DC423C4506B2C07D18673387CEA3E40C
:10105000C53EDDFCC2C2E720412D1BC96CEDEC3F53
:1010600084F326C699281F26E0C49CF6B13F71EA96
:10107000CACA6B2F2B1EECC10000143ED5E195D0DF
:1010800036358F154FC06409203BE1D967D7DA396F
:101090007C0C14C09412E536BFD219DF3E3D230309
:1010A0003BC15D1B793199CC83E74E3FBBF9BEC391
:1010B0008E23FA2A8FC774F0004074F08FC7FA2A83
:1010C0008E23BEC3BBF94E3F83E799CC79315D1BBC
:1010D0003BC123033E3D19DFBFD2E536941214C055
:1010E0007C0CDA3967D7E1D9203B64094FC08F15F2
:1010F000363595D0D5E1143E0000ECC12B1E6B2F88
:10110000CACA71EAB13F9CF6E0C41F26992826C6D8
:1011100084F3EC3F6CED1BC9412DE720C2C2DDFC1E
:10112000C53EA3E487CE67337D18B2C04506423C76
:1011300072DC06D571388C0F00C08C0F713806D563
:1011400072DC423C4506B2C07D18673387CEA3E40B
:10115000C53EDDFCC2C2E720412D1BC96CEDEC3F52
:1011600084F326C699281F26E0C49CF6B13F71EA95
:10117000CACA6B2F2B1EECC10000713EA3E48CCDBC
:101180007931C61CECC16EFEC53E11E699CC7630B5
:101190002B1E52C2DDFC0E3F83E7ADCB6B2F8B1FA6
:1011A000C2C24BFB4E3FF8E8CACA5A2EE7203BC3E7
:1011B000BBF9843F71EAEEC9412D3D22BEC32BF835
:1011C000B13FEDEB1BC9212C8E234AC49CF6D33FC3
:1011D0006CED51C8FA2ADA24E0C40FF5EC3FEFEECB
:1011E0008FC7CD291F267EC584F3FB3F74F0D6C67A
:1011F00099285F2726C6FBF10040FBF126C65F2732
:101200009928D6C674F0FB3F84F37EC51F26CD29EE
:101210008FC7EFEEEC3F0FF5E0C4DA24FA2A51C88D
:101220006CEDD33F9CF64AC48E23212C1BC9EDEBF9
:10123000B13F2BF8BEC33D22412DEEC971EA843F78
:10124000BBF93BC3E7205A2ECACAF8E84E3F4BFB16
:10125000C2C28B1F6B2FADCB83E70E3FDDFC52C2AA
:101260002B1E763099CC11E6C53E6EFEECC1C61C35
:1012700079318CCDA3E4713E00008FC15D1B7432C7
:1012800087CE3AE3143E92013BC1EF1967338ACF10
:10129000D5E1AE3D2303F2C07D18533495D075E0FF
:1012A0003E3DB504B2C008173635A6D119DFC53C9E
:1012B00045067CC08F151236BFD2C3DD423CD50730
:1012C0004FC01314E536DFD372DCB63B64092DC082
:1012D0009412AF3706D526DB203BF10A14C011115A
:1012E000713833D6E1D9823A7C0C05C08C0F2A398B
:1012F00067D7A1D8DA39050E00C0050EDA39A1D8B2
:1013000067D72A398C0F05C07C0C823AE1D933D6D5
:101310007138111114C0F10A203B26DB06D5AF3716
:1013200094122DC06409B63B72DCDFD3E53613148A
:101330004FC0D507423CC3DDBFD212368F157CC0EB
:101340004506C53C19DFA6D136350817B2C0B5042D
:101350003E3D75E095D053347D18F2C02303AE3D79
:10136000D5E18ACF6733EF193BC19201143E3AE3CE
:1013700087CE74325D1B8FC10000713EA3E48CCD1B
:101380007931C61CECC16EFEC53E11E699CC7630B3
:101390002B1E52C2DDFC0E3F83E7ADCB6B2F8B1FA4
:1013A000C2C24BFB4E3FF8E8CACA5A2EE7203BC3E5
:1013B000BBF9843F71EAEEC9412D3D22BEC32BF833
:1013C000B13FEDEB1BC9212C8E234AC49CF6D33FC1
:1013D0006CED51C8FA2ADA24E0C40FF5EC3FEFEEC9
:1013E0008FC7CD291F267EC584F3FB3F74F0D6C678
:1013F00099285F2726C6FBF10040FBF126C65F2730
:101400009928D6C674F0FB3F84F37EC51F26CD29EC
:101410008FC7EFEEEC3F0FF5E0C4DA24FA2A51C88B
:101420006CEDD33F9CF64AC48E23212C1BC9EDEBF7
:10143000B13F2BF8BEC33D22412DEEC971EA843F76
:10144000BBF93BC3E7205A2ECACAF8E84E3F4BFB14
:10145000C2C28B1F6B2FADCB83E70E3FDDFC52C2A8
:101460002B1E763099CC11E6C53E6EFEECC1C61C33
:1014700079318CCDA3E4713E00008FC15D1B7432C5
:1014800087CE3AE3143E92013BC1EF1967338ACF0E
:10149000D5E1AE3D2303F2C07D18533495D075E0FD
:1014A0003E3DB504B2C008173635A6D119DFC53C9C
:1014B00045067CC08F151236BFD2C3DD423CD5072E
:1014C0004FC01314E536DFD372DCB63B64092DC080
:1014D0009412AF3706D526DB203BF10A14C0111158
:1014E000713833D6E1D9823A7C0C05C08C0F2A3989
:1014F00067D7A1D8DA39050E00C0050EDA39A1D8B0
:1015000067D72A398C0F05C07C0C823AE1D933D6D3
:101510007138111114C0F10A203B26DB06D5AF3714
:1015200094122DC06409B63B72DCDFD3E536131488
:101530004FC0D507423CC3DDBFD212368F157CC0E9
:101540004506C53C19DFA6D136350817B2C0B5042B
:101550003E3D75E095D053347D18F2C02303AE3D77
:10156000D5E18ACF6733EF193BC19201143E3AE3CC
:1015700087CE74325D1B8FC10000C53E83E7CACAA7
:10158000412D8E23E0C484F3004084F3E0C48E2315
:10159000412DCACA83E7C53E00003BC17D183635E0
:1015A000BFD272DC203B7C0C00C07C0C203B72DC88
:1015B000BFD236357D183BC10000C53E83E7CACA9D
:1015C000412D8E23E0C484F3004084F3E0C48E23D5
:1015D000412DCACA83E7C53E00003BC17D183635A0
:1015E000BFD272DC203B7C0C00C07C0C203B72DC48
:1015F000BFD236357D183BC10000C53E83E7CACA5D
:10160000412D8E23E0C484F3004084F3E0C48E2394
:10161000412DCACA83E7C53E00003BC17D1836355F
:10162000BFD272DC203B7C0C00C07C0C203B72DC07
:10163000BFD236357D183BC10000C53E83E7CACA1C
:10164000412D8E23E0C484F3004084F3E0C48E2354
:10165000412DCACA83E7C53E00003BC17D1836351F
:10166000BFD272DC203B7C0C00C07C0C203B72DCC7
:10167000BFD236357D183BC10000C53E83E7CACADC
:10168000412D8E23E0C484F3004084F3E0C48E2314
:10169000412DCACA83E7C53E00003BC17D183635DF
:1016A000BFD272DC203B7C0C00C07C0C203B72DC87
:1016B000BFD236357D183BC10000C53E83E7CACA9C
:1016C000412D8E23E0C484F3004084F3E0C48E23D4
:1016D000412DCACA83E7C53E00003BC17D1836359F
:1016E000BFD272DC203B7C0C00C07C0C203B72DC47
:1016F000BFD236357D183BC10000C53E83E7CACA5C
:10170000412D8E23E0C484F3004084F3E0C48E2393
:10171000412DCACA83E7C53E00003BC17D1836355E
:10172000BFD272DC203B7C0C00C07C0C203B72DC06
:10173000BFD236357D183BC10000C53E83E7CACA1B
:10174000412D8E23E0C484F3004084F3E0C48E2353
:10175000412DCACA83E7C53E00003BC17D1836351E
:10176000BFD272DC203B7C0C00C07C0C203B72DCC6
:10177000BFD236357D183BC10000C53E83E7CACADB
:10178000412D8E23E0C484F3004084F3E0C48E2313
:10179000412DCACA83E7C53E00003BC17D183635DE
:1017A000BFD272DC203B7C0C00C07C0C203B72DC86
:1017B000BFD236357D183BC10000C53E83E7CACA9B
:1017C000412D8E23E0C484F3004084F3E0C48E23D3
:1017D000412DCACA83E7C53E00003BC17D1836359E
:1017E000BFD272DC203B7C0C00C07C0C203B72DC46
:1017F000BFD236357D183BC10000C53E83E7CACA5B
:10180000412D8E23E0C484F3004084F3E0C48E2392
:10181000412DCACA83E7C53E00003BC17D1836355D
:10182000BFD272DC203B7C0C00C07C0C203B72DC05
:10183000BFD236357D183BC10000C53E83E7CACA1A
:10184000412D8E23E0C484F3004084F3E0C48E2352
:10185000412DCACA83E7C53E00003BC17D1836351D
:10186000BFD272DC203B7C0C00C07C0C203B72DCC5
:10187000BFD236357D183BC10000C53E83E7CACADA
:10188000412D8E23E0C484F3004084F3E0C48E2312
:10189000412DCACA83E7C53E00003BC17D183635DD
:1018A000BFD272DC203B7C0C00C07C0C203B72DC85
:1018B000BFD236357D183BC10000C53E83E7CACA9A
:1018C000412D8E23E0C484F3004084F3E0C48E23D2
:1018D000412DCACA83E7C53E00003BC17D1836359D
:1018E000BFD272DC203B7C0C00C07C0C203B72DC45
:1018F000BFD236357D183BC10000C53E83E7CACA5A
:10190000412D8E23E0C484F3004084F3E0C48E2391
:10191000412DCACA83E7C53E00003BC17D1836355C
:10192000BFD272DC203B7C0C00C07C0C203B72DC04
:10193000BFD236357D183BC10000C53E83E7CACA19
:10194000412D8E23E0C484F3004084F3E0C48E2351
:10195000412DCACA83E7C53E00003BC17D1836351C
:10196000BFD272DC203B7C0C00C07C0C203B72DCC4
:10197000BFD236357D183BC100000E3F71EA51C819
:101980009928CD291BC9F8E8C53E9201B2C01314AD
:101990007138A1D806D512367D188FC1DDFC843F81
:1019A0006CEDD6C61F26212CCACA11E6143EB5041A
:1019B0004FC01111DA3926DBBFD253345D1B52C23E
:1019C000BBF9D33F74F07EC58E235A2E99CC3AE3EF
:1019D0003E3DD50714C0050E203BC3DD95D07432C3
:1019E0002B1E3BC39CF6FB3F84F34AC4E7207630B2
:1019F00087CE75E0423CF10A00C0F10A423C75E036
:101A000087CE7630E7204AC484F3FB3F9CF63BC385
:101A10002B1E743295D0C3DD203B050E14C0D507B4
:101A20003E3D3AE399CC5A2E8E237EC574F0D33FC7
:101A3000BBF952C25D1B5334BFD226DBDA39111118
:101A40004FC0B504143E11E6CACA212C1F26D6C6C3
:101A50006CED843FDDFC8FC17D18123606D5A1D810
:101A600071381314B2C09201C53EF8E81BC9CD29E4
:101A7000992851C871EA0E3F0000F2C08F15AF37A8
:101A800067D733D6E53608173BC16EFE4E3FEDEB08
:101A90008FC75F27FA2AEEC983E7713E23037CC014
:101AA00094122A39E1D9DFD33635EF19ECC14BFB5B
:101AB000B13FEFEE26C6DA24412DADCBA3E4AE3D17
:101AC00045062DC08C0F823A72DCA6D16733C61C46
:101AD000C2C22BF8EC3FFBF1E0C43D226B2F8CCD52
:101AE000D5E1C53C640905C07C0CB63B19DF8ACF43
:101AF00079318B1FBEC30FF500400FF5BEC38B1F9E
:101B000079318ACF19DFB63B7C0C05C06409C53C2E
:101B1000D5E18CCD6B2F3D22E0C4FBF1EC3F2BF8DF
:101B2000C2C2C61C6733A6D172DC823A8C0F2DC0AC
:101B30004506AE3DA3E4ADCB412DDA2426C6EFEE3B
:101B4000B13F4BFBECC1EF193635DFD3E1D92A3970
:101B500094127CC02303713E83E7EEC9FA2A5F2703
:101B60008FC7EDEB4E3F6EFE3BC10817E53633D60F
:101B700067D7AF378F15F2C000000E3F71EA51C82A
:101B80009928CD291BC9F8E8C53E9201B2C01314AB
:101B90007138A1D806D512367D188FC1DDFC843F7F
:101BA0006CEDD6C61F26212CCACA11E6143EB50418
:101BB0004FC01111DA3926DBBFD253345D1B52C23C
:101BC000BBF9D33F74F07EC58E235A2E99CC3AE3ED
:101BD0003E3DD50714C0050E203BC3DD95D07432C1
:101BE0002B1E3BC39CF6FB3F84F34AC4E7207630B0
:101BF00087CE75E0423CF10A00C0F10A423C75E034
:101C000087CE7630E7204AC484F3FB3F9CF63BC383
:101C10002B1E743295D0C3DD203B050E14C0D507B2
:101C20003E3D3AE399CC5A2E8E237EC574F0D33FC5
:101C3000BBF952C25D1B5334BFD226DBDA39111116
